:10876800005EBCE2613FDD83C29C7E20A3FD1F4109
:108778009DC3217FFCA2401E5F01E3BD3E6082DCF9
:10878800237D9FC1421CFEA0E1BF5D0380DE3C62E9
:10879800BEE0025CDF81633D7C22C09E1D43A1FFD9
:1087A8004618FAA427799BC584DA3866E5BB5907C9
:1087B800DB856739BAE406581947A5FB7826C49AB9
:1087C800653BD987045AB8E6A7F91B45C6987A24A9
:1087D800F8A6441A99C7257B3A6486D85B05E7B999
:1087E8008CD2306EEDB3510F4E10F2AC2F7193CD89
:1087F800114FADF3702ECC92D38D6F31B2EC0E5079
:10880800AFF1134DCE90722C6D33D18F0C52B0EE68
:10881800326C8ED0530DEFB1F0AE4C1291CF2D7358
:10882800CA947628ABF517490856B4EA6937D58B48
:108838005709EBB536688AD495CB2977F4AA481638
:10884800E9B7550B88D6346A2B7597C94A14F6A828
:10885800742AC896154BA9F7B6E80A54D7896B3518
:10886800FB04FD82FEC1FF60FF96FFB0FFCBFFE572
:04887800FFEEFFF719
:03BD5400011D0AC4
:10C88200901CA3121BC8FFFFFFFF901CA3121B7476
:01C892002283
:10A4240090FFFE121D70ECF0A3EDF090FFFD121DE5
:0AA4340070121C4990FFFC121D700D
:10A43E00851083851182A3A3E4F085108385118294
:10A44E00F0A3F0900007121D94E0FEA3E0FF85102C
:10A45E0083851182E0FCA3E0C39FEE6480F8EC6478
:10A46E0080985051900004121D94121C298510835F
:10A47E00851182E0FEA3E0F5828E83121717FF8509
:10A48E001083851182A3A3E06FFF900003121D9429
:10A49E00EFF0900003121D94E0908768938510836F
:10A4AE00851182A3A3F0851083851182E475F001D6
:0FA4BE00121848808E851083851182A3A3E0FFBA
:07A4CD00900009121D70222E
:0BC4F100901CAFEFF0A3ECF0A3EDF007
:10C4FC00901CB0E0A3E0FF901CAFE0FEEF6E786EF6
:07C50C00F6E690876893FF3B
:01C513002205
:08BCB800901A71EFF0A3EDF00A
:10BCC000901A71E0703DF584759850F58475911562
:10BCD000F58475C908A3E025E02466F582E434887C
:10BCE000F583E493F5CB901A72E025E02467F582A2
:10BCF000E43488F583E493F5CA75C804E4F584D286
:05BD0000ACC2BCD2AF93
:01BD0500221B
:10B66D00901C67121BC800000000901C6B121BC8B9
:10B67D0000000000901C5E7464F0E47812F67812FD
:10B68D00E6C39402748094805043E625E025E024BF
:10B69D005FF582E4341CF583E4F0E625E025E02433
:10B6AD0060F582E4341CF583E4F0E625E025E02422
:10B6BD0061F582E4341CF583E4F0E625E025E02411
:0DB6CD0062F582E4341CF583E4F00680B1E0
:01B6DA00224D
:10C5FF00D2AFD2A9C2BBE4F584E589540F4401F54B
:10C60F0089758E02758CAFE4F58AD28C12B66D22C5
:1083E400E4901C5DF07402F0E4F0F0901C5DE0C3D6
:1083F4009402748094804003028516E025E025E011
:108404002462F582E4341CF583E0D39400748094F0
:108414008050030284E5901C5DE025E025E02460A3
:10842400F582E4341CF583E060030284E5901C5D6E
:10843400E025E025E02462F582E4341CF583E03095
:10844400E027901C5DE025E025E02462F582E43419
:108454001CF583E0D3940174809480400C7D0090DB
:108464001C5DE0FF12A57D800A7D01901C5DE0FF8C
:1084740012A57D901C5DE025E025E02462F582E4F0
:10848400341CF583E06401700A7D01901C5DE0FFFB
:1084940012A57D901C5DE025E025E02462F582E4D0
:1084A400341CF583E014F0901C5DE025E025E02405
:1084B40062F582E4341CF583E06026901C5DE025BF
:1084C400E025E02461F582E4341CF583E0FF901C90
:1084D4005DE025E025E02460F582E4341CF583EFBB
:1084E400F0901C5DE025E025E02460F582E4341C76
:1084F400F583E06014901C5DE025E025E02460F540
:1085040082E4341CF583E014F0901C5DE004F00276
:0285140083EFF3
:018516002242
:03000B0002B056EA
:10B05600C0E0C0F0C083C082C0D0E8C0E0E9C0E074
:10B06600EAC0E0EBC0E0ECC0E0EDC0E0EEC0E0EF2F
:10B07600C0E012C5DE901C67121B74E47B01FAF96E
:10B08600F81219A8901C67121BBC901C5EE014F005
:10B09600E07017901C6B121B74E4F81219A8901C30
:10B0A6006B121BBC901C5E7464F01283E412B94AE6
:10B0B600D0E0FFD0E0FED0E0FDD0E0FCD0E0FBD059
:10B0C600E0FAD0E0F9D0E0F8D0D0D082D083D0F04A
:03B0D600D0E03295
:10BBC30090FFFF121D70EDF090FFFF121D70EFF05C
:10BBD300851083851182E0C3940274809480502D74
:10BBE300A3E0FF851083851182E025E025E0245F33
:10BBF300F582E4341CF583EFF0851083851182A36D
:10BC0300E0FD851083851182E0FF12A57D9000027F
:04BC1300121D70226C
:10A12E0090FFFE121D70EAF0A3EBF090FFFF121DE0
:10A13E0070EDF090FFFF121D70EFF085108385110A
:10A14E0082E0C3940274809480400302A1E6E0256D
:10A15E00E025E02462F582E4341CF583E070798515
:10A16E001083851182E025E025E02460F582E43439
:10A17E001CF583E07062851083851182A3E025E0D3
:10A18E0004FF851083851182E025E025E02462F529
:10A19E0082E4341CF583EFF0851083851182A3A32E
:10A1AE00E0FEA3E0FF7C007D0A1218128510838565
:10A1BE001182E025E025E02461F582E4341CF5836C
:10A1CE00EFF0851083851182E025E025E02460F50F
:0FA1DE0082E4341CF583E4F0900004121D70221B
:10A57D0090FFFF121D70EDF090FFFF121D70EFF0B8
:06A58D0090FFFF121D709B
:10A59300851083851182A3E0C39402748094805054
:10A5A30033851083851182A3E025E025E0245FF540
:10A5B30082E4341CF583E0601B851083851182A33C
:10A5C300A3E070047F0180027F00851083851182E0
:10A5D300A3A3EFF0851083851182E584F075840FC2
:10A5E300851083851182A3E0700F85108385118206
:10A5F300A3A3E024FF92828019851083851182A38F
:10A60300E06401700D851083851182A3A3E024FF0C
:0BA613009283851083851182E0F5849E
:07A61E00900003121D7022E1
:10C7A400C2AF901C67121B74901A5D121BBCD2AFEF
:06C7B400901A5D121B74D7
:01C7BA00225C
:06C4800090FFFC121D708C
:10C48600C2AF901C6B121B74851083851182121B20
:0CC49600BCD2AF851083851182121B748C
:07C4A200900004121D70223E
:10B5FE0090FFFF121D70EFF090FFFF121D7085106F
:10B60E0083851182A3E07005781EF608F6781DE694
:10B61E0075F064A4FF08E6FC08E6C39FEC95F050B5
:01B62E0037E4
:10B62F00851083851182E584F075840175D480E4DB
:10B63F00F58475D103758401AFD2EF9400748094B3
:10B64F008040047F0080027FFF8FD285D2D3851088
:07B65F0083851182E0F584F0
:07B66600900002121D70228A
:10C75900901A82EFF0D209E4781EF608F6E0600438
:09C76900781DF622781D760A22E3
:10C82400C209E4781EF608F6781D76FF75FFDE75FA
:03C83400FFAD2233
:10B94A0090FFFF121D70781F06E618700106781D19
:10B95A00E675F064A4FF08E6FC08E6C39FEC95F0E0
:02B96A00503754
:10B96C00851083851182E584F075840175D480E49B
:10B97C00F58475D103758401AFD2EF940074809473
:10B98C008040047F0080027FFF8FD285D2D3851048
:07B99C0083851182E0F584B0
:07B9A300900001121D70224B
:08C11200901A71EEF0A3EFF0AA
:10C11A00E4A3F0A3F0901A71E0FEA3E0FFA3E0FC11
:10C12A00A3E0C39FEC9E50187FE87E0312AEBD7F4A
:10C13A000112B5FE901A73E475F00112184880D501
:01C14A0022D2
:08AEBD00901A7DEEF0A3EFF006
:0FAEC500901A7DE0FEA3E0D394FAEE9400502A99
:10AED400901A7DE0A3E0F526D3E5269400748094CF
:10AEE400804060752701D3E52794007480948040E6
:0AAEF4000500152780F0152680DE0A
:10AEFE00901A7DE0FEA3E0FFA3EEF0A3EFF0901A10
:10AF0E007FE0FEA3E0D394FAEE940040147FFA7E25
:10AF1E000012AEBD901A7F74FF75F00612184880AD
:10AF2E00DD901A7DE0FEA3E0D39400EE940040097C
:09AF3E00A3E0FEA3E0FF12AEBD8A
:01AF470022E7
:10C69A004D53434246464600323032342D30392D0E
:0DC6AA003039202D203662376130393100E3
:04BD57004100120095
:10955F00E4F584901A82F0A3F0758F04901A82E0DC
:10956F00FEA3E0F5828E83742E93FE742F93B43492
:10957F0007EEB41203D38001C39202E4F58F2002E9
:10958F002F7BFF7AC6799A782D7C057D01122008F2
:10959F00E4900007F0A37450F0A374C2F0A37446D4
:1095AF00F0A374DFF0A374FFF0E4900A56F0805339
:1095BF00758F04901A82E0FEA3E0AA06F97BFF786C
:1095CF002D7C057D01122008901A82E0FEA3E02475
:1095DF0014FFE43EFAA9077BFF78567C0A7D01123F
:1095EF002008901A82E0FEA3E02428FFE43EFAA9A7
:1095FF00077BFF78077C007D017E007F061216D85F
:10960F00E4F58FE4900000F0A3F0C207900541F05D
:10961F00901A35121C29900541E075F010A4F582BF
:10962F0085F083121717D3940074809480400890AC
:07963F000541E004F080D9B1
:019646002201
:06B51C00901A7F121C4989
:10B52200901A7F121C2990002E12189F6434700406
:10B53200E5F0641260037F0022C2AFE4F58412C812
:10B5420024E47812F608F643B701758F0718E6FE71
:10B5520008E6F5828E83E4F0758F05901A7F121C3F
:10B5620029C00218E6FE08E6AA06F8AC027D01D060
:10B57200027E007F301216D853B7FEE4F58FD2AFA9
:0AB582007F0A12C75912955F7F017E
:01B58C00229C
:03002300026086F2
:0D608600C0E0C0F0C083C082C0D075D0085B
:10609300309972C299900004E004F0A3E0FF9000ED
:1060A30004E0C39F5054E0C394047480948050115F
:1060B300E0240DF582E43400F583E06004D29B8094
:0360C30002C29B7B
:1060C600752214D3E52294007480948040177523BA
:1060D60001D3E52394007480948040050015238045
:0560E600F0152280DE30
:1060EB00900004E02449F582E43409F583E0F59946
:1060FB00800BC284900005E4F0900004F030982BE4
:10610B00300628900002E0FEA3E0C3EE9404501981
:10611B00900002E475F00112185EFE744925F0F54B
:10612B008274053EF583E599F0C2982098030262CC
:10613B00F93006030262F9209A0F20080CC29890DE
:10614B000002E4F0A3F00262F9C29A900002E47537
:10615B00F00112185EFE744925F0F58274053EF5C8
:10616B0083E599F0C298900002E0FEA3E064014E33
:10617B00700F900549E07009900002F0A3F00262E5
:10618B00F9900549E05407FF901A57E4F0A3EFF09C
:10619B00901A57E0FEA3E064074E7053900002E0A4
:1061AB00FEA3E0D39401EE9400404490054AE02412
:1061BB0003FFE433901A57F0A3EFF0901A57E0A3C4
:1061CB00E030E735900002E0FEA3E0D39402EE94BA
:1061DB0000402690054AE0547FFEA3E02404FDE432
:1061EB00334EFEEDFF901A57EEF0A3EFF0800A90BE
:1061FB001A57E475F002121848901A57E0FEA3E004
:10620B00FF901A55EEF0A3EFF0900002E0FEA3E032
:10621B00B4000EEEB4040A900002E4F0A3F00262A4
:10622B00F9901A55E0FEA3E0FF900002E0FCA3E01A
:10623B00C39FEC9E50030262F9900002E0FEA3E0C4
:10624B0024FFFDEE34FFFC7B017A05794912A4246F
:10625B00900002E0FCA3E02448F58274053CF58332
:10626B00E06F600A900002E4F0A3F00262F990057F
:10627B0049E064B76005E064BF700BD20090000288
:10628B00E4F0A3F0806830080B7A007B327D017F4D
:10629B000012A12E90052CE004F07B017A097949BC
:1062AB0090FFFD121D70121C497B017A0579491272
:1062BB000026901A57EEF0A3EFF0901A57E0FEA3CA
:1062CB00E0D39400EE940040157A007B327D017F81
:1062DB000112A12E901A57E0A3E0FF12B7B63005BA
:0E62EB000675840075EF10900002E4F0A3F039
:0B62F900D0D0D082D083D0F0D0E032B3
:01C91E0022F6
:06C9080090052CE0FF2267
:10C3A60012B94A900546E0FEA3E0D39400EE94004D
:10C3B600400A90054674FFF5F0121848900546E0CD
:0DC3C600FEA3E04E7006900000F0A3F022F0
:1055C5007BFF7AC679A2901A5D121C49901A5D126A
:1055D5001C291216FEFF3395E04F600C901A5EE40D
:1055E50075F00112184880E47BFF7AC679A2C003E2
:1055F500C002C001901A5D121C29D3D082D083D07D
:10560500E0E99582EA95834019901A5D121C2912EA
:1056150016FE642D600C901A5E74FFF5F0121848A2
:1056250080C6901A5D121C29EB8A8389827BFF7ADA
:10563500C679A2F4700A74A26582700474C6658383
:1056450070030258B3901A5EE475F0021218489080
:105655001A5D121C29900001121717FF3395E0FE01
:10566500C3EF9430EE64809480402D901A5D121C37
:1056750029900001121717FF3395E0FED3EF9439F7
:10568500EE648094805011901A5D121C29900001DF
:1056950012171724D0FF804B901A5D121C29900019
:1056A50001121717FF3395E0FEC3EF9461EE648096
:1056B5009480402D901A5D121C2990000112171735
:1056C500FF3395E0FED3EF9466EE6480948050112D
:1056D500901A5D121C2990000112171724A9FF804A
:1056E500027F00EF7D00FC901A5D121C291216FE48
:1056F500FF3395E0FEC3EF9430EE6480948040273D
:10570500901A5D121C291216FEFF3395E0FED3EFA9
:105715009439EE64809480500E901A5D121C291203
:1057250016FE24D0FF8042901A5D121C291216FE27
:10573500FF3395E0FEC3EF9461EE648094804027CB
:10574500901A5D121C291216FEFF3395E0FED3EF69
:105755009466EE64809480500E901A5D121C291296
:1057650016FE24A9FF80027F00EFC454F04CFCED27
:10577500901A5D121C29900002121717FF3395E04D
:10578500FEC3EF9430EE64809480402D901A5D1234
:105795001C29900002121717FF3395E0FED3EF94F2
:1057A50039EE648094805011901A5D121C29900086
:1057B5000212171724D0FF804B901A5D121C2990F6
:1057C5000002121717FF3395E0FEC3EF9461EE64F4
:1057D500809480402D901A5D121C299000021217AA
:1057E50017FF3395E0FED3EF9466EE648094805006
:1057F50011901A5D121C2990000212171724A9FF97
:1058050080027F00EF75F010A4FFE5F04CFEEF4D30
:10581500FF901A5D121C29900003121717FD33958E
:10582500E0FCC3ED9430EC64809480402D901A5DCB
:10583500121C29900003121717FD3395E0FCD3EDD8
:105845009439EC648094805011901A5D121C299053
:10585500000312171724D0FD804B901A5D121C29E6
:10586500900003121717FD3395E0FCC3ED9461EC2E
:1058750064809480402D901A5D121C2990000312BB
:105885001717FD3395E0FCD3ED9466EC64809480A6
:105895005011901A5D121C2990000312171724A9A4
:0E58A500FD80027D00EEEF4D786CA60608F641
:0158B30022D2
:09630400901A71EFF0A3121C497C
:10630D00901A72121C291216FE64207004D205FF19
:10631D0022901A72121C291216FE64616003026427
:10632D0013901A75121C297478121777901A75121A
:10633D001C299000017405121789786CE6FE08E699
:10634D00EEFF901A75121C29900002EF1217897832
:10635D006CE608E6FF901A75121C29900003EF12E7
:10636D00178912C480901A78121BBC901A78121BD0
:10637D0074EFE4901A75121C29900007EF1217891B
:10638D00901A78121B747808121AE0901A78121B62
:10639D00BC901A78121B74EFE4901A75121C299098
:1063AD000006EF121789901A78121B747808121ACA
:1063BD00E0901A78121BBC901A78121B74EFE490BF
:1063CD001A75121C29900005EF121789901A781270
:1063DD001B747808121AE0901A78121BBC901A7868
:1063ED00121B74EFE4901A75121C29900004EF1221
:1063FD001789901A78121B747808121AE0901A787F
:10640D00121BBC7F0822901A72121C291216FE64F0
:10641D00687055900A56E0FF3395E0FEEF4E602D03
:10642D007B017A0A7956C003C002C001901A72121C
:10643D001C29E92401F9E43AA801FCAD03D001D0EF
:10644D0002D003121F1FEF3395E04F700D901A7598
:10645D00121C297478121777800B901A75121C294B
:10646D0074FF1217777F0122901A72121C291216CF
:10647D00FE6498703E901A72121C29E92401F9E409
:10648D003AFA12B51CEF601D901A75121C2974781A
:10649D00121777901A75121C29900001E4121789B2
:1064AD00D2057F0222901A75121C2974FF121777DC
:1064BD007F0122901A72121C291216FE644160038C
:0364CD000265570E
:1064D000901A71E0FF3395E0FE7C007D3D1217AB12
:1064E000747B2FF974123EFA7B01901A7C121C49BE
:1064F000901A72121C299000011217176401703C47
:10650000901A7C121C29E92404F9E43AFA78427CB6
:10651000057D017E007F041216D8901A7C121C297A
:1065200090000212189FFF900000E5F0F0A3EFF03A
:106530009005467403F0A374E8F0800DE490000029
:10654000F0A3F0900546F0A3F0901A75121C297480
:07655000781217777F01228A
:026557007F00C3
:01655900221F
:08981300901A71EFF0A3EDF0D3
:10981B00E4900002F0A3F0F584FE7F04FD7B017A57
:10982B0000790D1221CF901A72E030E02FE4A3F0F3
:10983B00901A71E0FF901A73E0C39F501FE0C3941E
:10984B0004748094805015E0240DF582E43400F507
:10985B00837401F0901A73E004F080D4901A72E0D4
:10986B0030E53D900949E064107008901A74740259
:10987B00F08006901A747404F0E4901A73F0901A46
:10988B0074E0FF901A73E0C39F5015E0240DF5822E
:10989B00E43400F5837401F0901A73E004F080DE79
:1098AB0090000DE024FF929B901A71E0900005F060
:1098BB00752614D3E5269400748094804017752781
:1098CB0001D3E52794007480948040050015278010
:0598DB00F0152680DEFF
:0F98E000D284900949E0F599E4900004F07F01EB
:0198EF002256
:05B7B600901A59EFF0AC
:10B7BB00E4F584C29BE0900005F0E4900004F09067
:10B7CB001A5AF0901A59E0FFA3E0C39F5014E024DB
:10B7DB000DF582E43400F583E4F0901A5AE004F09E
:02B7EB0080E1FB
:10B7ED00752414D3E5249400748094804017752536
:10B7FD0001D3E525940074809480400500152580C3
:05B80D00F0152480DEAF
:0AB81200D284900949E0F5997F0106
:01B81C002209
:05B81D00901A5FEFF03E
:10B82200E4F584C29BE0900005F0E4900004F090FF
:10B832001A60F0901A5FE0FFA3E0C39F5014E02467
:10B842000DF582E43400F583E4F0901A60E004F030
:02B8520080E193
:10B85400752614D3E52694007480948040177527C8
:10B8640001D3E52794007480948040050015278057
:05B87400F0152680DE46
:0AB87900D284900949E0F5997F019F
:01B8830022A2
:095B6200901A71EFF0A3121C4926
:105B6B00901A71E030E104E4FEFF22901A71E030EC
:105B7B00E20B901A79E4F0A37432F0801D901A7145
:105B8B00E030E30C901A797475F0A37430F0800A4E
:105B9B00901A797401F0A374F4F0E4901A75F0A3E1
:105BAB00F0901A7BF0A3F0901A77F0A3F0901A798B
:105BBB00E0FEA3E0FF901A77E0FCA3E0C39FEC9E0E
:105BCB004003025DDA901A7BE0FEA3E0FF90000237
:105BDB00E0FCA3E09FEC9E4017E4901A77F0A3F053
:105BEB00900002E0FEA3E0FF901A7BEEF0A3EFF033
:105BFB00900949E0641A703E900002E0FEA3E06455
:105C0B00014E7032900549E06478702A7B017A0569
:105C1B007949C003C002C001901A72121C29A80155
:105C2B00AC02AD03D001D002D0037E007F0112166F
:105C3B00D87E007F0122900949E064A1600DE064E9
:105C4B000A704690094DE064A1703E900002E0FEA0
:105C5B00A3E064014E7032900549E06478702A7BB2
:105C6B00017A057949C003C002C001901A72121C57
:105C7B0029A801AC02AD03D001D002D0037E007F76
:105C8B00011216D87E007F0122900949E064A260C0
:105C9B000DE0640A704690094DE064A2703E9000DE
:105CAB0002E0FEA3E064014E7032900549E0647897
:105CBB00702A7B017A057949C003C002C001901A92
:105CCB0072121C29A801AC02AD03D001D002D00383
:105CDB007E007F011216D87E007F0122900002E029
:105CEB00FEA3E0D39400EE94005003025DC1900537
:105CFB0049E0547864786003025DC1E05407FF907B
:105D0B001A75E4F0A3EFF0901A75E0FEA3E06407B8
:105D1B004E7053900002E0FEA3E0D39401EE94008A
:105D2B00404490054AE02403FFE433901A75F0A336
:105D3B00EFF0901A75E0A3E030E735900002E0FE3B
:105D4B00A3E0D39402EE9400402690054AE0547FE2
:105D5B00FEA3E02404FDE4334EFEEDFF901A75EE36
:105D6B00F0A3EFF0800A901A75E475F00212184850
:105D7B00901A75E0FEA3E0FF900002E0FCA3E0B5F3
:105D8B000734ECB50630901A75E0A3E07B017A0579
:105D9B007949C003C002C001901A72121C29A801D4
:105DAB00AC02AD03D001D002D0031216D8901A75F5
:105DBB00E0FEA3E0FF227F0012B5FE7F647E00129F
:105DCB00AEBD901A77E475F001121848025BB890DB
:105DDB001A79E0FEA3E0FF901A77E0FCA3E0B50789
:105DEB0014ECB50610901A72121C2974FF12177757
:085DFB007E007F0122E4FEFF9F
:015E0300227C
:10B15C007B017A1B79CEC002C001E4901A66F0A381
:10B16C00F0A37402F0A37411F0E4A3F07A00791345
:10B17C00A3121C49901A6E7401F0A37413F0D00141
:10B18C00D0027D997C0412A95E901A5DEFF0E0FF6D
:10B19C003395E0FE7C007D3D1217AB747B2FF97468
:10B1AC00123EFA7B01A3121C497A017926C003C016
:10B1BC0002C001901A5E121C2990000E121CF19014
:10B1CC001A5E121C29900011740475F00512197B7B
:01B1DC002250
:067EDC00901A71121C490E
:107EE20090165DE0901A80F0E070057EFF7F9D2283
:107EF200901A80E0640A6005E0640B700990164DE8
:107F0200121B7412938712C31C901A77EFF0E020B1
:107F1200E10302802AE490127DF0A3F0FE7F04FDCB
:107F22007B017A12797F1221CF7E007F107D007B48
:107F3200017A0079131221CF7B017A1A7978124BD8
:107F42006C901A7EEEF0A3EFF07B007A007900C00D
:107F520003C002C001901A78121C29D082D083D0AB
:107F6200E06B7008E965827003EA65837003FEFFC7
:107F720022901A78121C29900013121CC1901A7BAD
:107F8200121C49901A7B121C291218742406FFE451
:107F920035F0FE901A7EE0FCA3E06F7002EE6C609A
:107FA20004E4FEFF22901A7B121C2990000512178E
:107FB2001764056014901A7B121C29900006121790
:107FC2001764616004E4FEFF22901A7B121C299060
:107FD200000212189FFF901A78121C2990002CE5BB
:107FE200F08FF012197B901A78121C29900013124C
:107FF2001CC1C003C002C001901A71121C29121CBC
:1080020072901A78121C2990001C121717FF901AEE
:1080120074121C29EF121777901A78121C299000FB
:0B8022001912189FFFAEF022E4FEFFD1
:01802D002230
:0B90AD00901A71EFF0A3ECF0A3EDF0BF
:1090B800901A71E0C3748094804009E09410748021
:1090C80094804004E4FEFF22901A72E0FEA3E0D3ED
:1090D8009406EE648094844004E4FEFF22901A71A2
:1090E800E075F03DA4247BF9741235F0FA7B019009
:1090F8001A74121C497A017926901A77121C499021
:109108001A77121C299000057405121789901A7293
:10911800E0FEA3E0FF901A77121C29EE8FF01219D7
:109128005C901A74121C2990002C12189FFF901A38
:1091380077121C29900002E5F08FF012197B901A23
:1091480077121C29900004E4121789901A72E0FE25
:10915800A3E02406FFE43EFEA3121C29900011EEB2
:109168008FF012197B901A74121C2912740D901A20
:109178007AEEF0A3EFF0901A7AE0FEA3E0C394062B
:10918800EE94005008901A7AE0A3E0FF22901A7A31
:0B919800E0FEA3E024FAFFEE34FFFE2F
:0191A30022A9
:10C6D400C208C203C205C206E4900002F0A3F0122D
:0CC6E40055C512955F12C55912B15C22B9
:062AB000901A71121C498E
:102AB600901A71121C291216FE5407FF901A7DE413
:102AC600F0A3EFF0901A7DE0FEA3E064074E705786
:102AD600901A71121C2990000112171730E72C90DA
:102AE6001A71121C29900001121717547FFE901AB2
:102AF60071121C29900002121717FDEEED2404FF37
:102B0600E43E901A7DF0A3EFF08026901A71121C15
:102B160029900001121717547F2403FFE433901AFB
:102B26007DF0A3EFF0800A901A7DE475F00212188A
:102B360048901A7DE0FEA3E024FFFDEE34FFFC90F2
:102B46001A71121C2912A424901A71121C29901AA7
:102B56007DE0FCA3E024FFFDEC34FF8D82F58312BB
:102B660017176F6004E4FEFF22E4901A7BF0A3F0CF
:102B7600901A71121C291216FE64B76003022DF119
:102B8600901A7DE0FEA3E024F7FFEE34FFFEE4FC9E
:102B9600FD901A83121BBC901A71121C2990000317
:102BA600121717901A87F0901A71121C29900004B8
:102BB600121717FFE4FCFDFE901A7F121BBC901A39
:102BC60071121C29900005121717FFE4FCFDFEC0C8
:102BD60004C005C006C007901A7F121B747808123D
:102BE6001AF3A804A905AA06AB07D007D006D00594
:102BF600D004121A91901A7F121BBC901A71121CE3
:102C060029900006121717FFE4FCFDFEC004C0055C
:102C1600C006C007901A7F121B747808121AF3A810
:102C260004A905AA06AB07D007D006D005D0041222
:102C36001A91901A7F121BBC901A71121C299000CF
:102C460007121717FFE4FCFDFEC004C005C006C04E
:102C560007901A7F121B747808121AF3A804A905A4
:102C6600AA06AB07D007D006D005D004121A919059
:102C76001A7F121BBC901A7F121B74781C121AE062
:102C8600E4FBFAF9F8C3121ACF6003022DED901A8D
:102C96007F121B74EFEEEDEC540FFC901A7F121BA3
:102CA600BCE4FF12C8C0901A87E0FF12C1BD901A9B
:102CB6007F121B747810121AE0EFEE540FFEE4FD3B
:102CC600FCFBFAF9F8C3121ACF50427F1412AC7407
:102CD600901A7F121B747818121AE0EFE412AC7483
:102CE600901A7F121B747810121AE0EFE412AC747B
:102CF600901A7F121B747808121AE0EFE412AC7473
:102D0600901A7F121B74EFE412AC74804C901A7FF9
:102D1600121B747808121AE0EFE4FEFDFCFBFAF9C8
:102D2600F8C3121ACF50227F1212AC74901A7F1277
:102D36001B747808121AE0EFE412AC74901A7F1232
:102D46001B74EFE412AC7480107F1112AC74901AED
:102D56007F121B74EFE412AC74E4901A79F0A3F0BE
:102D6600901A79E0FEA3E0FFE4FCFD901A83121BA3
:102D760080D3121ACF4029901A71121C29901A7901
:102D8600E0FEA3E02408FFE43E8F82F583121717C6
:102D9600FF12AC74901A79E475F00112184880C0DD
:102DA6007FFF12C1BD7F0112C8C0901A74121C2980
:102DB6007478121777901A83121B74AD07AC0690BD
:102DC6001A71121C29E92408F9E43AFA12A424908B
:102DD6001A74121C29900001EF121789901A7BE4CD
:102DE600F0A37402F08004E4FEFF22901A71121C14
:102DF600291216FE64BF600302311B901A71121C61
:102E060029900002121717FE901A71121C299000C1
:102E160003121717FDEEEDFFEE3395E0FDFC901A59
:102E260083121BBC901A71121C29900004121717EA
:102E3600901A87F0901A71121C2990000512171724
:102E4600FFE4FCFDFE901A7F121BBC901A71121C47
:102E560029900006121717FFE4FCFDFEC004C0050A
:102E6600C006C007901A7F121B747808121AF3A8BE
:102E760004A905AA06AB07D007D006D005D00412D0
:102E86001A91901A7F121BBC901A71121C2990007D
:102E960007121717FFE4FCFDFEC004C005C006C0FC
:102EA60007901A7F121B747808121AF3A804A90552
:102EB600AA06AB07D007D006D005D004121A919007
:102EC6001A7F121BBC901A71121C29900008121747
:102ED60017FFE4FCFDFEC004C005C006C007901A3B
:102EE6007F121B747808121AF3A804A905AA06AB68
:102EF60007D007D006D005D004121A91901A7F1277
:102F06001BBC901A83121B74EF2404FBE43EFAE404
:102F16003DF9E43CF8901A77E0FEA3E0FFEE339526
:102F2600E0FDFCD3121ACF4004E4FEFF22901A8380
:102F3600121B747D00901A74121C29E92403F9E40B
:102F46003AFA1221CF901A7F121B74781C121AE0DB
:102F5600E4FBFAF9F8C3121ACF6003023117901A8C
:102F66007F121B74EFEEEDEC540FFC901A7F121BD0
:102F7600BCE4FF12C8C0901A87E0FF12C1BD901AC8
:102F86007F121B747810121AE0EFEE540FFEE4FD68
:102F9600FCFBFAF9F8C3121ACF50427F2412AC7424
:102FA600901A7F121B747818121AE0EFE412AC74B0
:102FB600901A7F121B747810121AE0EFE412AC74A8
:102FC600901A7F121B747808121AE0EFE412AC74A0
:102FD600901A7F121B74EFE412AC74804C901A7F27
:102FE600121B747808121AE0EFE4FEFDFCFBFAF9F6
:102FF600F8C3121ACF50227F2212AC74901A7F1295
:103006001B747808121AE0EFE412AC74901A7F125F
:103016001B74EFE412AC7480107F2112AC74901A0A
:103026007F121B74EFE412AC74901A83121B74EFB8
:10303600E412AC74E4901A79F0A3F0901A79E0FEE9
:10304600A3E0FFE4FCFD901A83121B80D3121ACF73
:10305600402912A8BB901A74121C29901A79E0FC18
:10306600A3E02403FDE43C8D82F583EF12178990DB
:103076001A79E475F00112184880C07FFF12C1BDAD
:103086007F0112C8C0901A74121C29747F12177718
:10309600901A83121B747808121AE0EF547FFFE42B
:1030A600EF4480FFE4901A74121C29900001EF127D
:1030B6001789901A83121B74EFE4901A74121C2954
:1030C600900002EF121789901A83121B74EF2403E3
:1030D600FDE43EFC901A74121C2912A424C0079029
:1030E6001A83121B74EF2403FFE43EFE901A741237
:1030F6001C298F828E83D007EF121789901A8312AC
:103106001B74EF2404FFE43E901A7BF0A3EFF080DB
:0D31160004E4FEFF22901A7BE0FEA3E0FF20
:013123002289
:10BC17007B017A057949C002C0017A097949901AEE
:10BC270074121C49901A777401F0A3740DF0D001B7
:10BC3700D002122AB0901A5DEEF0A3EFF0901A5DD1
:10BC4700E0FEA3E0D39400EE940040157A007B3227
:10BC57007D017F0112A12E901A5DE0A3E0FF12B8CB
:01BC67001DBF
:01BC680022B9
:0F00260090FFFD121D70121C4990FFF2121D7009
:1000350090000E121D94121C291216FE5407FF7E05
:1000450000900005121D94EEF0A3EFF0900005124C
:100055001D94E0FEA3E064074E707090000E121D23
:1000650094121C2990000112171730E73A90000EE0
:10007500121D94121C29900001121717547F7F003E
:10008500FE90000E121D94121C29900002121717E3
:10009500FDEEEF4D2404FFE43EFE900005121D9495
:1000A500EEF0A3EFF0803190000E121D94121C2982
:1000B500900001121717547F2403FFE433FE9000CC
:1000C50005121D94EEF0A3EFF0800D900005121DB2
:1000D50094E475F002121848900005121D94E0FE94
:1000E500A3E024FFFDEE34FFFC90000E121D9412D8
:1000F5001C2912A42490000E121D94121C29900094
:1001050005121D94E0FCA3E024FFFDEC34FF8D8275
:10011500F5831217176F6006E4FEFF02122B90009D
:1001250003121D94E4F090000E121D94121C291266
:1001350016FE121D4A01650A023B1001E712016510
:100145001A025120025628042A2907113307D537E8
:1001550008475008E561064A7008E1980000093C27
:1001650090000E121D94121C299000011217177F82
:1001750000FE90000E121D94121C29900002121709
:1001850017FDEEEF4DFF901A3CE0FCA3E06F700207
:10019500EE6C7044D20890000604F07A007B32FDC4
:1001A5007F0012A12E90000E121D94121C2912160A
:1001B500FE641A600302093C900011121D94121C82
:1001C50029900003121D94E0FF04F08F82758300CF
:1001D500747812178902093CC208E4900006F002FF
:1001E500093C90000E121D94121C29900001121753
:1001F500177F00FE90000E121D94121C299000021C
:10020500121717FDEEEF4DFF901A3EE0FCA3E0B587
:10021500071AEEB50416D2089000067402F07A00AB
:100225007B327D017F0012A12E02093CC208E490B9
:100235000006F002093CD2089000067403F07A002B
:100245007B327D017F0012A12E02093CD2050209F5
:100255003C900011121D94121C29900003121D944C
:10026500E0FF04F08F82758300747F121789900078
:1002750011121D94121C29900003121D94E0FF0415
:10028500F08F827583007418121789900011121D62
:1002950094121C29900003121D94E0FF04F08F8234
:1002A5007583007405121789900541E0FF900011D0
:1002B500121D94121C29900003121D94E0FE04F0F7
:1002C5008E82758300EF121789901A3CE0FEA3E039
:1002D500EEFF900011121D94121C29900003121DAF
:1002E50094E0FE04F08E82758300EF121789901A50
:1002F5003CE0A3E0FF900011121D94121C29900010
:1003050003121D94E0FE04F08E82758300EF121730
:1003150089901A3EE0FEA3E0EEFF900011121D94B5
:10032500121C29900003121D94E0FE04F08E8275C4
:100335008300EF121789901A3EE0A3E0FF900011A9
:10034500121D94121C29900003121D94E0FE04F066
:100355008E82758300EF121789786CE6FE08E6EE4B
:10036500FF900011121D94121C29900003121D9478
:10037500E0FE04F08E82758300EF121789786CE633
:1003850008E6FF900011121D94121C29900003121B
:100395001D94E0FE04F08E82758300EF12178985A7
:1003A5001083851182E4F0851083851182E0C39462
:1003B50010748094805033E02440F582E4341AF5BB
:1003C50083E0FF900011121D94121C299000031266
:1003D5001D94E0FE04F08E82758300EF1217898567
:1003E5001083851182E004F080BD900003121D94F6
:1003F500E0FD7C00900011121D94121C2912A4240A
:10040500900011121D94121C29900003121D94E0F6
:10041500F582758300EF121789900003121D94E091
:1004250004F002093C90000E121D94121C29900044
:1004350001121717FF900541E0FEEFC39E4003022E
:0204450006208F
:1004470090000E121D94121C2990000112171775A7
:10045700F010A4FF901A35121C29E92FF9EA35F09C
:10046700FA90000B121D94121C49900011121D9452
:10047700121C29900003121D94E0FF04F08F82756F
:100487008300747F121789900011121D94121C2982
:10049700900003121D94E0FF04F08F8275830074AF
:1004A7000D12178990000B121D94121C291216FEAB
:1004B700FF900011121D94121C29900003121D9425
:1004C700E0FE04F08E82758300EF12178990000B0F
:1004D700121D94121C29900001121717FF9000118A
:1004E700121D94121C29900003121D94E0FE04F0C3
:1004F7008E82758300EF12178990000B121D9412DC
:100507001C29900002121717FF900011121D941258
:100517001C29900003121D94E0FE04F08E8275835F
:1005270000EF12178990000B121D94121C299000DE
:1005370003121717FF900011121D94121C29900027
:1005470003121D94E0FE04F08E82758300EF1217EC
:100557008990000B121D94121C2990000412171782
:10056700FF900011121D94121C29900003121D9474
:10057700E0FE04F08E82758300EF121789851083E1
:10058700851182E4F0851083851182E0C394087495
:10059700809480504990000B121D94121C29E92465
:1005A70005F9E43AFA851083851182E07E0029F97E
:1005B700EE3AFA1216FEFF900011121D94121C2932
:1005C700900003121D94E0FE04F08E82758300EF05
:1005D700121789851083851182E004F080A79000A7
:1005E70003121D94E0FD7C00900011121D94121C53
:1005F7002912A424900011121D94121C29900003A3
:10060700121D94E0F582758300EF1217899000039D
:06061700121D94E004F046
:10061D0002093C900011121D94121C2974781217B6
:10062D0077900011121D94121C29900001E41217ED
:10063D0089900003121D947402F002093C12C480CB
:10064D00900007121D94121BBC900011121D9412E4
:10065D001C29747C121777900007121D94E0FF90EF
:10066D000011121D94121C29900001EF1217897BA5
:10067D0001900007121D94A982AA83900001121700
:10068D0017FF900011121D94121C29900002EF12F9
:10069D0017897B01900007121D94A982AA839000EF
:1006AD0002121717FF900011121D94121C299000B1
:1006BD0003EF1217897B01900007121D94A982AADE
:1006CD0083900003121717FF900011121D94121C36
:1006DD0029900004EF1217897C007D0590001112FE
:1006ED001D94121C2912A424900011121D94121C89
:1006FD0029900005EF121789900003121D947406BE
:10070D00F002093C90000E121D94121C299000015C
:10071D001217176401703090000E121D94121C29CF
:10072D009000021217177F00FE90000E121D9412FA
:10073D001C29900003121717FDEEEF4DFF901A3C88
:10074D00EEF0A3EFF0807C90000E121D94121C2988
:10075D009000011217176402702890000E121D945C
:10076D00121C29900002121717FF7F0090000E1225
:10077D001D94121C299000031217174F901A3CF06C
:10078D00804190000E121D94121C29900001121729
:10079D00176403702E90000E121D94121C299000E8
:1007AD00021217177F00FE90000E121D94121C29C5
:1007BD00900003121717FDEEEF4DFF901A3EEEF06D
:1007CD00A3EFF0D20402093C851083851182E4F079
:1007DD00851083851182E0C39410748094805050ED
:1007ED0090000E121D94121C29900001121717FF74
:1007FD00851083851182E0C39F5035E02402FFE40C
:10080D0033FE90000E121D94121C298F828E8312BE
:10081D001717FF851083851182E02440F582E4349B
:10082D001AF583EFF0851083851182E004F080A026
:10083D00E4901A4FF0D20402093C20064D900011AD
:10084D00121D94121C297479121777900011121D24
:10085D0094121C2990000174011217897C007D02ED
:10086D00900011121D94121C2912A4249000111233
:10087D001D94121C29900002EF121789900003128B
:10088D001D947403F0D20302093C900011121D94C3
:10089D00121C297479121777900011121D94121CD5
:1008AD002990000174021217897C007D02900011BD
:1008BD00121D94121C2912A424900011121D9412C1
:1008CD001C29900002EF121789900003121D9474D9
:1008DD0003F0805BD2048057900011121D94121CFE
:1008ED0029747912177790000E121D94121C2990FD
:1008FD000001121717FF900011121D94121C299060
:10090D000001EF1217897C007D02900011121D94D9
:10091D00121C2912A424900011121D94121C29904E
:10092D000002EF121789900003121D947403F090CA
:10093D00000E121D94121C291216FE54F864A060AC
:10094D0003020EE190000E121D94121C291216FEC8
:10095D0064A16003020C0590000E121D94121C2957
:10096D00900001121717FF900004121D94EFF090E4
:10097D000541E0FF900004121D94E0C39F40030267
:10098D000BEB901A35121C29900004121D94E07582
:10099D00F010A4F58285F083121717FF9000031253
:1009AD001D94EFF0900004121D94E075F010A4FF5B
:1009BD00901A35121C29E92FF9EA35F0FA90000446
:1009CD0012171720E203020A64900011121D9412EF
:1009DD001C29747F121777900011121D94121C2977
:1009ED00E92402F9E43AFA900004121D94E0FF1292
:1009FD009D30900003121D94EFF0900003121D9492
:100A0D00E0FF900011121D94121C29900001EF12AD
:100A1D001789900003121D94E02402F09000031238
:100A2D001D94E0FD7C00900011121D94121C2912E2
:100A3D00A424900011121D94121C29900003121D64
:100A4D0094E0F582758300EF121789900003121D53
:100A5D0094E004F0020EE1900003121D94E0D39493
:100A6D0006748094805003020B1D900011121D948A
:100A7D00121C29747F121777900003121D94E0FF4A
:100A8D00900011121D94121C29900001EF1217896C
:100A9D00851083851182E4F0900003121D94E0FF10
:100AAD00851083851182E0C39F5058900004121D5C
:100ABD0094E075F010A4FF901A35121C29E92FF956
:100ACD00EA35F0FA90000D121CC185108385118254
:100ADD00E0F582758300121717FF8510838511824B
:100AED00E02402FDE433FC900011121D94121C2928
:100AFD008D828C83EF121789851083851182E00416
:100B0D00F08095900003121D94E02402F0020BB0CA
:100B1D00900003121D94E02478FF900011121D9493
:100B2D00121C29EF121777851083851182E4F0903E
:100B3D000003121D94E0FF851083851182E0C39F91
:100B4D005058900004121D94E075F010A4FF901AF7
:100B5D0035121C29E92FF9EA35F0FA90000D121C17
:100B6D00C1851083851182E0F582758300121717F8
:100B7D00FF851083851182E02401FDE433FC900094
:100B8D0011121D94121C298D828C83EF12178985E9
:100B9D001083851182E004F08095900003121D945E
:100BAD00E004F0900003121D94E0FD7C0090001114
:100BBD00121D94121C2912A424900011121D9412BE
:100BCD001C29900003121D94E0F582758300EF122D
:100BDD001789900003121D94E004F0020EE19000BD
:100BED0011121D94121C297478121777900003129C
:100BFD001D947401F0020EE190000E121D94121C52
:100C0D00291216FE64A26003020EE190000E121D61
:100C1D0094121C29900001121717FF900541E0FE58
:100C2D00EFC39E4003020ECA90000E121D94121CBB
:100C3D0029900002121717FF900541E0FEEFC39EA9
:100C4D004003020ECA90000E121D94121C29900032
:100C5D0002121717FF90000E121D94121C299000FE
:100C6D0001121717D39F4003020ECA90000E121DDA
:100C7D0094121C299000011217178510838511827B
:100C8D00F0A3A3E4F090000E121D94121C29900005
:100C9D0002121717FF851083851182E0D39F503004
:100CAD00901A35121C29851083851182E075F0107C
:100CBD00A4F58285F083121717FF851083851182A5
:100CCD00A3A3E02FF0851083851182E004F080B599
:100CDD00900003121D94E4F0900011121D94121C4B
:100CED0029900003121D94E0FF04F08F827583009C
:100CFD00747F121789851083851182A3A3E0C39495
:100D0D0080748094805028851083851182A3A3E080
:100D1D00FF900011121D94121C29900003121D94B6
:100D2D00E0FE04F08E82758300EF121789804F85E7
:100D3D001083851182A3A3E0E47480FF900011124B
:100D4D001D94121C29900003121D94E0FE04F08ED8
:100D5D0082758300EF121789851083851182A3A3F5
:100D6D00E0FF900011121D94121C29900003121D1A
:100D7D0094E0FE04F08E82758300EF1217899000C7
:100D8D000E121D94121C2990000112171785108345
:100D9D00851182F090000E121D94121C29900002F4
:100DAD00121717FF851083851182E0D39F40030230
:100DBD000E90A3E4F0901A35121C2985108385112D
:100DCD0082E075F010A4F58285F083121717FF8568
:100DDD001083851182A3E0C39F4003020E8485100A
:100DED0083851182E075F010A4FF901A35121C292D
:100DFD00E92FF9EA35F0FA90000412171730E21EC8
:100E0D00900011121D94121C29900003121D94E0E4
:100E1D00FF04F08F82758300E4121789804C8510D2
:100E2D0083851182E075F010A4FF901A35121C29EC
:100E3D00E92FF9EA35F0FA90000D121CC1851083E7
:100E4D00851182A3E0F582758300121717FF9000BC
:100E5D0011121D94121C29900003121D94E0FE0422
:100E6D00F08E82758300EF121789851083851182AC
:100E7D00A3E004F0020DC2851083851182E004F019
:100E8D00020DA1900003121D94E0FD7C0090001155
:100E9D00121D94121C2912A424900011121D9412DB
:100EAD001C29900003121D94E0F582758300EF124A
:100EBD001789900003121D94E004F0801790001123
:100ECD00121D94121C297478121777900003121DAD
:100EDD00947401F090000E121D94121C291216FE2E
:100EED0054F86480601590000E121D94121C291286
:100EFD0016FE54F86488600302122190000E121D34
:100F0D0094121C291216FE5407FF900003121D9413
:100F1D00EFF0900003121D94E06407703B85108381
:100F2D00851182A304F090000E121D94121C2990BD
:100F3D000001121717FF900003121D94EFF090009F
:100F4D000E121D94121C29900002121717FF90000B
:100F5D0004121D94EFF08021851083851182A3E486
:100F6D00F090000E121D94121C29900001121717FB
:100F7D00FF900004121D94EFF0900003121D94E0F9
:100F8D0014F0900541E0FF900004121D94E0C39F02
:100F9D004003021221901A35121C29900004121DD3
:100FAD0094E075F010A4F58285F083121717FF9069
:100FBD000003121D94E0D39F4022901A35121C2974
:100FCD00900004121D94E075F010A4F58285F08355
:100FDD00121717FF900003121D94EFF085108385F3
:100FED001182E4F0900003121D94E0FF85108385BB
:100FFD001182E0C39F40030211B3900004121D94AF
:10100D00E075F010A4FF901A35121C29E92FF9EAAA
:10101D0035F0FA90000412171730E2030211A79071
:10102D000004121D94E075F010A4FF901A35121CE7
:10103D0029E92FF9EA35F0FA9000011217176438F3
:10104D006003021125900003121D94E0D3940474E3
:10105D00809480405F851083851182A3E02402FF78
:10106D00E433FE851083851182E07C002FFFEC3E7A
:10107D00FE90000E121D94121C298F828E83121762
:10108D0017FD900004121D94E075F010A4FF901A46
:10109D0035121C29E92FF9EA35F0FA90000D121CD2
:1010AD00C1851083851182E0F582758300ED1217DD
:1010BD00890211A7900005121D94E0FEA3E024FE05
:1010CD00FFEE34FFFE851083851182E0FDC3EF9D99
:1010DD00FFEE9400FE90000E121D94121C298F82BB
:1010ED008E83121717FD900004121D94E075F010F9
:1010FD00A4FF901A35121C29E92FF9EA35F0FA9060
:10110D00000D121CC1851083851182E0F582758357
:10111D0000ED1217890211A7901A35121C299000A3
:10112D0004121D94E075F010A4F58285F08312175A
:10113D0017FF7E00900005121D94E0FCA3E024FF34
:10114D00FDEC34FFFCC3ED9FFFEC9EFE8510838507
:10115D001182E07C002FFFEC3EFE90000E121D94DC
:10116D00121C298F828E83121717FD900004121DF9
:10117D0094E075F010A4FF901A35121C29E92FF98F
:10118D00EA35F0FA90000D121CC18510838511828D
:10119D00E0F582758300ED12178985108385118224
:1011AD00E004F0020FF190000E121D94121C299014
:1011BD000004121D94E0FF129EDB90000E121D9490
:1011CD00121C291216FE54F86488704890001112F2
:1011DD001D94121C29747812177790000E121D940D
:1011ED00121C29900005121D94E0FEA3E024FFFFC0
:1011FD00EE34FF8F82F583121717FF900011121D29
:10120D0094121C29900001EF121789900003121DF2
:0E121D00947402F0900003121D94E0FF7E0016
:07122B00900014121D702257
:1031240012C90EEF4E60142007117B007A0079005B
:103134007F807EF47DFF7CFF12C1F290165DE06417
:1031440009700B12C90EEF4E6004D2078002C20749
:10315400300719900012E070137D01FF12BBC37D8C
:10316400017F0012A57D9000127401F020071990D0
:103174000012E060137D007F0012BBC37D017F005D
:1031840012A57DE4900012F07B017A1A795DC002E9
:10319400C0017A1A796D901A74121C49D001D002B8
:1031A400127EDC901A69EEF0A3EFF0D39400EE9453
:1031B400005003023659901A5D121C29901A6E129F
:1031C4001C497B017A01792C901A60121C499000E9
:1031D40000E0FEA3E04E605D901A6DE0FF3395E0E1
:1031E400FE90127D75F03DEF121C1DEE75F03DA4AE
:1031F4002583F583E0FEA3E0FF900000E0FCA3E05C
:103204006F7002EC6E6003023669901A6DE0FF3352
:1032140095E0FE7C007D3D1217AB747F2FF974128C
:103224003EFA78427C057D017E007F041221ABEFDB
:103234006003023669900000E0FEA3E04E606790F0
:103244001A6DE0FF3395E0FE90127D75F03DEF12AC
:103254001C1DEE75F03DA42583F583E0FEA3E0FF7D
:10326400900000E0FCA3E06F7002EC6E7038901ADE
:103274006DE0FF3395E0FE7C007D3D1217AB747F5B
:103284002FF974123EFA7B0178427C057D017E00A1
:103294007F041221ABEF3395E04F700A900546741A
:1032A40003F0A374E8F0901A69E0FEA3E0D394134A
:1032B400EE94014003023669901A6E121C29E92427
:1032C40006F9E43AFA901A65121C49901A6E121C17
:1032D400299000041217175410D39400748094801A
:1032E40040047F0180027F00901A64EFF0901A6E10
:1032F400121C29121874FF901A6BE5F0F0A3EFF07A
:10330400901A6E121C29900004121717901A63F079
:10331400901A6BE0FEA3E02406FFE43EFE901A69D7
:10332400E0FCA3E06F7002EE6C6003023669901A51
:103334006E121C2990000512171764056010901A6C
:1033440065121C291216FE646160030236697A0054
:103354007B327D017F0012A12E901A64E0605390AD
:103364001A6DE0FF901A65121C29C003C002C00147
:10337400901A60121C29901A75121C49D001D002AF
:10338400D003126304901A69E4F0A3EFF0901A6971
:10339400E0FEA3E0D39400EE94005003023659906B
:1033A4001A6DE0FF901A69E0FCA3E0FD1290AD02F3
:1033B4003659901A65121C291216FE64B7600D90D6
:1033C4001A65121C291216FE64BF7055901A6512F4
:1033D4001C29C003C002C001901A60121C29901A53
:1033E40074121C49901A777404F0A3E4F0D001D04D
:1033F40002D003122AB0901A69EEF0A3EFF0901AEB
:1034040069E0FEA3E0D39400EE9400500302366911
:10341400901A6DE0FF901A69E0FCA3E0FD1290ADF4
:1034240022901A60121C2990FFFD121D70121C4973
:10343400901A65121C29120026901A69EEF0A3EF67
:10344400F0901A69E0FEA3E0D39400EE94004010DB
:10345400901A6DE0FF901A69E0FCA3E0FD1290ADB4
:1034640020080302354C901A65121C291216FE54CA
:10347400072402901A68F0E0FF901A6BE0FCA3E0C6
:10348400D39FEC9400500302354C901A68E0901AD4
:1034940066E48FF0121848D206901A65121C29129D
:1034A40016FE64B7600D901A65121C291216FE648C
:1034B400BF7054901A65121C29C003C002C0019049
:1034C4001A60121C29901A74121C49901A777404F9
:1034D400F0A3E4F0D001D002D003122AB0901A690C
:1034E400EEF0A3EFF0901A69E0FEA3E0D39400EEAF
:1034F40094004010901A6DE0FF901A69E0FCA3E07C
:10350400FD1290ADC20622901A60121C2990FFFD94
:10351400121D70121C49901A65121C291200269063
:103524001A69EEF0A3EFF0901A69E0FEA3E0D394D9
:1035340000EE94004010901A6DE0FF901A69E0FCD0
:10354400A3E0FD1290ADC2063008030235FD901AC7
:103554006BE0FEA3E0FF901A65121C2978497C09F0
:103564007D011216D8D206901A6BE0A3E0FF901AE0
:1035740063E0FD129813EF607C900005E060077F24
:103584000012B5FE80F3901A63E0FF901A60121CDB
:1035940029125B62901A69EEF0A3EFF0901A69E0C9
:1035A400FEA3E0D39400EE94004032901A69E0A3A5
:1035B400E064014E700C901A60121C291216FEF47D
:1035C400600B7A007B327D017F0112A12E901A6D6F
:1035D400E0FF901A69E0FCA3E0FD1290AD90094968
:1035E400E06410701090094BE064397008A3E0FDAA
:1035F400E4FF12BCB8C206805C900006E06402607E
:1036040005E06403704F901A6BE0FEA3E0FF901A8C
:1036140065121C2978497C097D011216D8D20690BE
:103624001A6BE0A3E0FF901A63E0FD129813900078
:1036340005E060077F0012B5FE80F3900949E0645D
:1036440010701090094BE064397008A3E0FDE4FFAA
:1036540012BCB8C20630050D7F647E0012C112E4AC
:05366400F58475EF1074
:01366900223E
:10C7BB0075840FC2E8C2E9C2EAD2DBD2D9D2DAC29F
:06C7CB00ECC2EED2EB22ED
:10C25A00901A91EFF0A3EDF075840FE0701BC2D92C
:10C26A00901A91E01392E8E0FFC313F0E01392E909
:10C27A00E0FFC313F0E01392EA901A92E024FF92CF
:02C28A00DA22B6
:05BECC00901CBBEFF02B
:10BED10075840FE4A3F0901CBCE0C39408748094B3
:10BEE10080502A901CBBE0540194007480948040DF
:10BEF10003D38001C392D9901CBBE0FFC313F0D2DE
:0FBF0100DBD2DBD2DBC2DBA3E004F080C9C2D904
:01BF1000220E
:05ABDC00901A91EFF05A
:10ABE10075840FE0F526E5263392D9E52625E0F5B3
:10ABF10026D2DBD2DBD2DBC2DB3392D9E52625E0DC
:10AC0100F526D2DBD2DBD2DBC2DB3392D9E52625B6
:10AC1100E0F526D2DBD2DBD2DBC2DB3392D9E526EB
:10AC210025E0F526D2DBD2DBD2DBC2DB3392D9E5DC
:10AC31002625E0F526D2DBD2DBD2DBC2DB3392D98B
:10AC4100E52625E0F526D2DBD2DBD2DBC2DB33926F
:10AC5100D9E52625E0F526D2DBD2DBD2DBC2DB3318
:10AC610092D9E52625E0F526D2DBD2DBD2DBC2DBA9
:02AC7100C2D946
:01AC730022BE
:10A8180075840FE4901A6BF0E0FF25E0FFA2D8E4FE
:10A82800334FF0D2DBD2DBD2DBC2DBE0FF25E0FF27
:10A83800A2D8E4334FF0D2DBD2DBD2DBC2DBE0FFBD
:10A8480025E0FFA2D8E4334FF0D2DBD2DBD2DBC263
:10A85800DBE0FF25E0FFA2D8E4334FF0D2DBD2DB08
:10A86800D2DBC2DBE0FF25E0FFA2D8E4334FF0D211
:10A87800DBD2DBD2DBC2DBE0FF25E0FFA2D8E4338A
:10A888004FF0D2DBD2DBD2DBC2DBE0FF25E0FFA258
:10A89800D8E4334FF0D2DBD2DBD2DBC2DBE0FF25DA
:10A8A800E0FFA2D8E4334FF0D2DBD2DBD2DBC2DB4D
:02A8B800E0FFBF
:01A8BA00227B
:10C57B00901CBDEFF0A3EDF0901CBDE0FFE4FD12AD
:10C58B00C25A901CBEE0FF12BECC0DE4FF12C25A81
:01C59B00227D
:10C59C00901CBFEFF0A3EDF0901CBFE0FFE4FD1288
:10C5AC00C25A901CC0E0FF12ABDC0DE4FF12C25A61
:01C5BC00225C
:0EC8C000901A88EFF075840FE024FF92EB22AF
:05BF1100901CC1EFF0DF
:10BF160075840FE4A3F0901CC2E0C3940874809467
:10BF260080502A901CC1E054019400748094804093
:10BF360003D38001C392EE901CC1E0FFC313F0D27D
:0FBF4600ECD2ECD2ECC2ECA3E004F080C9C2EE66
:01BF550022C9
:05AC7400901A88EFF0CA
:10AC790075840FE0F526E5263392EEE52625E0F505
:10AC890026D2ECD2ECD2ECC2EC3392EEE52625E0EA
:10AC9900F526D2ECD2ECD2ECC2EC3392EEE52625C5
:10ACA900E0F526D2ECD2ECD2ECC2EC3392EEE526FA
:10ACB90025E0F526D2ECD2ECD2ECC2EC3392EEE5EB
:10ACC9002625E0F526D2ECD2ECD2ECC2EC3392EE9A
:10ACD900E52625E0F526D2ECD2ECD2ECC2EC339293
:10ACE900EEE52625E0F526D2ECD2ECD2ECC2EC3327
:10ACF90092EEE52625E0F526D2ECD2ECD2ECC2ECB8
:02AD0900C2EE98
:01AD0B002225
:10A8BB0075840FE4901A88F0E0FF25E0FFA2EFE427
:10A8CB00334FF0D2ECD2ECD2ECC2ECE0FF25E0FF40
:10A8DB00A2EFE4334FF0D2ECD2ECD2ECC2ECE0FFBF
:10A8EB0025E0FFA2EFE4334FF0D2ECD2ECD2ECC276
:10A8FB00ECE0FF25E0FFA2EFE4334FF0D2ECD2EC1B
:10A90B00D2ECC2ECE0FF25E0FFA2EFE4334FF0D234
:10A91B00ECD2ECD2ECC2ECE0FF25E0FFA2EFE4338B
:10A92B004FF0D2ECD2ECD2ECC2ECE0FF25E0FFA270
:10A93B00EFE4334FF0D2ECD2ECD2ECC2ECE0FF25DB
:10A94B00E0FFA2EFE4334FF0D2ECD2ECD2ECC2EC4E
:02A95B00E0FF1B
:01A95D0022D7
:0BBD5B00481C8EFFFFFFFFFFFFFFFFF3
:10B88400E4901A60F0901A60E0C394047480948089
:10B894005028E0FF7B087D0A12C14B901A60E0FF3C
:10B8A400E4FBFD12C14B901A60E0FFE4FB7D011242
:10B8B400C14B901A60E004F080CB7FFF12C1BD7BC6
:10B8C400017D017F031299CD7B017D027F031299D3
:10B8D400CD7B017D037F031299CDE4FF12C537E4CC
:04B8E400FF12C2EE9F
:01B8E800223D
:10C14B00901A8EEFF0A3EDF0A3EBF0E4FD7F01125C
:10C15B00C25A901A8EE05407FF25E04440FF12AB01
:10C16B00DC901A8FE0FF12ABDC901A90E0FF12AB61
:09C17B00DC7D01E4FF12C25A222E
:08C0D700901CB2EFF0A3EDF0A4
:10C0DF00E4FD7F0112C25A901CB2E05407FF25E025
:10C0EF004441FF12ABDC901CB3E0FF12ABDC12A893
:10C0FF0018901CB4EFF07D01E4FF12C25A901CB4EB
:02C10F00E0FF4F
:01C11100220B
:0B99CD00901A8AEFF0A3EDF0A3EBF07E
:1099D800901A8BE0C39408748094805007E4901A1E
:1099E8008DF0800D901A8D7401F0901A8BE024F898
:1099F800F0901A8CE06039A3E0FF901A8AE025E025
:109A0800248EF582E4341CF583E5822FF582E43553
:109A180083F583C083C082E0FF901A8BE0FEF87460
:109A280001088002C333D8FC4FD082D083F0803A3B
:109A3800901A8DE0FF901A8AE025E0248EF582E4E2
:109A4800341CF583E5822FF582E43583F583C083E2
:109A5800C082E0FF901A8BE0FEF87401088002C310
:109A680033D8FCF45FD082D083F0901A8DE0FF9059
:109A78001A8AE025E0248EF582E4341CF583E58219
:109A88002FF582E43583F583E0FB901A8AE0FF9096
:0E9A98001A8DE070047D1480027D1512C14B02
:019AA600229D
:10C6F000901CC3EFF0A3EDF0901CC3E0FFA3E0702B
:0BC70000047D1280027D1312C0D722BE
:06BF9A00901A60121C4920
:10BFA000E4901A63F0901A63E0C394107480948054
:10BFB000502AE0FD901A60121C29901A63E0F58265
:10BFC00075830012171720E0047B0180027B007F3D
:0CBFD000021299CD901A63E004F080C9C1
:01BFDC002242
:05C1BD00901A88EFF06C
:10C1C200E4A3F0901A89E0C3941074809480501F05
:10C1D200E0FD901A88E0FFA3E06F60047B0180021B
:0FC1E2007B00E4FF1299CD901A89E004F080D41D
:01C1F100222B
:0FC89300901A5EEFF0E0FBE4FD7F031299CD22D7
:10C83700E4FB7D017F031299CD7B017D017F03120C
:03C8470099CD2266
:10C84A00E4FB7D027F031299CD7B017D027F0312F7
:03C85A0099CD2253
:10C85D00E4FB7D037F031299CD7B017D037F0312E2
:03C86D0099CD2240
:10C53700901A61EFF0E05401FB7D047F031299CD5F
:10C54700901A61E0FFC3135401FB7D057F03129925
:02C55700CD22F3
:10C2EE00901A61EFF0E020E0047B0180027B007D7C
:10C2FE000A7F031299CD901A61E0FFC31320E00468
:0EC30E007B0180027B007D0B7F031299CD2204
:0CBAC400901A64EFF0A3EDF0A3121C49EF
:10BAD000E4FDFF12C25A901A64E0FFC454F0FFA3C1
:10BAE000E0540F4FFF12ABDCE4901A6AF0901A6931
:10BAF000E0FFA3E0C39F501912A818901A66E475DE
:10BB0000F001121C32EF121777901A6AE004F080ED
:08BB1000DC7D01E4FF12C25AC2
:01BB1800220A
:10C5BD00901A60EFF0A3EDF0E4FDFF12C25A901A4D
:10C5CD0060E0FFC454F0FFA3E0540F4FFF12ABDC4B
:01C5DD00223B
:080003007D01E4FF12C25A2244
:0BC8E900901A60EFF0E0FF12ABDC22C1
:10C3FF00E4FD7F0712C5BDE4FD7F0D12C5BD7FFFB4
:10C40F0012C8E97FFF12C8E9E4FF12C8E9E4FF127E
:0BC41F00C8E97F1512C8E912000322D3
:05816E00901A5DEFF026
:10817300E0FD7B017A1A795E901A697402F0FF12AE
:10818300BAC4901A5EE0FEA3E0FFEEC4F854F0C850
:1081930068FCEFC4540F48FDE41214D5E4FBFA79EC
:1081A30020784012132AE4FBFA79807845121433BD
:1081B300901A60121BBC901A5DE0121D4A81D30015
:1081C300821801822F0382480482610500008278AD
:1081D300901A60121B747BCD7ACC794C78431213BE
:1081E3002A901A60121BBCE4FFFE7D207C41901A8A
:1081F30060121B8012132AE4FBFAF9783F1212393A
:10820300129297E4FBFA79207841121433901A60A2
:10821300121BBC8060901A60121B74E4FBFAF9789D
:108223004012132A901A60121BBC8049901A6012E4
:108233001B747BCD7ACC79CC783D121433901A60C1
:10824300121BBC8030901A60121B747B8B7A2E79C0
:108253003A783F121433901A60121BBC8017901A9D
:1082630060121B747B907AC279F5783E12143390B6
:108273001A60121BBCE4FFFE7DC87C42901A601298
:108283001B8012132AE4FBFAF9783F121239129277
:1082930097E4FBFA79C87842121433901A60121BE0
:0782A300BC901A60121B746D
:0182AA0022B1
:10F00000C2AF7584015398FC75FFDE75FFADE478DF
:10F0100013F618F6E4F584209848E47817F608F615
:0FF0200020983BC37818E6948818E69413502F75
:10F02F0075260AD3E52694007480948040177527BF
:10F03F0001D3E52794007480948040050015278044
:05F04F00F0152680DE33
:10F05400781806E61870C50680C2B28280B57812A8
:10F06400A699C298E6FF7E00641A600302F1BB7899
:10F0740017F608F620983BC37818E6948818E694A7
:03F0840013502FF7
:10F0870075280AD3E5289400748094804017752961
:10F0970001D3E529940074809480400500152980E8
:05F0A700F0152880DED9
:10F0AC00781806E61870C50680C220980302F01482
:10F0BC007813A699C298E47817F608F620983BC303
:0BF0CC007818E6948818E69413502F83
:10F0D700752A0AD3E52A9400748094804017752B0B
:10F0E70001D3E52B940074809480400500152B8094
:05F0F700F0152A80DE87
:10F0FC00781806E61870C50680C220980302F01432
:10F10C007813A699C298E47817F608F620983BC3B2
:0BF11C007818E6948818E69413502F32
:10F12700752C0AD3E52C9400748094804017752DB4
:10F1370001D3E52D940074809480400500152D803F
:05F14700F0152C80DE34
:10F14C00781806E61870C50680C220980302F014E1
:0AF15C007813A699C298D284C299D4
:10F16600752E14D3E52E9400748094804017752F65
:10F1760001D3E52F940074809480400500152F80FC
:05F18600F0152E80DEF3
:06F18B007599783099FD32
:10F1910075300AD3E530940074809480401775313E
:10F1A10001D3E531940074809480400500153180CD
:05F1B100F0153080DEC6
:10F1B600C28402F976EF64504E600302F2C67817F5
:10F1C600F608F620983BC37818E6948818E6941358
:02F1D600502FB8
:10F1D80075320AD3E53294007480948040177533F1
:10F1E80001D3E53394007480948040050015338082
:05F1F800F0153280DE7D
:10F1FD00781806E61870C50680C220980302F01430
:0AF20D007813A699C298D284C29922
:10F21700753414D3E53494007480948040177535A1
:10F2270001D3E5359400748094804005001535803E
:05F23700F0153480DE3B
:08F23C007599793099FDC29922
:10F24400753614D3E536940074809480401775376E
:10F2540001D3E5379400748094804005001537800D
:05F26400F0153680DE0C
:08F269007599013099FDC2996D
:10F27100753814D3E538940074809480401775393B
:10F2810001D3E539940074809480400500153980DC
:05F29100F0153880DEDD
:06F29600E4F5993099FD3A
:10F29C00753A0AD3E53A9400748094804017753B14
:10F2AC0001D3E53B940074809480400500153B80AD
:05F2BC00F0153A80DEB0
:10F2C100C28402F9767812E6FF7E006401600302CF
:06F2D100F359D284C2993A
:10F2D700753C14D3E53C9400748094804017753DC9
:10F2E70001D3E53D940074809480400500153D806E
:05F2F700F0153C80DE73
:08F2FC007599783099FDC29963
:10F30400753E14D3E53E9400748094804017753F95
:10F3140001D3E53F940074809480400500153F803C
:05F32400F0153E80DE43
:06F32900E4F5993099FDA6
:10F32F0075400AD3E540940074809480401775416E
:10F33F0001D3E5419400748094804005001541800D
:05F34F00F0154080DE16
:10F35400C28402F976EF64024E600302F4837817E4
:10F36400F608F620983BC37818E6948818E69413B8
:02F37400502F18
:10F3760075420AD3E5429400748094804017754321
:10F3860001D3E543940074809480400500154380C2
:05F39600F0154280DECD
:10F39B00781806E61870C50680C220980302F01490
:10F3AB007813A699C298E408F618E6FF13B3928275
:10F3BB00EF25E0FEC3E49400EE94F0502CE6FD7FC5
:10F3CB000025E0FEC394E05020ED20E023E4F5841B
:10F3DB0043B701758F037819EEF608EFF6F5828EB9
:10F3EB0083F053B7F0F58F8004781476FFE4F5843F
:04F3FB00D284C2995D
:10F3FF00754414D3E5449400748094804017754588
:10F40F0001D3E54594007480948040050015458034
:05F41F00F0154480DE41
:08F424007599783099FDC29939
:10F42C00754614D3E5469400748094804017754754
:10F43C0001D3E54794007480948040050015478003
:05F44C00F0154680DE12
:08F451007814E6F5993099FDED
:10F4590075480AD3E548940074809480401775492B
:10F4690001D3E549940074809480400500154980D2
:05F47900F0154880DEE3
:10F47E00C28402F9767812E66403600302F67078AD
:10F48E0017F608F620983BC37818E6948818E69489
:03F49E0013502FD9
:10F4A100754A0AD3E54A9400748094804017754BDD
:10F4B10001D3E54B940074809480400500154B8086
:05F4C100F0154A80DE99
:10F4C600781806E61870C50680C220980302F01464
:10F4D6007813A699C298E47817F608F620983BC3E5
:0BF4E6007818E6948818E69413502F65
:10F4F100754C0AD3E54C9400748094804017754D87
:10F5010001D3E54D940074809480400500154D8031
:05F51100F0154C80DE46
:10F51600781806E61870C50680C220980302F01413
:10F526007815A699C2987813E6FF139282EF25E024
:10F53600FEC3E49400EE94F0400302F014E625E0E6
:10F54600FCC394E0400302F014E4F58443B701756C
:10F556008F017815E675F020A42400FFE5F03C78CD
:10F5660019F608A607E4F5847816F67816E6C39425
:10F5760020748094805063E408F608F620983BC314
:0BF586007818E6948818E69413502FC4
:10F59100754E0AD3E54E9400748094804017754FE0
:10F5A10001D3E54F940074809480400500154F808D
:05F5B100F0154E80DEA4
:10F5B600781806E61870C50680C220980302F01473
:10F5C60078190806E618860670010614F5828E83F9
:10F5D600E599F0C2987816068091E4F58453B7F061
:08F5E600F58FF584D284C2996F
:10F5EE00755014D3E5509400748094804017755173
:10F5FE0001D3E5519400748094804005001551802C
:05F60E00F0155080DE44
:08F613007599783099FDC29948
:10F61B00755214D3E552940074809480401775533F
:10F62B0001D3E553940074809480400500155380FA
:05F63B00F0155280DE15
:06F64000E4F5993099FD8C
:10F6460075540AD3E5549400748094804017755518
:10F6560001D3E555940074809480400500155580CB
:05F66600F0155480DEE8
:10F66B00C28402F9767812E6FD7C00640460030222
:10F67B00F78F7817F608F620983BC37818E694882E
:06F68B0018E69413502F55
:10F6910075560AD3E55694007480948040177557C7
:10F6A10001D3E5579400748094804005001557807C
:05F6B100F0155680DE9B
:10F6B600781806E61870C50680C220980302F01472
:10F6C6007813A699C298E625E0781BF6087600E43A
:10F6D6007814F67817F608F6781B0806E6188606F4
:10F6E60070010614F5828E83E493781426F6781852
:10F6F60006E6187001067818E6B400DC18E6B402CF
:05F70600D7D284C29976
:10F70B00755814D3E558940074809480401775593C
:10F71B0001D3E559940074809480400500155980FD
:05F72B00F0155880DE1E
:08F730007599783099FDC2992A
:10F73800755A14D3E55A9400748094804017755B09
:10F7480001D3E55B940074809480400500155B80CC
:05F75800F0155A80DEEF
:08F75D007814E6F5993099FDDE
:10F76500755C0AD3E55C9400748094804017755DE0
:10F7750001D3E55D940074809480400500155D809B
:05F78500F0155C80DEC0
:10F78A00C28402F976ED64054C600302F96A7817BF
:10F79A00F608F620983BC37818E6948818E694137E
:02F7AA00502FDE
:10F7AC00755E0AD3E55E9400748094804017755F93
:10F7BC0001D3E55F940074809480400500155F8050
:05F7CC00F0155E80DE77
:10F7D100781806E61870C50680C220980302F01456
:10F7E1007813A699C298E47817F608F620983BC3D7
:0BF7F1007818E6948818E69413502F57
:10F7FC0075600AD3E560940074809480401775613D
:10F80C0001D3E561940074809480400500156180FB
:05F81C00F0156080DE24
:10F82100781806E61870C50680C220980302F01405
:0AF831007815A699C298D284C299F6
:10F83B00756214D3E56294007480948040177563ED
:10F84B0001D3E563940074809480400500156380B8
:05F85B00F0156280DEE3
:08F8600075997F3099FDC299F2
:10F86800756414D3E56494007480948040177565BA
:10F8780001D3E56594007480948040050015658087
:05F88800F0156480DEB4
:10F88D007599203099FD7813E625E0FC7815E6751D
:10F89D00F020A42400FFE5F03C781BF608A607E451
:10F8AD007814F67816F67816E6C394207480948052
:04F8BD005053C29949
:10F8C100756614D3E566940074809480401775675B
:10F8D10001D3E5679400748094804005001567802A
:05F8E100F0156680DE59
:10F8E600781BE6FE08E6F5828E83E493F599309957
:10F8F600FD781B0806E618860670010614F5828E4A
:0EF9060083E493781426F678160680A1C29941
:10F91400756814D3E5689400748094804017756901
:10F9240001D3E569940074809480400500156980D2
:05F93400F0156880DE03
:08F939007814E6F5993099FD00
:10F94100756A0AD3E56A9400748094804017756BD8
:10F9510001D3E56B940074809480400500156B80A1
:05F96100F0156A80DED4
:10F96600C284800C7812E664067005F58475EF1083
:0CF976007812E66407600302F014D2AFC0
:01F982002262
:1043AF0046455F4343000134000000537461747548
:1043BF007300000119500418000001553234000039
:1043CF00000000011951041800000155332E33006D
:1043DF00000000011955041800000155352E30005A
:1043EF00000000011959040800000154656D7000A8
:1043FF0000000001195D01320000004645423030D7
:10440F0000000001196101320000004645423031C1
:10441F0000000001196201320000004645423032AF
:10442F00000000011963013200000046454230339D
:10443F00000000011964013200000046454230348B
:10444F000000000119650132000000464542303579
:10445F000000000119660132000000464542303667
:10446F000000000119670132000000464542303755
:10447F000000000119680132000000464542303843
:10448F000000000119690132000000464542303931
:10449F0000000001196A0132000000464542313028
:1044AF0000000001196B0132000000464542313116
:1044BF0000000001196C0132000000464542313204
:1044CF0000000001196D01320000004645423133F2
:1044DF0000000001196E01320000004645423134E0
:1044EF0000000001196F01320000004645423135CE
:1044FF0000000001197001320000004D6178636601
:10450F0067000001197101320000045273744650A4
:10451F004741000000000132000004527374435001
:10452F0055000000000001320000045273744D4129
:10453F00580000000000013400000042504D6F642D
:10454F0065000001197201340000004174746E009F
:10455F000000000119730137000004535049000097
:10456F0000000000000001340000005350495F5369
:10457F004C54000119740408000001315754656D43
:10458F007030300119750408000001315754656D02
:10459F007030310119790408000001315754656DED
:1045AF0070303201197D0408000001315754656DD8
:1045BF007030330119810408000001315754656DC3
:1045CF007030340119850408000001315754656DAE
:1045DF007030350119890408000001315754656D99
:1045EF0070303601198D0408000001315754656D84
:1045FF007030370119910408000001315754656D6F
:10460F007030380119950408000001315754656D59
:10461F007030390119990408000001315754656D44
:10462F0070313001199D0408000001315754656D38
:10463F007031310119A10408000001315754656D23
:10464F007031320119A50408000001315754656D0E
:10465F007031330119A90408000001315754656DF9
:10466F007031340119AD0408000001315754656DE4
:10467F007031350119B108340000083157416472A7
:10468F003030000119B50834000008315741647209
:10469F003031000119BD08340000083157416472F0
:1046AF003031000119C508340000083157416472D8
:1046BF003031000119CD08340000083157416472C0
:1046CF003031000119D508340000083157416472A8
:1046DF003031000119DD0834000008315741647290
:1046EF003031000119E50834000008315741647278
:1046FF003031000119ED0834000008315741647260
:10470F003031000119F50834000008315741647247
:10471F003031000119FD083400000831574164722F
:10472F00303100011A050834000008315741647216
:10473F00303100011A0D08340000083157416472FE
:10474F00303100011A1508340000083157416472E6
:10475F00303100011A1D08340000083157416472CE
:10476F00303100011A2508340000083157416472B6
:10477F00303100011A2D0000000000000000000081
:06478F0000000000000024
:0DBD6600431A35FF43B54418880000000063
:109C5A0012C82475840F75E104E4F5E275E34075D2
:109C6A00A4FF75A5FF75A6FF75A7FF759DDE759EF6
:109C7A007F7580E0F590F5A075B0FF75D8FF75E89F
:109C8A00FF758A83F597F589F58475B71075840F82
:109C9A00438901758D01758F01758E02901A5DF0E9
:109CAA00A3F0901A5DE0FEA3E0C3EE9401500C907D
:109CBA001A5DE475F00112184880E7438902E490BE
:109CCA001A5DF0A3F0901A5DE0FEA3E0FFE4FCFD4C
:109CDA007B507AC3F9F8D3121AB94011E5895410A6
:109CEA00700B901A5D75F00112184880D8759702AA
:109CFA00E4F58475A3D775A1B7C2847F0AFE12C1A1
:109D0A0012C2857D08E4FF12BCB8D2BC12B66D7AC5
:109D1A00007B967D037F0012A12E7A007B967D033D
:059D2A007F0112A12ED3
:019D2F002211
:058CB600901A5DEFF0D3
:108CBB00E0602DE4A3F0901A5EE0C3941B748094E3
:108CCB00805014E02461F582E43419F583E4F090CC
:108CDB001A5EE004F080DFE4901971F0A3F0A3F0CA
:108CEB009019507401F0E4901974F012C7BB12B8CC
:108CFB008412C3FF7B017A19796112BF9AE4FF12C8
:108D0B00C8C0E4901A5EF0901A5EE0C394107480B1
:108D1B0094805056E025E025E02475F582E4341963
:108D2B00F583121BC8C479C000E4901A5FF0901A47
:108D3B005FE0C39408748094805027E0FF901A5E24
:108D4B00E075F008A424B5F582E43419F583E582C7
:108D5B002FF582E43583F583E4F0901A5FE004F09D
:108D6B0080CC901A5EE004F0809DE4901A5EF09047
:108D7B001A5EE0C3941074809480501AE0FF12C105
:108D8B00BD901A5EE0FF1286457FFF12C1BD901A9F
:108D9B005EE004F080D990188C121BC80000000014
:108DAB007B007A0079007F00129EDBE4901A52F070
:028DBB00A3F023
:018DBD002293
:109EDB0090FFFD121D70121C4990FFFF121D70EFB9
:079EEB00F090FFFE121D7054
:109EF200851083851182A3A3E07008901950E02495
:109F0200FF92DC851083851182A3A3E0641B707726
:109F1200900003121D94121C291216FE540785107C
:109F220083851182F0A37402F0851083851182E08B
:109F32006407701A900003121D94121C29900001EC
:109F4200121717851083851182F0A37403F0851010
:109F520083851182E014F0E0FF7E00900003121D61
:109F620094121C29851083851182A3E07C0029F9B3
:109F7200EC3AFA78107C197D011216D88510838587
:109F82001182E0901A54F0851083851182A3A3E018
:0C9F92002490F582E43418F5837401F08B
:079F9E00900006121D702265
:109D300090FFFD121D70121C4990FFFF121D70EF65
:079D4000F090FFFE121D7000
:109D4700851083851182A3A3E06416601A851083AA
:109D5700851182A3A3E06417600D851083851182A6
:109D6700A3A3E064187012900003121D94121C291B
:109D7700E41217777F01029DFF851083851182A367
:109D8700A3E0641B7070851083851182F0A3F085B2
:109D97001083851182E0FEA3E0C3EE9401504B903F
:109DA7001A52E0FFA3E06F6041901A52E024D0F509
:109DB70082E43418F583E0FF900003121D94121C0F
:109DC70029851083851182E0FCA3E0F5828C83EF5F
:109DD700121789901A52E004543FF08510838511B9
:109DE70082E475F00112184880A5851083851182D9
:089DF700E0A3E0FF80027F0001
:079DFF00900006121D702206
:107AAA00E4901A5DF0901A5DE0C39410748094809B
:107ABA00502DE02495F582E43418F583E060187BB4
:107ACA00017A19796112BF9A901A5DE02495F582BC
:107ADA00E43418F583E4F0901A5DE004F080C6906F
:107AEA0018A5E0600D901971E0FF12C893E4901890
:107AFA00A5F09018A6E0600812C837E49018A6F01E
:107B0A009018A7E0600812C84AE49018A7F09018E5
:107B1A00A8E0600812C85DE49018A8F09018A9E0DF
:107B2A00600D901972E0FF12C537E49018A9F09021
:107B3A0018AAE0600D901973E0FF12C2EEE49018E3
:107B4A00AAF09018ABE0603B901974E0FF12C1BD37
:107B5A00E4901A5DF0901A54E0FF901A5DE0C39F1A
:107B6A005017E02410F582E43419F583E0FF12ACD3
:107B7A0074901A5DE004F080DC7FFF12C1BDE490CE
:107B8A0018ABF0E4901A5DF0901A5DE0C39410749B
:107B9A00809480505AE024BDF582E43418F583E0DD
:107BAA006045901A5DE075F008A424B5F582E434C6
:107BBA0019F583E064017020901A5DE0FF12C1BDDF
:107BCA00901A5DE0FF1286457FFF12C1BD7A007BE5
:107BDA00647D057F0012A12E901A5DE024BDF58216
:107BEA00E43418F583E4F0901A5DE004F08099908B
:107BFA0018BEE0601B9019BDE070107F0112864527
:107C0A007A007B647D057F0012A12EE49018BEF0F5
:017C1A002247
:10C51400901A53E0FF901A52E0B50716A3E024D016
:10C52400F582E43418F5837458F0901A53E00454F7
:03C534003FF022B3
:10A6CD007E007F167D007B017A1A793C1221CF7EA8
:10A6DD00007FE57D007B017A1979501221CFE4F5D9
:10A6ED0084901A5DF0A37480F0758F04901A5DE06C
:10A6FD00FEA3E0AA06F97BFF783C7C1A7D017E0063
:10A70D007F161216D8901A5DE4F0A37496F0901A85
:10A71D005DE0FEA3E0AA06F97BFF78507C197D0170
:10A72D007E007FE51216D8E4F58F901A50E0FEA357
:10A73D00E064347003EE6412602774FF901A3CF0ED
:10A74D00A3F0A3F0A3F0FB7A4379AF78407C1A7D98
:10A75D0001122008901A507412F0A37434F07F0186
:05A76D0022D2017F0073
:01A7720022C4
:10B2D80012C824C2AFE4F5847812F608768043B722
:10B2E80001758F0718E6FE08E6F5828E83E4F0758F
:10B2F8008F0518F60876807B017A1A793CC0021807
:10B30800E6FE08E6AA06F8AC027D01D0027E007FC0
:10B31800161216D8781276000876967B017A197973
:10B3280050C00218E6FE08E6AA06F8AC027D01D075
:10B33800027E007FE91216D853B7FEE4F58FD2AF2C
:05B348007F0A12C75945
:01B34D0022DD
:10BD060012C7A4901888121B801219B5E47B0AFA90
:10BD1600F9F8D3121ACF503512C7A4901888121BFF
:10BD2600BC7F0312816E901951121BBC7F041281D5
:10BD36006E901955121BBC7F0512816E901959120F
:0DBD46001BBCE4FF12816E90195D121BBC46
:01BD530022CD
:1091A400E4F58475EF02901A5B7464F0901A5BE046
:1091B400D39400748094804005E014F080EE129CF7
:1091C4005AC204C203C20012A6CD901A5BEFF0E0AB
:1091D400FF128CB612C6D47F0A12C759901A5C7457
:1091E40001F030010320020B7A007B327D017F0005
:1091F40012A12E30040AC20412B2D8D20112A6CD92
:1092040030030CC2037F0A7E0012C11212F0003038
:10921400000512BC17C200901A5CE0601C12C480E6
:10922400E47B05FAF9F8D3121ACF500DE4901A5CD6
:10923400F090189004F0127AAA7F0012B5FE123151
:109244002412BD06127AAA12C51412C7A4A804A92E
:1092540005AA06AB0790188C121B74EF24E8FFEEE6
:109264003403FEE43DFDE43CFCD3121ACF50030268
:1092740091E612C7A490188C121BBC7B017A197951
:1092840075127C1B7A007B647D017F0012A12E0283
:0292940091E661
:0192960022B5
:10BD7300511C703031323334353637383941424310
:04BD830044454600ED
:10C28C0075840FD2DE7F587E0212AEBDC2DE7F4BAC
:10C29C007E0012AEBD20DD047F0180027F00901A6B
:10C2AC006AEFF07FF47E0112AEBDC2DE901A6AE036
:01C2BC00FF82
:01C2BD00225E
:0CA4D400901A6CEFF0C2DED2DEE06025D2
:10A4E00075260FD3E526940074809480403C752730
:10A4F00001D3E527940074809480400500152780DF
:05A50000F0152680DECD
:10A50500752869D3E52894007480948040177529CF
:10A5150001D3E529940074809480400500152980B5
:05A52500F0152880DEA6
:08A52A00C2DE901A6CE060250E
:10A53200752A69D3E52A940074809480403C752B77
:10A5420001D3E52B940074809480400500152B8084
:05A55200F0152A80DE77
:10A55700752C0FD3E52C9400748094804017752DCB
:10A5670001D3E52D940074809480400500152D805B
:05A57700F0152C80DE50
:01A57C0022BC
:05BE3800901A6AEFF012
:10BE3D00E4A3F0901A6BE0C394087480948050359D
:10BE4D00E0FF7E007401A807088005C333CE33CE12
:10BE5D00D8F9FF901A6AE0FDE4EF5DD39400748089
:10BE6D00948040047F0180027F0012A4D4901A6B4D
:05BE7D00E004F080BEAE
:01BE8200229D
:04B0D900C2DED2DE23
:10B0DD0075260AD3E5269400748094804017752751
:10B0ED0001D3E527940074809480400500152780D6
:05B0FD00F0152680DEC5
:02B10200C2DEAB
:10B1040075280AD3E5289400748094804017752923
:10B1140001D3E529940074809480400500152980AA
:05B12400F0152880DE9B
:08B12900A2DDE433901A6CF082
:10B13100752A50D3E52A9400748094804017752BAA
:10B1410001D3E52B940074809480400500152B8079
:05B15100F0152A80DE6C
:05B15600901A6CE0FFFF
:01B15B0022D1
:10BDA000E4901A6BF0901A6AF0901A6AE0C3940853
:10BDB00074809480503012B0D9EF6018901A6AE005
:10BDC000FF7E007401A807088005C333CE33CED8A8
:10BDD000F9FF80047E007F00901A6BE04FF0901A0C
:0BBDE0006AE004F080C3901A6BE0FFE3
:01BDEB002235
:05864500901A60EFF047
:10864A007F0012B5FEE4901A61F0901A61E0C394BB
:10865A0008748094805027E0FF901A60E075F00853
:10866A00A424B5F582E43419F583E5822FF582E472
:10867A003583F583E4F0901A61E004F080CCC2AF50
:10868A0012C28C901A61EFF0E07017901A60E075D0
:10869A00F008A424B5F582E43419F583E4F0D2AFE6
:1086AA00FF227FCC12BE387F9912BE387F5A12BE83
:1086BA00387FA512BE3812BDA07FF47E0112AEBD6E
:1086CA007F0012B5FE12C28C7F0F12BE38E4901AD8
:1086DA0061F0901A61E0C3940874809480502D125E
:1086EA00BDA0901A61E0FE901A60E075F008A4241B
:1086FA00B5F582E43419F583E5822EF582E43583F3
:10870A00F583EFF0901A61E004F080C612BDA07FF5
:10871A000A7E0012C1127F0012B5FE12C28C7FCCF3
:10872A0012BE387F9912BE387F3C12BE387FC31200
:10873A00BE3812BDA0D2AF7F0012B5FE901A60E01B
:10874A0075F008A424B5F582E43419F583E0D394CE
:0D875A00007480948040047F0180027F0045
:0187670022EF
:067C1B00901A5D121C49E5
:107C2100E4901A62F0901A62E0C394107480948018
:107C31004003027D69E075F008A424B5F582E434BF
:107C410019F583E0701D901A5D121C29901A62E0EB
:107C510075F004A4F58285F083121BF9C479C00084
:107C6100027D607F0012B5FE12C28C901A61EFF0A6
:107C7100E0701D901A5D121C29901A62E075F004E3
:107C8100A4F58285F083121BF9C479C000027D60DE
:107C910012C908901A65EFF07F5512BE38E4901AA8
:107CA10060F0901A60E0C3940874809480502AE0D8
:107CB100FF901A62E075F008A424B5F582E4341946
:107CC100F583E5822FF582E43583F583E0FF12BE6B
:107CD10038901A60E004F080C97FBE12BE3812BD30
:107CE100A0901A63EFF012BDA0901A64EFF012C9D0
:107CF10008901A65E06F7067901A64E0FE901A634D
:107D0100E0FDEEFCEDEC1214D5E4FBFA79AA784221
:107D110012132AE4FBFA79AA7844121433901A66F2
:107D2100121BBCE4FFFE7D207C41901A66121B8071
:107D310012132AE4FBFAF9783F121239129297E4EE
:107D4100FBFA79207841121433901A5D121C2990A4
:107D51001A62E075F004A4F58285F083121B50903D
:107D61001A62E004F0027C267F0012B5FE12C28C7A
:107D7100C2AF7FCC12BE387F4412BE38D2AF7F0073
:037D810012B5FE3A
:017D840022DC
:0300000002AD0C42
:10AD0C00787FE4F6D8FD75102075110075816E0200
:02AD1C00AD592F
:05BD870042164B000014
:10C4A90090166374FFF07E027F247D007B017A166B
:10C4B90079641221CF7E007F167D007B017A16797F
:04C4C9004D0221CF30
:0FC1F200901A71EBF0A3EAF0A3E9F0A3121BBCC3
:10C201007E007F047D007B017A1C79471221CF904B
:10C21100165D7401F0901A71E0FBA3E0FAA3E0F956
:04C22100A312479588
:01C2250022F6
:10C63F00E4FFFE90165DE060157407F07B007A0052
:0EC64F0079007D007C001247A0E490165DF09B
:01C65D0022BA
:06938700901A81121BBCCC
:10938D0090165EE0600302946390165DE0C394094D
:10939D0050030294637B007A007900901A81124782
:1093AD0095901A85EEF0A3EFF064014E70030294D0
:1093BD005B90165DE0B40A47E47B02FAF9F890166B
:1093CD004DE0FCA3E0FDA3E0FEA3E0FF1219FF902A
:1093DD001655E0F8A3E0F9A3E0FAA3E0FBC3121AD7
:1093ED00CF701C901655E0FCA3E0FDA3E0FEA3E0BA
:1093FD00FFE47B02FAF9F81219FF901655804C9094
:10940D00165DE0B40B48E47B08FAF9F890164DE0D0
:10941D00FCA3E0FDA3E0FEA3E0FF1219FF90165997
:10942D00E0F8A3E0F9A3E0FAA3E0FBC3121ACF70B2
:10943D001D901659E0FCA3E0FDA3E0FEA3E0FFE4C0
:10944D007B02FAF9F81219FF901659121BBC9016EF
:10945D005D7409F08008901A85E4F0A304F0901A69
:06946D0085E0FEA3E0FF14
:0194730022D6
:10972F0090165EE0600302981290165DE0C39409F4
:10973F00500302981290164CE004F0700690164BEE
:10974F00E004F090164BE07004A3E064647028907E
:10975F00164BF0A3F0901651E0FCA3E0FDA3E0FE42
:10976F00A3E024FFFFEE34FFFEED34FFFDEC34FFEA
:10977F00FC901651121BBC901655E0FCA3E0FDA304
:10978F00E0FEA3E0FF901651E0F8A3E0F9A3E0FAA2
:10979F00A3E0FBD3121ACF506AE4FFFEFDFC901634
:1097AF0051E0F8A3A3A3E0C3121ACF700590165D82
:1097BF00F022901659E0FCA3E0FDA3E0FEA3E0FF2A
:1097CF00901651E0F8A3E0F9A3E0FAA3E0FBD3125F
:1097DF001ACF500790165D740BF022901655E0FCCF
:1097EF00A3E0FDA3E0FEA3E0FF901651E0F8A3E095
:1097FF00F9A3E0FAA3E0FBD3121ACF500690165D3F
:03980F00740AF0E8
:019812002233
:0B479500E0FCA3E0FDA3E0FEA3E0FFBA
:0F47A000901A87EBF0A3EAF0A3E9F0A3121BBC79
:1047AF00E4901A8EF0A3F0A3F0A3F0901A9DF0A35B
:1047BF00F090165DE07003024B63E064076004E065
:1047CF00B40A10901A9F7401F0A37416F0A3745FCB
:1047DF00F0800E901A9F7401F0A3741BF0A374CA9B
:1047EF00F0901B3BE4F0A37443F0A37411F0E4A327
:1047FF00F0A304F0A37416F0A37464F0A37402F092
:10480F00A37424F0901A9FE0FBA3E0FAA3E0F97DD4
:10481F00447C00125292901A92EFF0C364809480FD
:10482F005003024B54E0FF3395E0FE7C007D3D12B8
:10483F0017AB747B2FF974123EFA901A947401F02F
:10484F00A3EAF0A3E9F0901A8EE07002A3E06003F0
:10485F00024B44901A93F0901A87E0FBA3E0FAA35F
:10486F00E0F9A3E0FCA3E0FDA3E0FEA3E0FF123F0D
:10487F00C1901A97121BBC901A9DE0FCA3E0FDECAF
:10488F0090166CF0EDA3F0901A9FE0FBA3E0FAA353
:10489F00E0F97401901BCA6B7008E965827003EA36
:1048AF006583700790166304F08005E4901663F03B
:1048BF007B017A167964C003C002C001901A94E09C
:1048CF00FBA3E0FAA3E0F990000E121CF1901A94EA
:1048DF00E0FBA3E0FAA3E0F9900011740275F02455
:1048EF0012197B12740D901A90EEF0A3EFF0901640
:1048FF005DE0B4070B901A8EE4F0A304F0024B278F
:10490F00901A93E02401FEE433901A9BF0A3CEF0AB
:10491F00C3901A90E0648094805015901A9BE0FE2B
:10492F00A3E0FF7C007D641217AB12C73F024B1848
:10493F009016637401F07B017A167964901AA6744D
:10494F0002F0A37424F0901A9BE0FEA3E0FF7C001A
:10495F007D641217AB901AA8EEF0A3EFF0901A92A5
:10496F00E0FF127231901A90EEF0A3EFF0D39400A3
:10497F00EE648094805003024AFA90166BE0FFE4D5
:10498F00FCFDFE7808121AF3A804A905AA06AB07C6
:10499F0090166AE0FFEB4FFFEAFEE9FDE8FC7808AE
:1049AF00121AF3A804A905AA06AB07901669E0FF2F
:1049BF00EB4FFFEAFEE9FDE8FC7808121AF3A804B2
:1049CF00A905AA06AB07901668E0FFEB4FFFEAFEBA
:1049DF00E9FDE8FC901A97E0F8A3E0F9A3E0FAA349
:1049EF00E0FBC3121ACF6003024AFA901664E06428
:1049FF00026003024AFA90165DE024FD602324F959
:104A0F00601F14601C240A6003024AEE12000EBFDE
:104A1F00020C90165D7403F012C65E024B0E024A32
:104A2F00EE12000EEF64056003024AE378477C1C28
:104A3F007D017B017A167974FE7F041216D812C697
:104A4F007C12C6B712802E901651121BBC901651B5
:104A5F00E0FCA3E0FDA3E0FEA3E0FF90164D121BC8
:104A6F00BC12C65E74FFFFFEFDFC901651E0F8A36A
:104A7F00E0F9A3E0FAA3E0FBC3121ACF7007901678
:104A8F005E04F0803FE47B02FAF9F8901651E0FCE7
:104A9F00A3E0FDA3E0FEA3E0FF1219FF901655124D
:104AAF001BBCE47B08FAF9F8901651E0FCA3E0FD7B
:104ABF00A3E0FEA3E0FF1219FF901659121BBCE4EE
:104ACF0090165EF090165D7409F0901A8EE4F0A3C4
:104ADF0004F0802B12000EBF0203024945800090A4
:104AEF001A8E74FFF0A3749CF08014901A9BE0FE52
:104AFF00A3E0FF901A9EE02FF0901A9DE03EF090F9
:104B0F001A8EE07002A3E0700F901A93E004F0E0A9
:104B1F00C394035003024866901A90E0FEA3E0FF8F
:104B2F00D39400EE648094804003024855901A8E0F
:104B3F00EEF0A3EFF090166374FFF0901A92E0FF7F
:104B4F0012A625800F901A92E0FE3395E0901A8EF0
:0C4B5F00F0A3CEF0901A8EE0FEA3E0FF61
:014B6B002227
:0F3FC100901AA2EBF0A3EAF0A3E9F0A3121BBC45
:103FD00090165DE024FD700302408924FC601424E7
:103FE000FD7003024089147003024089240A6003B3
:103FF00002412712C8DCEF2401FFE43EFEE433FD5A
:10400000E433FC7810121AF3C004C005C006C007E0
:1040100012C8DCEF2401FFE43EFED003D002D00141
:10402000D000EB4FFFEA4EFEE9FDE8FC901AA91222
:104030001BBC901AA9E0FCA3E0FDA3E0FEA3E0FFF7
:10404000901668EFF0901AA9A3A3A3E07808121ABB
:10405000E0901669EFF0901AA9E0FCA3E0FDA3E060
:10406000FEA3E0FF7810121AE090166AEFF0901AA3
:10407000A9E0FCA3E0FDA3E0FEA3E0FF7818121A7C
:10408000E090166BEFF002413190166BE0FFE4FC1C
:10409000FDFE901AA9121BBC901AA9E0FCA3E0FD3A
:1040A000A3E0FEA3E0FF7808121AF3A804A905AA6A
:1040B00006AB0790166AE0FFEB4FFFEAFEE9FDE86A
:1040C000FC901AA9121BBC901AA9E0FCA3E0FDA366
:1040D000E0FEA3E0FF7808121AF3A804A905AA06D7
:1040E000AB07901669E0FFEB4FFFEAFEE9FDE8FC45
:1040F000901AA9121BBC901AA9E0FCA3E0FDA3E052
:10410000FEA3E0FF7808121AF3A804A905AA06ABDB
:1041100007901668E0FFEB4FFFEAFEE9FDE8FC9030
:104120001AA9121BBC800A901AA9121BC800000011
:10413000009016647401F0A3F0A37406F07E007F73
:10414000047D007B017A1679781221CF7E007F04EE
:104150007D007B017A16797C1221CF78807C167DD8
:10416000017B017A0079077E007F061216D8901A2B
:10417000A2A3E0FAA3E04A601478D07C167D0190F7
:104180001AA2E0FBA3A3E0F91220088005E4901630
:10419000D0F0901AAD7401F0A37417F0A37450F02E
:1041A000901AADE0FBA3E475F00112185EA9F0FAD5
:1041B0007463121777901AADE0FBA3E475F0011257
:1041C000185EA9F0FA7482121777901AADE0FBA37B
:1041D000E475F00112185EA9F0FA74531217779083
:1041E0001AADE0FBA3E475F00112185EA9F0FA74B1
:1041F00063121777901AADE0FBA3E475F001121873
:104200005EA9F0FA7435121777901AADE0FBA3E4BB
:1042100075F00112185EA9F0FA7401121777901662
:104220005DE024FD605A24FC700302435B24FD70B2
:1042300003024328147003024328240A6003024344
:104240009090166E7480F07E007F047D007B017A72
:104250001679741221CF7E007F047D007B017A16CF
:1042600079701221CF901AADE0FBA3E475F0011232
:10427000185EA9F0FA740112AB5112887C02435601
:1042800090166E7480F07E007F047D007B017A16AC
:1042900079701221CF12AB3F12B3C4901AADEBF07C
:1042A000A3EAF0A3E9F0901AADE0FBA3E475F001F6
:1042B00012185EA9F0FA7432121777901AADE0FB6B
:1042C000A3E475F00112185EA9F0FA7404121777CE
:1042D000E4FF74742FF582E43416F583E0FE901A3F
:1042E000ADE0FBA3E475F00112185EA9F0FAEE123E
:1042F00017770FEFB404DB901AADE0FBA3E0FAA34D
:10430000E0F912888712B1DD12B34E901AADEBF0CE
:10431000A3EAF0A3E9F07E007F047D007B017A161A
:1043200079741221CF024390E490166EF0FE7F0460
:10433000FD7B017A1679741221CF78707C167D018D
:104340007B017A1C79477E007F041216D812AB3F9E
:1043500012887C12B1DD12B34E802AE490166EF002
:10436000FE7F04FD7B017A1679741221CF901AAD7D
:10437000E0FBA3E475F00112185EA9F0FA740712CD
:10438000AB5112B3C4901AADEBF0A3EAF0A3E9F07D
:10439000901AADE0FBA3E0FAA3E0F974FF121777DF
:0E43A000901AA9E0FCA3E0FDA3E0FEA3E0FF5D
:0143AE0022EC
:10A1ED007B017A177954901AA9EBF0A3EAF0A3E951
:10A1FD00F02437F9EA3401FAA3EBF0A3EAF0A3E96E
:10A20D00F0901AA9E0FBA3E0FAA3E0F91216FEFE06
:10A21D00B50702807EEEF46029901AACE0FBA3E056
:10A22D00FAA3E0F9C003C002C001901AA9A3E0FA95
:10A23D00A3E0F9D3D082D083D0E0E99582EA95836B
:10A24D00400B901AA9E4F0A3F0A3F08046EE701C29
:10A25D00901AAAE475F001121848901AA9E0FBA310
:10A26D00E0FAA3E0F91216FE60E68095901AAAE4D2
:10A27D0075F001121848901AA9E0FBA3E0FAA3E0CB
:10A28D00F91216FE04FEFD901AAAE48DF01218487C
:0EA29D0002A20E901AA9E0FBA3E0FAA3E0F9DA
:01A2AB002290
:10000E00E4FC7F3512A1EDE94A6007900002121759
:04001E0017FCAF0418
:0100220022BB
:10802E00901AA2121BC8000000007F3312A1ED901F
:10803E001AA6EBF0A3EAF0A3E9F0AE024E7003022B
:10804E00815F901AA7E475F002121848901AA6E004
:10805E00FBA3E0FAA3E0F91216FEFFE4FCFDFE78A6
:10806E0018121AF3901AA2121BBC901AA7E475F0FC
:10807E0001121848901AA2E0F8A3E0F9A3E0FAA3BF
:10808E00E0FBC000C001C002C003A3E0FBA3E0FA06
:10809E00A3E0F91216FEFFE4FCFDFE7810121AF3AF
:1080AE00D003D002D001D000EB2FFFEA3EFEE93D17
:1080BE00FDE83CFC901AA2121BBC901AA7E475F0C6
:1080CE0001121848901AA2E0F8A3E0F9A3E0FAA36F
:1080DE00E0FBC000C001C002C003A3E0FBA3E0FAB6
:1080EE00A3E0F91216FEFFE4FCFDFE7808121AF367
:1080FE00D003D002D001D000EB2FFFEA3EFEE93DC7
:10810E00FDE83CFC901AA2121BBC901AA7E475F075
:10811E0001121848901AA2E0F8A3E0F9A3E0FAA31E
:10812E00E0FBC001C002C003A3E0FBA3E0FAA3E0A2
:10813E00F91216FEFFE4FCFDFED003D002D001EBD7
:10814E002FFFEE3AFEED39FDEC38FC901AA2121B11
:0F815E00BC901AA2E0FCA3E0FDA3E0FEA3E0FFAB
:01816D0022EF
:10C65E007F3612A1EDE94A6014740229F9E43AFA20
:0DC66E00785F7C167D017E007F041216D8D7
:01C67B00229C
:10AB3F00901AADE0FBA3E475F00112185EA9F0FACC
:10AB4F007403121777901AADE0FBA3E0FAA3E0F9B4
:0BAB5F00901AB0EBF0A3EAF0A3E9F0BD
:10AB6A00901AB0E0FBA3E475F00112185EA9F0FA9E
:10AB7A00743D121777901AB0E0FBA3E475F0011246
:10AB8A00185EA9F0FA7407121777901AB0E0FBA3BF
:10AB9A00E475F00112185EA9F0FA7401121777E44D
:10ABAA00FF74072FF582E43400F583E0FE901AB0B3
:10ABBA00E0FBA3E475F00112185EA9F0FAEE121791
:10ABCA00770FEFB406DB901AB0E0FBA3E0FAA3E03C
:01ABDA00F981
:01ABDB002257
:0BB3C400901AADEBF0A3EAF0A3E9F053
:0BB3CF00901AB0EBF0A3EAF0A3E9F045
:10B3DA00901AB0E0FBA3E475F00112185EA9F0FA26
:10B3EA007436121777901AB0E0FBA3E475F00112D5
:10B3FA00185EA9F0FA7404121777E4FF745F2FF548
:10B40A0082E43416F583E0FE901AB0E0FBA3E475FB
:10B41A00F00112185EA9F0FAEE1217770FEFB404D2
:0CB42A00DB901AB0E0FBA3E0FAA3E0F90D
:01B4360022F3
:0BB1DD00901AADEBF0A3EAF0A3E9F03C
:0BB1E800901AB0EBF0A3EAF0A3E9F02E
:10B1F300901AB0E0FBA3E475F00112185EA9F0FA0F
:10B20300740C1217777B017A05792D12C7E7901A10
:10B21300B0E0FBA3E475F00112185EA9F0FAEF1297
:10B223001777E4FEEEC39F5023742D2EF582E4348A
:10B2330005F583E0FD901AB0E0FBA3E475F001127D
:10B24300185EA9F0FAED1217770E80D8901AB0E0C5
:07B25300FBA3E0FAA3E0F900
:01B25A0022D1
:10887C00901AADEBF0A3EAF0A3E9F0901AA5E0FC96
:09888C00A3E0FDA3E0FEA3E0FF60
:10889500901AB0EBF0A3EAF0A3E9F0A3121BBCE435
:1088A500FFFEFDFC901AB3E0F8A3E0F9A3E0FAA3FC
:1088B500E0FBC3121ACF700A901AB3121BC800004E
:1088C5008CA0901AB0E0FBA3E475F00112185EA924
:1088D500F0FA7433121777901AB0E0FBA3E475F041
:1088E5000112185EA9F0FA7404121777901AB3E012
:1088F500FCA3E0FDA3E0FEA3E0FF7818121AE090C8
:108905001AB0E0FBA3E475F00112185EA9F0FAEFC6
:10891500121777901AB3E0FCA3E0FDA3E0FEA3E0F5
:10892500FF7810121AE0901AB0E0FBA3E475F0018D
:1089350012185EA9F0FAEF121777901AB3E0FCA3AC
:10894500E0FDA3E0FEA3E0FF7808121AE0901AB05C
:10895500E0FBA3E475F00112185EA9F0FAEF121717
:1089650077901AB3A3A3A3E0FF901AB0E0FBA3E4AA
:1089750075F00112185EA9F0FAEF121777901AB088
:09898500E0FBA3E0FAA3E0F922F3
:0BB34E00901AADEBF0A3EAF0A3E9F0C9
:10B35900901AB0EBF0A3EAF0A3E9F0901AB0E0FB81
:10B36900A3E475F00112185EA9F0FA743712177781
:10B37900901AB0E0FBA3E475F00112185EA9F0FA87
:10B389007402121777901AB0E0FBA3E475F001126A
:10B39900185EA9F0FA7401121777901AB0E0FBA3AE
:10B3A900E475F00112185EA9F0FA74031217779088
:0BB3B9001AB0E0FBA3E0FAA3E0F922C9
:10C67C007F0112A1EDE94A6014740229F9E43AFA37
:0DC68C0078517C1C7D017E007F041216D8C1
:01C69900227E
:10C6B7007F0312A1EDE94A6013740229F9E43AFAFB
:0CC6C70078557C1C7D017E000F1216D8F7
:01C6D3002244
:05BD8C00421BC3000092
:10B74900E4901BC5F0A3F0F9A3C9F0A3F0A3E9F0B5
:10B759007E007F047D007B017A1C79231221CF7E34
:10B76900007F047D007B017A1B79D21221CF7E00F4
:10B779007F047D007B017A1B79CE1221CF7E007F69
:10B78900497D007B017A1B79D61221CF901BCD749C
:10B79900FFF0901BCCF0901BCBF0901BCAF0901CD3
:0DB7A9001F74E0F0E4A3F0A3F0A304F0226D
:10C31C00128A9C901AB8EFF030E21012791DC3EF1C
:10C32C00648094804012128FB5800D901AB8E03062
:0DC33C00E60612777E129647901AB8E0FFD1
:01C3490022D1
:108A9C00E4901BC5F0A3F0126E51D3EF9400EE647A
:108AAC0080948050037F002212BC69EF901B1AF057
:108ABC00A3E4F012BC69901B1BE02FF0901B1AE092
:108ACC003EF0E0FEA3E0FFD394EEEE94055004EFED
:108ADC004E700612C7D17F0022900A73E0FBA3E010
:108AEC00FAA3E0F9901B1AE0FEA3E0FFE92FF9EAE4
:108AFC003EFAA3EBF0A3EAF0A3E9F0901B1CA3E071
:108B0C00FAA3E0D39012779582EA9583500E901BCE
:108B1C001CE0F9A3A3E0901BC7C9802C900A73A397
:108B2C00E0FAA3E0FFC374779FFF74129AFEC39020
:108B3C001B1BE09FFF901B1AE09EFE74772FF974AD
:108B4C000E3EFA901BC77401F0A3EAF0A3E9F012F1
:108B5C00AF48EF1460090470037F20227F002212BB
:108B6C00655A901B19EFF06004E030E3051296474C
:108B7C008025901B19E0FF20E00620E10330E2176E
:108B8C00901B397401F0A3741CF0A3744BF07B019F
:0C8B9C007A1C7923129FA5901B19E0FFA2
:018BA80022AA
:1069FF00901AEDEDF0901AEAEBF0A3EAF0A3E9F0AC
:106A0F004A70037F8522901663E0FEF46017901A98
:106A1F00EAE0FBA3E0FAA3E0F9121874644445F02E
:106A2F0060037FA422EE6401601D78477C1C7D010A
:106A3F007B017A1B79CE7E007F041221ABEF339559
:106A4F00E04F70037F8522901AEFE02414F0901A24
:106A5F00EEE03400F0901BC4E004F07006901BC30E
:106A6F00E004F0901BC3E0FFA3E0901AF6CFF0A371
:106A7F00EFF0901AEAE0FBA3E0FAA3E0F990001D13
:106A8F00121717901AED30E406E0FF74048004E04B
:106A9F00FF7440901AF8F0A3EFF0901AEEE0FCA309
:106AAF00E0FDE4901B36F0A3F0901AF8E0FFA3E0AE
:106ABF00901B38CFF0A3EFF0A37401F0A3741CF078
:106ACF00A37447F0901AEAE0FBA3E0FAA3E02404D2
:106ADF00F9E43AFA901B3DEBF0A3EAF0A3E9F0E4F6
:106AEF00A3F0901AF6E0FAA3E0FB7F007E45125E5A
:106AFF0004901AF0121BBC901AF0E0FCA3E0FDA367
:106B0F00E0FEA3E0FF7808121AE0A3EFF0901AF06E
:106B1F00A3A3E0FEA3E0FF901AF5EFF0901AEDE0CB
:106B2F00B40107E4901AFAF08012901663E0B401F2
:106B3F00047F0180027F00901AFAEFF0901AEAE0CA
:106B4F00FBA3E0FAA3E0F9901AFAE0901B00F07DA6
:106B5F00007C08127D85EF64016001227F4512C71A
:106B6F008BE4FF12C78B901AEEE0FF12C78B901ABF
:106B7F00EEA3E0FF12C78B901AF6E0FF12C78B90BF
:106B8F001AF6A3E0FF12C78BE4FF12C78BE4FF12C4
:106B9F00C78B901AEAE0FBA3E0FAA3E0F990001D7F
:106BAF0012171730E4047F0480027F4012C78B90C6
:106BBF001AEDE0FF12C78B901AF4E0FF12C78B900B
:106BCF001AF5E0FF12C78B901C47E0FF12C78B909E
:106BDF001C48E0FF12C78B901C49E0FF12C78B9037
:106BEF001C4AE0FF12C78B901AEAE0FBA3E0FAA35E
:106BFF00E0F9900004121717FF12C78B901AEAE002
:106C0F00FBA3E0FAA3E0F9900005121717FF12C7D4
:106C1F008B901AEAE0FBA3E0FAA3E0F990000612CA
:106C2F001717FF12C78B901AEAE0FBA3E0FAA3E055
:0D6C3F00F9900007121717FF12C78B7F0195
:016C4C002225
:10964700901BC7E0FBA3E0FAA3E0F9C003C002C088
:1096570001900A73E0FBA3E0FAA3E0F9D082D0837C
:10966700D0E06B7008E965827003EA6583700302D6
:10967700972E901BC7E0FBA3E0FAA3E0F9C003C055
:1096870002C001900A73A3E0FAA3E0F9C3D082D025
:1096970083D0E0E99582EA9583501F900A73A3A3CC
:1096A700E0AE02FF901BC7A3E0FAA3E0C39FFFEA67
:1096B7009E901B22F0A3EFF08027901BC7A3E0FA30
:1096C700A3E0AE02FF900A73A3E0FAA3E0C39FFFF3
:1096D700EA9EFEC3E49F901B23F074049E901B2216
:1096E700F0901278E0FEA3E0FFD3901B23E09F9059
:1096F7001B22E09E400302C7D1C2AF901B22E0FEAF
:10970700A3E0FFC3901279E09FF0901278E09EF0FB
:10971700901BC7E0F9A3E0FAA3E0900A73C9F0A38E
:07972700EAF0A3E9F0D2AF64
:01972E002218
:10655A00E4901B27F012BC69901B24EFF0E0FE5474
:10656A000FA3F0EEC4540F640460030267ADE0FFAA
:10657A00C3940550030267ADEF25E025E0F0C3940C
:10658A0014A3F012BC69901B1FEFF012BC69EF90C4
:10659A001BC5F0A3E4F012BC69901BC6E02FF09073
:1065AA001BC5E03EF0C3A3E09414901BC5E0940021
:1065BA0050037F002212BC69EF901B28F0A3E4F07D
:1065CA0012BC69901B29E02FF0901B28E03EF012C4
:1065DA00BC69EF901B2AF0A3E4F012BC69901B2B54
:1065EA00E02FF0901B2AE03EF0A3E030E507901B75
:1065FA0027E04410F012BC69901B20EFF012BC692E
:10660A00901B21EFF014601D14602324F1600D2407
:10661A000B7024901B27E04401F08022901B27E096
:10662A004402F08019901B27E04404F08010901B6C
:10663A0027E04440F08007901B27E04408F012BC92
:10664A0069901B22EFF012BC69901B23EFF012BC79
:10665A0069901C23EFF012BC69901C24EFF012BC65
:10666A0069901C25EFF012BC69901C26EFF0901C73
:10667A0023E0FFC394E04009EFD394EF50037F0077
:10668A002212BC69901BD2EFF012BC69901BD3EFA7
:10669A00F012BC69901BD4EFF012BC69901BD5EFC5
:1066AA00F012BB19EF7047901C47E0FF901BD2E035
:1066BA00FE6F6004EEF47033901C48E0FF901BD329
:1066CA00E0FE6F6004EEB4FF22901C49E0FF901BCD
:1066DA00D4E0FE6F6004EEB4FF11901C4AE0FF9014
:1066EA001BD5E0FE6F6007EEF460037F0022901B6B
:1066FA0024E0FE901B1FE0FDEDFFC006C007901BC3
:10670A00C5E0FCA3E0FD901B2AE0FFA3E0901B3646
:10671A00CFF0A3EFF0901B20E0FEA3E0FBEBFF908D
:10672A001B38EEF0A3EFF0A37401F0A3741BF0A3DF
:10673A0074D2F0A37401F0A3741CF0A37423F09034
:10674A001B26E0901B40F0901B28E0FAA3E0FBD048
:10675A0007D006125E04901B2C121BBC901B2CE067
:10676A00FCA3E0FDA3E0FEA3E0FF7808121AE09084
:10677A001B22E0B50711901B2CA3A3A3E0FF901BDB
:10678A0023E0FEEF6E60037F0022901B25E0FFC32B
:10679A00901BC6E09FF0901BC5E09400F0901B2769
:0567AA00E0FF227F006A
:0167AF0022C7
:10BB1900E4901B30F078D27C1B7D017B017A1C7983
:10BB29001FFE7F041221ABEF7005901B3004F090CB
:10BB39001B30E0702A7B017A1B79D212AE38E94AB0
:10BB4900601D90000612171760159000071217174D
:10BB5900FF64016004EFB40206901B307401F09099
:04BB69001B30E0FFAE
:01BB6D0022B5
:0E5E0400901B32ECF0A3EDF0A3EAF0A3EBF05C
:105E1200E4FCFD901B41121BBC901B41E0F8A3E087
:105E2200F9A3E0FAA3E0FBC000C001C002C00390E6
:105E32001B3AE0FBA3E0FAA3E0F990000112171766
:105E4200FD1216FEFEEDFFE4FCFDD003D002D001F0
:105E5200D000EB2FFFEA3EFEED39FDEC38FC901B43
:105E620041121BBC901B41E0F8A3E0F9A3E0FAA3A6
:105E7200E0FBC000C001C002C003901B3AE0FBA3DC
:105E8200E0FAA3E0F9900002121717FE9000031245
:105E92001717FDEDFFE4FCFDD003D002D001D000C6
:105EA200EB2FFFEA3EFEED39FDEC38FC901B411270
:105EB2001BBC901B41E0F8A3E0F9A3E0FAA3E0FBCE
:105EC200901B32E0FEA3E0FFE4FCFDEB2FFFEA3E75
:105ED200FEED39FDEC38FC901B41121BBC901B41BE
:105EE200E0F8A3E0F9A3E0FAA3E0FB901B34E0FEA4
:105EF200A3E0FFE4FCFDEB2FFFEA3EFEED39FDECF3
:105F020038FC901B41121BBC901B41E0F8A3E0F946
:105F1200A3E0FAA3E0FB901B36E0FEA3E0FFE4FC63
:105F2200FDEB2FFFEA3EFEED39FDEC38FC901B4104
:105F3200121BBC901B41E0F8A3E0F9A3E0FAA3E036
:105F4200FB901B38E0FEA3E0FFE4FCFDEB2FFFEA31
:105F52003EFEED39FDEC38FC901B41121BBC901B40
:105F620041E0F8A3E0F9A3E0FAA3E0FBC000C0011E
:105F7200C002C003901B3DE0FBA3E0FAA3E0F9904E
:105F82000001121717FD1216FEFEEDFFE4FCFDD014
:105F920003D002D001D000EB2FFFEA3EFEED39FD27
:105FA200EC38FC901B41121BBC901B41E0F8A3E0B3
:105FB200F9A3E0FAA3E0FBC000C001C002C0039055
:105FC2001B3DE0FBA3E0FAA3E0F9900002121717D1
:105FD200FE900003121717FDEDFFE4FCFDD003D085
:105FE20002D001D000EB2FFFEA3EFEED39FDEC3886
:105FF200FC901B41121BBC901B40E0606120E05EE4
:10600200E4901B47F0901B40E0FF901B47E0C39FCA
:10601200504C12BC69EF901B45F0A3E4F012BC692E
:10602200901B46E02FF0901B45E03EF0901B41E0B4
:10603200F8A3E0F9A3E0FAA3E0FBA3E0FEA3E0FFEC
:10604200E4FCFDEB2FFFEA3EFEED39FDEC38FC905F
:106052001B41121BBC901B47E02402F080A7901B3F
:1060620041E0FCA3E0FDA3E0FEA3E0FF12B58D90AA
:106072001B41121BBC901B41E0FCA3E0FDA3E0FE10
:03608200A3E0FF99
:0160850022F8
:10791D00901ABA74FFF012BC69901AB9EFF06408AE
:10792D006003027AA1901BC5E0FEA3E0FFD394484B
:10793D00EE94004003027AA1C3EF9404EE9400503C
:10794D0003027AA1E4901B3BF0A3F0A304F0E4A39F
:10795D00F0F9A3C9F0A3F0A3E9F0E4A3F0A3F07B41
:10796D00017A1C7923FDFC125292901ABAEFF0C3E2
:10797D00648094805003027AA112BC69901AB9EF09
:10798D00F0901BC6E024FEFE901BC5E034FF901A5C
:10799D00BCF0A3CEF0901ABAE0901BD6F0901ABCB2
:1079AD00E0FCA3E0FDEC901BD7F0EDA3F0901ABD29
:1079BD0024FEF0901ABCE034FFF012BC69901ABBA3
:1079CD00EFF012BC69901ABBE02408F0C394085084
:1079DD00010F901ABBE0901BD9F0A3EFF0901ABEE7
:1079ED007401F0A3741BF0A374DBF0900A73A3E091
:1079FD00FAA3E0FFC374779FFF74129ACF2401CFCF
:107A0D003400901AC1F0FCA3EFF0FD901ABCE0FE1B
:107A1D00A3E0FFD39DEE9C501AA3E0FBA3E0FAA3D5
:107A2D00E0F8AC02AD03900A73E0FBA3E0FAA3E02B
:107A3D00F9805E901AC1E0FEA3E0FF901ABEE0FB54
:107A4D00A3E0FAA3E0F8AC02AD03900A73E0FBA348
:107A5D00E0FAA3E0F91216D8901AC1E0FEA3E0FFF8
:107A6D00C3901ABDE09FF0901ABCE09EF0E0FCA31D
:107A7D00E0FDC004C005A3E0FBA3E0FAA3E02FF9ED
:107A8D00EA3EA801FCAD037B017A0E7978D007D0D0
:0C7A9D00061216D8129647901ABAE0FFA5
:017AA90022BA
:108FB500901BD6E0901ABBF0C364809480500302E6
:108FC50090ACE0FFFD3395E0FC90129975F03DED16
:108FD500121C1DEC75F03DA42583F583E020E0030C
:108FE5000290ACEF3395E0FE7C007D3D1217AB742B
:108FF5007B2FF974123EFA7B01901ABCEBF0A3EAC1
:10900500F0A3E9F090001B121717640160030290AA
:10901500AC901BD7E0901AB9F0A3E4F0901BD8E010
:10902500FF901ABAE02FF0901AB9E03400F0E0FE94
:10903500A3E0FFD39446EE940050647A1B79D9C01F
:1090450003C002C001901ABCE0FBA3E0FAA3E0F95B
:1090550090000E121CF1901ABCE0FBA3E0FAA3E00D
:10906500F9900011EE8FF012197BEF2402FFE43E18
:10907500901AEEF0A3EFF07D011269FFEF6020E496
:10908500FF12C78BE4FF12C78B901ABCE0FBA3E06D
:10909500FAA3E0F9901AB9E0FCA3E0FD12C09B9099
:0790A5001ABBE0FF12A62533
:0190AC0022A1
:10C7D100C2AF12C4CD901BC77401F0A3740EF0A3B5
:06C7E1007478F0D2AF22D3
:10C61F00901B3BEFF07B017A0A7978900A6AEBF076
:10C62F00A3EAF0A3E9F0A3EBF0A3EAF0A3E9F02269
:10C4CD007B017A0E7978900A73EBF0A3EAF0A3E979
:10C4DD00F0900A70EBF0A3EAF0A3E9F0E490127883
:04C4ED00F0A3F022A6
:0EC8CE0012C4CDE4FF12C61FE490127AF022CD
:10C05E0090127AE0601F7B017A1B79367D587C0244
:10C06E0012AD9E7B017A1B793612B9AAEF7006903B
:10C07E00127AE070EE90127AE070057F0112C61F00
:0CC08E0090127AE070047F0180027F00B5
:01C09A002283
:10C77200C2AF438901758C60758A7FD28CD2A9E4DD
:09C78200900A76F0A3F0D2AF2278
:10C5DE00C28C758C60758A7FD28C900A77E004F0DD
:10C5EE007006900A76E004F012C3A612972F02BFCF
:01C5FE00DD5F
:10C559007E037FD07D007B017A12797B1221CF1275
:10C56900B74912C77212C8B112C4A912C8A212C817
:01C57900F4CD
:01C57A00229E
:10A95E00C003C002C001901A66E0FFA3E0901B3B4B
:10A96E00CFF0A3EFF0901A69E0901B3DF0901A6AB9
:10A97E00E0901B3EF0901A6BE0F9A3E0FAA3E09092
:10A98E001B3FC9F0A3EAF0A3E9F0901A6EE0FFA313
:10A99E00E0901B42CFF0A3EFF0D001D002D0031213
:10A9AE005292901A70EFF0901A69E06406703D9022
:10A9BE001A70E0FFC3648094804031EF3395E0FE5F
:10A9CE007C007D3D1217AB747B2FF974123EFA7B1F
:10A9DE0001901A68E0FF128DBED3EF648094805010
:10A9EE000B901A70E0FF12A6257F8422901A70E059
:01A9FE00FF59
:01A9FF002235
:10529200901B36EBF0A3EAF0A3E9F0A3ECF0A3ED48
:0152A200F01B
:1052A300901B447482F0901B3DE0FE146018146060
:1052B3001524FC601124F5600D240D700E901B3E27
:1052C300E0B420078000E4901B44F0901B44E0FF0F
:1052D300B4820122901B36E0FBA3E0FAA3E0F912AB
:1052E30016FEFFC394E0400DEFD394EF5007901BDD
:1052F3003EE04410F0901B39E07002A3E0700EEE24
:1053030064066036901B3DE0B41102802D901B3D76
:10531300E0B40607A3E030E402801F1216FE64E047
:1053230070219000011217177019900002121717BD
:1053330070119000031217177009901B447485F0C5
:105343000255BF901B3BE0FCA3E0FD901B36E0FB46
:10535300A3E0FAA3E0F9901B3DE0901B4FF0901BF4
:1053630039E0FEA3E0FF1282AB901B45EBF0A3EA0A
:10537300F0A3E9F04A602C901B45E0FBA3E0FAA3FD
:10538300E0F990001C12171775F03DA42499F582DB
:10539300E5F03412F583E030E009901B447481F0AA
:1053A3000255BF12C42A901B44EFF06480700302BD
:1053B30055BF7E007F3DC006C0077F00C007E0FFEA
:1053C3003395E0FE7C007D3D1217AB747B2FF9749F
:1053D300123EFA7B01D005D007D0061221CF901BD5
:1053E30044E0FF3395E0FE7C007D3D1217AB747BF8
:1053F3002FF974123EFA7B01A3EBF0A3EAF0A3E9C1
:10540300F0901B44E090001C121789901B39E0FFB9
:10541300A3E0CF8FF012195C901B3BE0FEA3E0FFEB
:10542300901B45E0FBA3E0FAA3E0F9900002EE8FA6
:10543300F012197B901B36E0FBA3E0FAA3E0F9120C
:1054430016FEFF901B45E0FBA3E0FAA3E0F99000F2
:1054530004EF121789901B36E0FBA3E0FAA3E0F9EF
:10546300900001121717FF901B45E0FBA3E0FAA37E
:10547300E0F9900005EF121789901B36E0FBA3E0DB
:10548300FAA3E0F9900002121717FF901B45E0FB07
:10549300A3E0FAA3E0F9900006EF121789901B36F8
:1054A300E0FBA3E0FAA3E0F9900003121717FF90C3
:1054B3001B45E0FBA3E0FAA3E0F9900007EF121706
:1054C30089901B3EE0FF64207044901B3DE0640420
:1054D300703C901C4BE0900008121789901C4CE024
:1054E300900009121789901C4DE090000A12178949
:1054F300901C4EE090000B121789901C4FE0900017
:105503000C121789901C50E090000D121789901B04
:105513003DE0FE901B45E0FBA3E0FAA3E0F9900019
:105523001BEE12178990001DEF121789901B3FE0A5
:10553300FBA3E0FAA3E0F9EA494B604EA3E0FCA326
:10554300E0FD4C6045C003C002C001901B45E0FB79
:10555300A3E0FAA3E0F9900013121CF1901B3FE0C3
:10556300FBA3E0FAA3E02DF9EA3CFAE924FFF9EA08
:1055730034FFFAC003C002C001901B45E0FBA3E067
:10558300FAA3E0F9900016121CF1EEB4060E901B7C
:1055930045E0FBA3E0FAA3E0F9129474901B44E006
:1055A300FF3395E0FE90129975F03DEF121C1DEE4E
:1055B30075F03DA42583F583E04401F0901B44E09E
:0155C300FFE8
:0155C40022C4
:1075D100901C82EBF0A3EAF0A3E9F0901C81EFF09C
:1075E100901C8A74FFF0A37489F0E4A3F0A3F0C3A4
:1075F100EF64809480400B901C81E0FD6480949046
:1076010040057EFF7F8522EDFF3395E0FE901299C4
:1076110075F03DEF121C1DEE75F03DA42583F58339
:10762100E020E0057EFF7F862290165DE0FF700579
:107631007EFF7F9D22901663E0B4FF1AEF640A601B
:1076410004EFB40B1190164DE0FCA3E0FDA3E0FEA6
:10765100A3E0FF12938712B25B901C81E0FF339588
:10766100E0FE7C007D3D1217AB747B2FF974123E56
:10767100FA901C877401F0A3EAF0A3E9F0901C8250
:10768100E0FBA3E0FAA3E0F9EA494B6034A3E0FE92
:10769100A3E0FF4E602BC003C002C001901C87E035
:1076A100FBA3E0FAA3E0F990000E121CF1901C87F5
:1076B100E0FBA3E0FAA3E0F9900011EE8FF01219BC
:1076C1007B901C87E0FBA3E0FAA3E0F990001B127A
:1076D100171764066003027763901C87E0FBA3E041
:1076E100FAA3E0F9127042901C8CEEF0A3EFF0D3F4
:1076F1009400EE648094804060901C8AE0B4FF2383
:10770100A3E0B4891E901C81E0FF7B007A00790020
:10771100E4901AA6F0A3127228901C8AEEF0A3EF4F
:10772100F080D6901C8AE0FEA3E0FFC3EE64809453
:10773100805011EF64877002EEF46008A3EEF0A3AD
:10774100EFF08015901C87E0FBA3E0FAA3E0F9902D
:10775100002412189F45F07080901C8CE0FEA3E07D
:10776100FF22901C87E0FBA3E0FAA3E0F990001B45
:0C777100121717B4110302740DE4FEFFA0
:01777D0022E9
:10C87000901CA1E0FDA3E0901AA6CDF0A3ED1272EA
:02C8800028226C
:09722800F0A37402F0A37458F005
:0D723100901AA3EBF0A3EAF0A3E9F0AD077B
:10723E00E4901AAAF0A3F0C3ED648094804007EDA9
:10724E0064809490400302731FEDFB3395E0FA9037
:10725E00129975F03DEB121C1DEA75F03DA42583C5
:10726E00F583E020E0057EFF7F862290165DE070BC
:10727E00057EFF7F9D227C007D3DAF03AE0212177F
:10728E00AB747B2FF974123EFA901AAC7401F0A312
:10729E00EAF0A3E9F0901AA3E0FBA3E0FAA3E0F969
:1072AE00EA494B604EA3E0FEA3E0FF4E6045C003EB
:1072BE00C002C001901AACE0FBA3E0FAA3E0F99083
:1072CE000013121CF1901AA3E0FBA3E0FAA3E02F27
:1072DE00F9EA3EFAE924FFF9EA34FFFAC003C002E4
:1072EE00C001901AACE0FBA3E0FAA3E0F9900016FF
:1072FE00121CF1901AACE0FBA3E0FAA3E0F99000A7
:10730E001B121717B4110F900013121CC1E94A700B
:10731E00057EFF7F8522901AACE0F9A3E0FAA3E088
:10732E00A3C9F0A3EAF0A3E9F0901AA8E0FCA3E049
:10733E00FD4C60097B017A1A79B212AD9E12C31C04
:10734E00901AB7EFF054077029901AA8E07002A3B4
:10735E00E0600C7B017A1A79B212B9AAEF60057E51
:10736E00FF7F872212B25B12C918BF9AD07EFF7FB1
:10737E009A22901AB7E0FF20E2C3EF30E0197B01AA
:10738E007A1A79AC1222C7901AAAEEF0A3EFF0BEC9
:10739E00FF1DBFFA1A805F901AB7E030E1117B0132
:1073AE007A1A79AC124B6C901AAAEEF0A3EFF09009
:1073BE001AAFE0FBA3E0FAA3E0F9C003C002C001DC
:1073CE00901AACE0FBA3E0FAA3E0F9D082D083D010
:1073DE00E06B7008E965827003EA65836018901AA5
:1073EE00AFE0F9A3E0FAA3E0901AACC9F0A3EAF07B
:0E73FE00A3E9F002734B901AAAE0FEA3E0FF91
:01740C00225D
:05A36900901CA7EFF0BD
:10A36E00C3648094804008E0FD6480949040057E34
:10A37E00FF7F8522EDFF3395E0FE90129975F03D3B
:10A38E00EF121C1DEE75F03DA42583F583E020E051
:10A39E00057EFF7F862290165DE0700D901CA7E073
:10A3AE00FF12A6257EFF7F9D22901CA7E0FF33950E
:10A3BE00E0FE7C007D3D1217AB747B2FF974123ECC
:10A3CE00FA7B01A3EBF0A3EAF0A3E9F090001B12D5
:10A3DE001717B4060E901CA8E0FBA3E0FAA3E0F951
:10A3EE0012C01F901CA7E0FF3395E0FE90129975E6
:10A3FE00F03DEF121C1DEE75F03DA42583F583E4B0
:10A40E00F0901CA8E0FBA3E0FAA3E0F9E4F5F0124B
:05A41E00195CE4FEFFE3
:01A423002216
:05A62500901B36EFF070
:10A62A00C3648094804008E0FD6480949040057E75
:10A63A00FF7F8522EDFF3395E0FE90129975F03D7C
:10A64A00EF121C1DEE75F03DA42583F583E020E092
:10A65A00057EFF7F8622901B36E0FF3395E0FE7C65
:10A66A00007D3D1217AB747B2FF974123EFA7B0101
:10A67A00A3EBF0A3EAF0A3E9F090001B121717B4BA
:10A68A00060E901B37E0FBA3E0FAA3E0F912B8E943
:10A69A00901B36E0FF3395E0FE90129975F03DEF7E
:10A6AA00121C1DEE75F03DA42583F583E4F0901B82
:10A6BA0037E0FBA3E0FAA3E0F9E4F5F012195CE451
:02A6CA00FEFF91
:01A6CC00226B
:10C09B0090165DE06033E94A601390001B1217178E
:10C0AB00B4060A90002074FF121744800090127A95
:10C0BB007401F01258B4E490127AF0D3EF9400EEBE
:0BC0CB006480948040057F01227F9D6F
:01C0D6002247
:10C3D300EE7024EF24EC601314601024FC6010242E
:10C3E300D4601024F570107D81800E7D02800A7D5B
:0BC3F3000480067D088002E4FDAF0519
:01C3FE00221C
:1082AB00901B48EEF0A3EFF0A3ECF0A3EDF0A3EBE3
:0782BB00F0A3EAF0A3E9F0D3
:1082C200901663E0901B54F0901B51E4F0A3F0A3CE
:1082D200F0901B4CA3E0FAA3E04A70030283D8E4B7
:1082E200901B50F0901B50E0FFC394104003028398
:1082F200D875F03DEFA4247BF582E5F03412F583C6
:10830200E0FEA3E0FF901B48E0FCA3E0FDEF6D70F0
:1083120002EE6C60030283CF901B50E0FF75F03DCC
:10832200A4247DF582E5F03412F583E0FCA3E0FDA0
:10833200901B4AE0FAA3E0FBED6B7002EC6A60036B
:108342000283CF75F03DEFA42496F582E5F0341256
:10835200F583E0FF901B4FE0FEEF6E7070901B54B0
:10836200E0B40124901B50E075F03DA4247FF97421
:108372001235F0A801FC7D017B017A1B79CA7E00CF
:108382007F041221ABEF6029901B50E075F03DA4F1
:10839200247FF9741235F0A801FC7D01901B4CE09A
:1083A200FBA3E0FAA3E0F97E007F041221ABEF7099
:1083B2001C901B50E075F03DA4247BF9741235F03B
:1083C200FAA37401F0A3EAF0A3E9F08009901B502C
:1083D200E004F00282E6901B51E0FBA3E0FAA3E086
:0183E200F9A1
:0183E3002277
:10C42A007F80E4FEEEFD3395E0FC90129975F03DB5
:10C43A00ED121C1DEC75F03DA42583F583E020E088
:0AC44A0004AF0680050EEEB410DA10
:01C4540022C5
:04C90E0012C8102219
:0B4B6C00901AB8EBF0A3EAF0A3E9F008
:104B770012BC69EF901AC1F0A3E4F012BC69901A55
:104B8700C2E02FF0901AC1E03EF012BC69EF901A14
:104B9700BFF0A3E4F012BC69901AC0E02FF0901A9E
:104BA700BFE03EF0E0FEA3E0FFA3E0FCA3E0FD7B57
:104BB700017A1C7923901B4F7411F01282AB901A63
:104BC700CBEBF0A3EAF0A3E9F04A6003024C649050
:104BD7001ABFE0FEA3E0FF7B017A1C7923901B4FED
:104BE7007411F0E4FDFC1282AB901ACBEBF0A3EA50
:104BF700F0A3E9F04A7025901ABFE0FEA3E0FF7B1F
:104C0700017A1B79CE901B4F7411F0E4FDFC1282E0
:104C1700AB901ACBEBF0A3EAF0A3E9F0901ACBE044
:104C2700FBA3E0FAA3E0F94A6012901AC1E0FFA3E0
:104C3700E0900002CF8FF012197B80217B007A0071
:104C47007900C003C002C001901AB8E0FBA3E0FAE4
:104C5700A3E0F9121C72129647E4FEFF22901ACBCA
:104C6700E0FBA3E0FAA3E0F9C003C002C001901A79
:104C7700B8E0FBA3E0FAA3E0F9121C72901ACBE0AC
:104C8700FBA3E0FAA3E0F990000412171770549001
:104C9700001D12171730E423901BD2E09000041276
:104CA7001789901BD3E0900005121789901BD4E059
:104CB700900006121789901BD58021901C23E09045
:104CC7000004121789901C24E090000512178990A0
:104CD7001C25E0900006121789901C26E09000071B
:104CE70012178912BC69EF901AC5F0A3E4F012BC41
:104CF70069901AC6E02FF0901AC5E03EF0C3A3E012
:104D07009408901AC5E0940050227B007A0079003D
:104D1700C003C002C001901AB8E0FBA3E0FAA3E009
:104D2700F9121C721296477EFF7FFF2212BC69EFB1
:104D3700901ABDF0A3E4F012BC69901ABEE02FF000
:104D4700901ABDE03EF0901AC7121BC80000000081
:104D5700E4901ACEF0A3F0901ABDE07002A3E060D1
:104D670042901AC5E0FCA3E0FD901AC1E0FFA3E062
:104D7700901AEFCFF0A3EFF0A37401F0A3741BF028
:104D8700A374D2F0A37401F0A3741CF0A37423F0EE
:104D9700901ABFE0FAA3E0FB7F11126C4D901AC77F
:104DA700121BBC901AC6E024F8F0901AC5E034FF35
:104DB700F0E0FEA3E0FF901AC3EEF0A3EFF04E7011
:104DC70003024EB0E4901ABCF0901AC3E0FEA3E0D1
:104DD700FF901ACBE0FBA3E0FAA3E0F912C8FF1299
:104DE700BC69901ABBEFF0901ABDE07002A3E060B7
:104DF70057901ABCE0901ABB700FE0901ACEF0A340
:104E0700E4F0901ABC04F0803FE0FF901ACFE02F47
:104E1700F0901ACEE03400F0901AC7E0F8A3E0F95A
:104E2700A3E0FAA3E0FB901ACEE0FEA3E0FFE4FCC8
:104E3700FDEB2FFFEA3EFEED39FDEC38FC901AC77B
:104E4700121BBCE4901ABCF0901ABBE0FF901ACB7F
:104E5700E0FBA3E0FAA3E0F912A773901AC374FF6B
:104E6700F5F012184845F06003024DE6901ABDE0D0
:104E77007002A3E06047901ABCE06041901AC7E057
:104E8700F8A3E0F9A3E0FAA3E0FB901ACEE0FEA3B3
:104E9700E0FFE4FCFDEB2FFFEA3EFEED39FDEC38C9
:104EA700FC901AC7121BBC8014901ACBE0FBA3E03E
:104EB700FAA3E0F9900019E4F5F012197B901ABDF6
:104EC700E07002A3E0603E901AC7E0FCA3E0FDA3F8
:104ED700E0FEA3E0FF12B58D901AC7121BBC901A13
:104EE700BDE0FEA3E0FFE4FCFD901AC7E0F8A3E0F5
:104EF700F9A3E0FAA3E0FBC3121ACF6008129647A2
:104F07007EFF7FFC22901ACBE0FBA3E0FAA3E0F937
:104F170012C912129647901ACBE0FBA3E0FAA3E05E
:0A4F2700F990001912189FFFAEF078
:014F3100225D
:0B740D00901AA2EBF0A3EAF0A3E9F054
:107418004A70057EFF7F8522901AA2E0FBA3E0FA5E
:10742800A3E0F912C34A901AA5EEF0A3EFF04E704C
:1074380003FEFF22901AA2E0FBA3E0FAA3E0F99072
:10744800000E121CC1901AA9EBF0A3EAF0A3E9F010
:10745800901AA6E02408FF901AA5E03400FE901ABE
:10746800A7F0FCA3EFF0FD901AA2E0FBA3E0FAA3BB
:10747800E0F9121874FBAAF0C002C003901AA2E047
:10748800FBA3E0FA90000212189FFF901AEFE5F0B4
:10749800F0A3EFF0A37401F0A3741CF0A37447F0F9
:1074A800901AA2A3A3E02404F9E43AFA901AF4EBA0
:1074B800F0A3EAF0A3E9F0D003D0027F11126C4DDB
:1074C800C007901AA9E0FBA3E0FAA3E0F9901AA577
:1074D800E0FFA3E0901AF1CFF0A3EFF0D0071289F4
:1074E8008E12B58D901AACEEF0A3EFF0901AA2E0D0
:1074F800FBA3E0FAA3E0F990001B121717FD901AFE
:10750800A7E0FFA3E0901AEECFF0A3EFF0901AA245
:10751800A3A3E01269FFEF640160030275B6901A35
:10752800A2E0FBA3E0FAA3E0F9121874E5F0FF1259
:10753800C78B901AA2E0FBA3E0FAA3E0F912187433
:10754800FF12C78B901AA2E0FBA3E0FAA3E0F99020
:10755800000212189FE5F0FF12C78B901AA2E0FBF9
:10756800A3E0FAA3E0F990000212189FFF12C78B5C
:10757800901AA7E0FF12C78B901AA7A3E0FF12C7C3
:107588008B901AACE0FF12C78B901AACA3E0FF12E5
:10759800C78B901AA2E0FBA3E0FAA3E0F9A3E0FCF2
:1075A800A3E0FD12C09BD3EF648094805006EF33B4
:1075B80095E0FE22901AA2E0FBA3E0FAA3E0F9907E
:0875C800001112189FFFAEF044
:0175D0002298
:104F3200901B3174FFF012BC69EF4E600302528C79
:104F420012BC69EF64014E600302528C12BC69EF1D
:104F520064084E600302528C12BC69EF4E60030279
:104F6200528C12BC69EF64064E600302528C12BC72
:104F720069EF64044E600302528C12BC69EF4E600A
:104F82000302528C12BC69EF24FE70030251C30467
:104F9200600302528CE4901B22F012BC69901B2227
:104FA200E0242BF582E4341BF583EFF0901B22E022
:104FB20004F0E0C3940640E2E4901B22F012BC69C4
:104FC200901B22E02427F582E4341BF583EFF09056
:104FD2001B22E004F0E0C3940440E2E4901B22F0C0
:104FE20012BC69901B22E004F0E0C3940640F1E495
:104FF200901B22F012BC69901B22E02423F582E46C
:10500200341BF583EFF0901B22E004F0E0C394041C
:1050120040E2901C47E0FF901B23E06F60030252C6
:105022008C901C48E0FF901B24E06F600302528CBE
:10503200901C49E0FF901B25E06F600302528C90A8
:105042001C4AE0FF901B26E06F600302528C7B013A
:10505200901B3904F0A3741BF0A3742BF07A1B7914
:1050620027129FA574FF901B3BF0A3F0A37404F0DA
:10507200A37420F0A3E4F0A3F0A3F0A3F0A3F07BC9
:10508200017A1B792774FFFDFC125292901B32EFBA
:10509200F0C364809480500302528C901663E0F453
:1050A20060030251B812C05EEF70030251B8901B48
:1050B20032E0FF3395E0FE7C007D3D1217AB747B3E
:1050C2002FF974123EFA7B01A3EBF0A3EAF0A3E9F5
:1050D200F0E4FD12C2BEE4FF12C78B7F0212C78B3F
:1050E200E4901B22F0901B22E0FFC3940650177439
:1050F200072FF582E43400F583E0FF12C78B901B83
:1051020022E004F080DFE4901B22F0901B22E0FFFB
:10511200C39404501774232FF582E4341BF583E003
:10512200FF12C78B901B22E004F080DFE4901B2269
:10513200F0901B22E0FFC394065027901B33E0FB44
:10514200A3E0FAA3E02408F9E43AFA7E00E92FF991
:10515200EE3AFA1216FEFF12C78B901B22E004F001
:1051620080CFE4901B22F0901B22E0FFC3940450F6
:1051720027901B33E0FBA3E0FAA3E02404F9E43A0E
:10518200FA7E00E92FF9EE3AFA1216FEFF12C78BE9
:10519200901B22E004F080CF901B33E0FBA3E0FAE7
:1051A200A3E0F9E4FDFC12C09BD3EF64809480403D
:1051B20005E4901B31F0901B32E0FF12A62502524B
:1051C2008CE4901B22F012BC69901B22E0242BF588
:1051D20082E4341BF583EFF0901B22E004F0E0C37D
:1051E200940640E2E4901B22F012BC69901B22E07C
:1051F2002427F582E4341BF583EFF0901B22E004B0
:10520200F0E0C3940440E2E4901B22F012BC6990E7
:105212001B22E004F0E0C3940640F1E4901B22F06C
:1052220012BC69901B22E02423F582E4341BF5832F
:10523200EFF0901B22E004F0E0C3940440E2901CE3
:1052420047E0FF901B23E06F7040901C48E0FF9006
:105252001B24E06F7034901C49E0FF901B25E0B5E1
:105262000728901C4AE0FF901B26E0B5071C901B04
:10527200397401F0A3741BF0A3742BF07B017A1B29
:0F5282007927129FA5E4901B31F0901B31E0FFBC
:0152910022FA
:0FC8A2007E007F6E7D007B017A1B79550221CFCE
:039FA500901B36D8
:109FA80012B4AA901B3CEBF0A3EAF0A3E9F04A70C4
:109FB8000E12B437901B3CEBF0A3EAF0A3E9F09043
:109FC8001B3CE0FBA3E0FAA3E0F990000A12171784
:109FD80030E00302A06BE9240AF9E43AFA1216FE0B
:109FE8004401121777E4FF901B36E0FBA3E0FAA3C5
:109FF800E0F98F82758300121717FE901B3CE0FB77
:10A00800A3E0FAA3E0F98F82758300EE1217890F97
:10A01800EFB404D3E4FF901B39E0FBA3E0FAA3E01C
:10A02800F98F82758300121717FE901B3CE0FBA383
:10A03800E0FAA3E02404F9E43AFAEF7C0029F9EC09
:10A048003AFAEE1217770FEFB406CB901B3CE0FB01
:10A05800A3E0FAA3E0240AF9E43AFA1216FE54FE41
:03A0680012177755
:01A06B0022D2
:0398F000901B05C5
:1098F30012B4AA901B08EBF0A3EAF0A3E9F04A60C4
:10990300030299C1F9901B08C9F0A3F0A3E9F0740D
:10991300FF901B3BF0A3F0A37404F0A37420F0A307
:10992300E4F0A3F0A3F0A3F0A3F0901B05E0FBA3E6
:10993300E0FAA3E0F974FFFDFC125292901B0CEFC6
:10994300F0C3648094804076E0FF3395E0FE7C00B2
:109953007D3D1217AB747B2FF974123EFAA3740189
:10996300F0A3EAF0A3E9F0E4901B0BF0901B0DE0E9
:10997300FBA3E0FAA3E0F9128EBAEF6039901B0D56
:10998300E0FBA3E0FAA3E0F912BF56EF601C901BC3
:1099930005E0FBA3E0FAA3E0F912B4B2901B08EBD5
:1099A300F0A3EAF0A3E9F04A700C901B0BE004F07B
:1099B300E0C3940640B6901B0CE0FF12A625901B53
:0999C30008E0FBA3E0FAA3E0F9BF
:0199CC002278
:08B4AA00EBF0A3EAF0A3E9F0C6
:0BB4B200901B3FEBF0A3EAF0A3E9F0D1
:10B4BD00E4A3F0901B42E0FFC3940A504BEF75F0EC
:10B4CD000BA42455F9741B35F0FA7B01C003C0029F
:10B4DD00901B3FE0FBA3E0FAA3E0F8AC02AD03D074
:10B4ED0002D0037E007F041221ABEF7013901B423C
:10B4FD00E075F00BA42455F9741B35F0FA7B01228D
:0EB50D00901B42E004F080AB7B007A007900D6
:01B51B00220D
:10B43700E4901B3FF0901B3FE0FFC3940A501FEFBF
:10B4470075F00BA42455F582E4341BF583E07006F0
:10B45700901B3FE0803E901B3FE004F080D712C86E
:10B46700DC7C007D0A1217BD901B3FEDF0901B3F5F
:10B47700E0FF75F00BA4245FF582E4341BF583E04D
:10B4870030E010901B3FE004F0E075F00A84E5F02F
:10B49700F080DAEF75F00BA42455F9741B35F0FA38
:02B4A7007B0127
:01B4A9002280
:0B8EBA00901B10EBF0A3EAF0A3E9F01E
:108EC500E4901B14F0901663E064017003028FAF09
:108ED50012C05EEF7003028FAF901B10E0FBA3E0A2
:108EE500FAA3E0F97D0112C2BEE4FF12C78B7F0130
:108EF50012C78BE4901B13F0901B13E0FFC394067D
:108F0500501774072FF582E43400F583E0FF12C78C
:108F15008B901B13E004F080DFE4901B13F0901B93
:108F250013E0FFC39404501774472FF582E4341CF3
:108F3500F583E0FF12C78B901B13E004F080DFE49C
:108F4500901B13F0E4FF12C78B901B13E004F0E0B5
:108F5500C3940640EFE4901B13F0901B13E0FFC38E
:108F650094045027901B10E0FBA3E0FAA3E024042F
:108F7500F9E43AFA7E00E92FF9EE3AFA1216FEFF05
:108F850012C78B901B13E004F080CF901B10E0FB01
:108F9500A3E0FAA3E0F9E4FDFC12C09BD3EF6480E3
:0F8FA50094804006901B147401F0901B14E0FFA1
:018FB400229A
:0BBF5600901B10EBF0A3EAF0A3E9F051
:10BF61007B017A1B79147D587C0212AD9E7B017A8C
:10BF71001B791412B9AAEF701D128A9C901B13EF42
:10BF8100F030E5037F0122901B13E0FF60DF20E327
:08BF9100DC12964780D77F0007
:01BF99002285
:0EBD9100441C59C0A80202441C47C0A802036B
:0BC34A00901AAEEBF0A3EAF0A3E9F0BC
:10C3550090000E121CC1E94A7004FEFF8014901A69
:10C36500AEE0FBA3E0FAA3E0F990001112189FFFDD
:02C37500AEF028
:01C3770022A3
:09C8FF00900019E4F5F002197B28
:0BA77300901AD0EBF0A3EAF0A3E9F08D
:10A77E00900013121CC1E94A700302A817901AD058
:10A78E00E0FBA3E0FAA3E0F9900013121CC1C00392
:10A79E00C002C001901AD0E0FBA3E0FAA3E0F9904A
:10A7AE00001912189FD001D002D00329F9EA35F012
:10A7BE00FA901AD3EBF0A3EAF0A3E9F0901AD0E0E6
:10A7CE00FBA3E0FAA3E0F9900016121CC1C003C06F
:10A7DE0002C001901AD3A3E0FAA3E0F9D3D082D03D
:10A7EE0083D0E0E99582EA9583501E901AD3E0FB60
:10A7FE00EF121777901AD0E0FBA3E0FAA3E0F990DE
:09A80E000019E475F00112190FA4
:01A81700221E
:03C912007F012280
:10AAA000901AD8EBF0A3EAF0A3E9F0901AD8E0FBF3
:10AAB000A3E0FAA3E0F990001112189FFDACF0D3C7
:10AAC000EF9DEE9C40028004AC06AD07AE04AF05DE
:10AAD00090001112189FD39400E5F09400401E904E
:10AAE0001AD8E0FBA3E0FAA3E02411F9E43AFA1241
:10AAF0001874C39FFDE5F09E8DF012195C901AD872
:10AB0000E0FBA3E0FAA3E0F990001112189FD394A0
:10AB100000E5F09400400A90000EA3EE8FF00219B9
:10AB20000F7B007A007900C003C002C001901AD8E0
:0FAB3000E0FBA3E0FAA3E0F990000E121CF12263
:03C915007F00227E
:03C918007F00227B
:03C91B007F002278
:0BC8F400C2AF12C8CED2AF129AA7222A
:10AF4800901B2174FFF090165DE06078E4901B2060
:10AF5800F012BC69901B20E004F0E0C3940640F1B5
:10AF6800E4901B20F012BC69901B20E0244BF58272
:10AF7800E4341CF583EFF0901B20E004F0E0C39468
:10AF88000640E212BC69901B1FEFF012BC69901BCF
:10AF98001FE0B40821EF24FA600C24067018901BF7
:10AFA800217401F08010901663E064016008124F6C
:10AFB80032901B21EFF0901B21E0D36480948050E5
:09AFC80003129647901B21E0FFE3
:01AFD100225D
:0B7D8500901AFBEBF0A3EAF0A3E9F07A
:107D90004A70037F852290165DE070037F9D22AEBE
:107DA00004AF05ED6003027ED9EE24F86003027E85
:107DB000D9901AFBE0FBA3E0FAA3E0F990001D12B2
:107DC000171730E4409000087401121789900009D9
:107DD000E412178990000A745E1217899000051248
:107DE0001717547F90000B1217899000061217176F
:107DF00090000C12178990000712171790000D12AF
:107E00001789027EB3901B00E06003027EB3901CD2
:107E100055E0FFF4601EEF601BE92404F9E43AFA30
:107E2000901B087401F0A3741CF0A37447F0126750
:107E3000B0EF6012901AFBE0FBA3E0FAA3E0240489
:107E4000F9E43AFA80067B017A1C79551298F09091
:107E50001B01EBF0A3EAF0A3E9F0901B01A3E0FA09
:107E6000A3E04A604BE4A3F0901B04E0FFC3940638
:107E70005041901B01E0FBA3E0FAA3E02404F9E4E5
:107E80003AFA7E00E92FF9EE3AFA1216FEFD901A40
:107E9000FBE0FBA3E0FAA3E02408F9E43AFAE92FB7
:107EA000F9EE3AFAED121777901B04E004F080B86F
:107EB0007FA12212C05EEF70037F8F22901AFBE039
:107EC000FBA3E0FAA3E0F9901B00E0FD12AFD27F24
:0B7ED0000812C78BE4FF12C78B7F0174
:017EDB002284
:10C2BE00E94A602B12AFD27F0812C78B7F0612C7D6
:10C2CE008BE4FF12C78B7F0112C78B7F0812C78BBF
:10C2DE00E4FF12C78B7F0612C78B7F0412C78B2217
:10C70B00900A6DE0FBA3E0FAA3E0F91216FEFF908E
:09C71B000A6EE475F001121848E1
:01C7240022F2
:10BE8300900A70E0FBA3E0FAA3E0F9EF12177790B2
:10BE93000A71E475F001121848900A70A3E0FAA33E
:10BEA300E0D39012779582EA9583400E900A7074DE
:10BEB30001F0A3740EF0A37478F0901279E004F00B
:09BEC3007006901278E004F022F0
:0BAFD200901B36EBF0A3EAF0A3E9F0BF
:10AFDD004A6075ED6016E4A3F07FFF12C78B901BDE
:10AFED0039E004F0E0C3940640EF8036E4901B395D
:10AFFD00F0901B39E0FFC394065027901B36E0FB01
:10B00D00A3E0FAA3E02408F9E43AFA7E00E92FF967
:10B01D00EE3AFA1216FEFF12C78B901B39E004F0C0
:10B02D0080CFE4901B39F0901B39E0FFC39406509C
:10B03D001774072FF582E43400F583E0FF12C78BF8
:08B04D00901B39E004F080DFE4
:01B0550022D8
:0B67B000901B05EBF0A3EAF0A3E9F05A
:1067BB00900001121717FFE4FCFDFE7810121AF37C
:1067CB00C004C005C006C007901B05E0FBA3E0FAA0
:1067DB00A3E0F91216FEFFE4FCFDFE7818121AF383
:1067EB00D003D002D001D000EF4BFFEE4AFEED49B3
:1067FB00FDEC48FCC004C005C006C007901B05E0BB
:10680B00FBA3E0FAA3E0F9900002121717FFE4FCD8
:10681B00FDFE7808121AF3D003D002D001D000EF9E
:10682B004BFFEE4AFEED49FDEC48FCC004C005C031
:10683B0006C007901B05E0FBA3E0FAA3E0F990006C
:10684B0003121717FFD003D002D001D000EB4FFF7C
:10685B00EAFEE9FDE8FC901B0B121BBC901C52E0FE
:10686B00FFE4FCFDFE7810121AF3C004C005C0064D
:10687B00C007901C51E0FFE4FCFDFE7818121AF3E0
:10688B00D003D002D001D000EF4BFFEE4AFEED4912
:10689B00FDEC48FCC004C005C006C007901C53E0CB
:1068AB00FFE4FCFDFE7808121AF3D003D002D001EE
:1068BB00D000EF4BFBEE4AFAED49F9EC48F8A3E0B8
:1068CB00FFEB4FFFEAFEE9FDE8FC901B0F121BBC30
:1068DB00901B0FE0FCA3E0FDA3E0FEA3E0FF901BE9
:1068EB000BE0F8A3E0F9A3E0FAA3E05FFFEA5EFE9A
:1068FB00E95DFDE85CFC901B13121BBC901B08E0D0
:10690B00FBA3E0FAA3E0F9900001121717FFE4FCD8
:10691B00FDFE7810121AF3C004C005C006C00712A2
:10692B0016FEFFE4FCFDFE7818121AF3D003D0021A
:10693B00D001D000EF4BFFEE4AFEED49FDEC48FCD9
:10694B00C004C005C006C007901B08E0FBA3E0FA1B
:10695B00A3E0F9900002121717FFE4FCFDFE780884
:10696B00121AF3D003D002D001D000EF4BFFEE4A46
:10697B00FEED49FDEC48FCC004C005C006C0079005
:10698B001B08E0FBA3E0FAA3E0F990000312171732
:10699B00FFD003D002D001D000EB4FFFEAFEE9FDA0
:1069AB00E8FC901B0B121BBC901B0FE0FCA3E0FD43
:1069BB00A3E0FEA3E0FF901B0BE0F8A3E0F9A3E03C
:1069CB00FAA3E05FFFEA5EFEE95DFDE85CFC901B6D
:1069DB0013E0F8A3E0F9A3E0FAA3E0FBC3121ACF8C
:1069EB007007901B1704F08005E4901B17F0901BA9
:0369FB0017E0FFA3
:0169FE002276
:109AA70090C00BE0FE90C00AE07C002400FFEC3E73
:109AB700FEEF7003EE64306002803BE4FFFE12C7E6
:109AC70025EF640E7003EE6463600280297F207EB9
:109AD7000012C725EF7003EE64036002801812C4FA
:109AE70055E4FDFC7F22FE12C8017F227E0012C7CB
:109AF70025EF540F60057EFF7F8B227F0A12C7FC7C
:109B07007F0212C7FC7D807C097F047E0112C80199
:109B1700E4FDFC7F067E0112C801900008E0FE907C
:109B27000007E0FDEEFCED7F587E0112C8019000B2
:109B37000AE0FE900009E0FDEEFCED7F5A7E01127F
:109B4700C80190000CE0FE90000BE0FDEEFCED7FFD
:109B57005C7E0112C801E4FDFC7F187E0112C8017A
:109B6700E4FDFC7F167E0112C8017DC07C007F12D8
:0A9B77007E0112C8017E007F01226A
:1058B400901B36EBF0A3EAF0A3E9F0A3ECF0A3ED20
:0158C400F0F3
:1058C500E4901B45F0A3F0A3F0900A6AE0FBA3E087
:1058D500FAA3E0F9C003C002C001900A6DE0FBA382
:1058E500E0FAA3E0F9D082D083D0E06B7008E965D7
:1058F500827003EA65837003025B59900A6DA3E029
:10590500FAA3E0AE02FF900A6AA3E0FAA3E0C39F00
:10591500FFEA9E901B41F0A3EFF0901B39E0FEA338
:10592500E0FF4E6029901B36E0FBA3E0FAA3E0F907
:1059350090000E121CC1E94A6014901B4DEBF0A3B8
:10594500EAF0A3E9F0EF5401901B47F0801A901B91
:1059550042E030E013E4FF12C78B901B42E004F0F5
:105965007006901B41E004F0901B41E0FEA3E0FFB0
:10597500901B3AE02FFF901B39E03EFE901B43F051
:10598500A3EFF0D394EEEE94054002806290C0043C
:1059950074C0F0A3E4F0901B43E0FEA3E090C006C2
:1059A500F0EEA3F07B017A1B79487D057C0012ADF2
:1059B5009E7B017A1B794812B9AAEF70187F387E51
:1059C5000112C725EE30E0E9901B43E0FFA3E0A3F9
:1059D500CFF0A3EFF0901B45E07002A3E070057EC9
:1059E500FF7F8F227F387E0112C725EF30E7057EC6
:1059F500FF7F8C22E4901B3BF0A3F0901B41E0FE5F
:105A0500A3E0FFC3901B3CE09F901B3BE09E5048EA
:105A1500900A6DE0FBA3E0FAA3E0F91216FE90C030
:105A250000F0900A6EE475F001121848900A6DE0D6
:105A3500FBA3E0FAA3E0F91216FE90C001F0900A6C
:105A45006EE475F001121848901B3CE02402F090BA
:105A55001B3BE03400F080A3901B47E0600E901BD9
:105A65003AE024FFF0901B39E034FFF0E4901B3B53
:105A7500F0A3F0901B39E0FEA3E0FFC3901B3CE0D0
:105A85009F901B3BE09E503E901B4DE0FBA3E475B1
:105A9500F00112185EA9F0FA1216FE90C000F090FF
:105AA5001B4DE0FBA3E475F00112185EA9F0FA1294
:105AB50016FE90C001F0901B3CE02402F0901B3BC9
:105AC500E03400F080AD901B47E06015901B4DE081
:105AD500FBA3E0FAA3E0F91216FE90C000F0A3E4E0
:105AE500F0901B3D121BC8000000007F407E0D7D1D
:105AF500037C00901B3DE0F8A3E0F9A3E0FAA3E0E6
:105B0500FBC3121ACF504D7F287E0112C725901B6B
:105B15003BEEF0A3EFF0EE5486FEEF54C04E600C62
:105B2500901B4574FFF0A3748CF08028901B3BE01C
:105B350020E021901B3DE0FCA3E0FDA3E0FEA3E0F7
:105B45002401FFE43EFEE43DFDE43CFC901B3D12D8
:0C5B55001BBC8097901B45E0FEA3E0FF06
:015B61002221
:106E5100E4901B28F0A3F07F247E0112C725EE20C9
:106E6100E03B7B017A1B79237D057C0012AD9E7B83
:106E7100017A1B792312B9AAEF70137F247E0112C4
:106E8100C725EE30E0E9901B28E4F0A304F0901B45
:106E910028E07002A3E070057EFF7F872290C00189
:106EA100E0FE90C000E07C002400FFEC3E901B1F40
:106EB100F0A3EFF0901B1FE0FEA3E0FF12C91F90AB
:106EC100C001E0FE90C000E07C002400FFEC3E9099
:106ED1001B21F0A3EFF0901B21E0FCA3E0FD540186
:106EE100901B2AF0901278E0FEA3E0FFC374FE9F8E
:106EF100FF74039EFED3ED9FEC9E4003027024902D
:106F01001B21E0FEA3E0FF901B28EEF0A3EFF0EEC3
:106F1100FF12BE83901B21A3E0FF12BE83901B2AA8
:106F2100E0600E901B22E024FFF0901B21E034FF73
:106F3100F0E4FFFED3901B22E09F901B21E09E50C6
:106F410003026FD390C000E0FD900A70E0FBA3E064
:106F5100FAA3E0F9ED121777900A70A3E475F00136
:106F6100121848FAD3901277E5F09582EA9583409A
:106F71000E900A707401F0A3740EF0A37478F0906F
:106F8100C001E0FD900A70E0FBA3E0FAA3E0F9ED97
:106F9100121777900A70A3E475F001121848FAD31A
:106FA100901277E5F09582EA9583400E900A70740D
:106FB10001F0A3740EF0A37478F0901279E024022A
:106FC100F0901278E03400F074022FFFE43EFE02EC
:106FD1006F35901B2AE0606090C000E0FF900A705E
:106FE100E0FBA3E0FAA3E0F9EF121777900A70A390
:106FF100E475F001121848FAD3901277E5F0958202
:10700100EA9583400E900A707401F0A3740EF0A308
:107011007478F0901279E004F07006901278E00430
:10702100F080157D407C007F027E0112C801901B1B
:107031002874FFF0A3748DF0901B28E0FEA3E0FFFD
:01704100222C
:10C72500EF90C00AF0EEA3F090C00DE0FE90C00CB3
:0AC73500E07C002400FFEC3EFE2231
:05C7FC00E4FDFC7E01DC
:0FC80100EF90C00AF0EEA3F0EDA3F0ECA3F0224D
:10C455007D407C007F147E0112C8017F021E12C739
:10C465003F7F017E0012C73F7F147E0112C7257FE3
:0BC47500367E0112C725EF30E7E722FA
:01C91F0022F5
:10C810007F347E0112C725EF30E7057E007F0122BD
:03C82000E4FEFF34
:01C8230022F2
:106C4D00901AEAEFF0A3ECF0A3EDF0A3EAF0A3EBBA
:016C5D00F046
:106C5E00901AF1E0FBA3E0FAA3E0F99000011217FD
:106C6E0017FD1216FEFEEDFFE4FCFD901AF7121B47
:106C7E00BC901AF7E0F8A3E0F9A3E0FAA3E0FBC09A
:106C8E0000C001C002C003901AF1E0FBA3E0FAA31A
:106C9E00E0F9900002121717FE900003121717FD6D
:106CAE00EDFFE4FCFDD003D002D001D000EB2FFFAE
:106CBE00EA3EFEED39FDEC38FC901AF7121BBC9043
:106CCE001AF7E0F8A3E0F9A3E0FAA3E0FBC000C0D6
:106CDE0001C002C003901AF4E0FBA3E0FAA3E0F9AE
:106CEE00900001121717FD1216FEFEEDFFE4FCFDDB
:106CFE00D003D002D001D000EB2FFFEA3EFEED39DB
:106D0E00FDEC38FC901AF7121BBC901AF7E0F8A3B2
:106D1E00E0F9A3E0FAA3E0FBC000C001C002C0038B
:106D2E00901AF4E0FBA3E0FAA3E0F9900002121728
:106D3E0017FE900003121717FDEDFFE4FCFDD003C4
:106D4E00D002D001D000EB2FFFEA3EFEED39FDEC74
:106D5E0038FC901AF7121BBC901AF7E0F8A3E0F972
:106D6E00A3E0FAA3E0FB901AEAE0FFE4FCFDFEEBE1
:106D7E002FFFEE3AFEED39FDEC38FC901AF7121BA0
:106D8E00BC901AF7E0F8A3E0F9A3E0FAA3E0FB90B9
:106D9E001AEBE0FEA3E0FFE4FCFDEB2FFFEA3EFE64
:106DAE00ED39FDEC38FC901AF7121BBC901AF7E087
:106DBE00F8A3E0F9A3E0FAA3E0FB901AEDE0FEA33E
:106DCE00E0FFE4FCFDEB2FFFEA3EFEED39FDEC3873
:106DDE00FC901AF7121BBC901AF7E0F8A3E0F9A387
:106DEE00E0FAA3E0FB901AEFE0FEA3E0FFE4FCFD67
:106DFE00EB2FFFEA3EFEED39FDEC38FC901AF71250
:106E0E001BBC901AEAE0B4112B901AF7E0F8A3E03D
:106E1E00F9A3E0FAA3E0FB901AEBE0FEA3E0FFE497
:106E2E00FCFDEB2FFFEA3EFEED39FDEC38FC901A2F
:106E3E00F7121BBC901AF7E0FCA3E0FDA3E0FEA343
:026E4E00E0FF63
:016E5000221F
:10898E00901AEA121BBC901AEEEBF0A3EAF0A3E9E0
:01899E00F0E8
:10899F00A3E07002A3E07003028A8D901AF1E0FC4D
:1089AF00A3E0FD5401901AF5F0ECC313FFED139003
:1089BF001AF1CFF0A3EFF0901AF174FFF5F012183F
:1089CF005E45F06068901AEEE0FBA3E475F00112CB
:1089DF00185EA9F0FA1216FE901AF3F0A3E4F090C5
:1089EF001AEEE0FBA3E475F00112185EA9F0FA127B
:1089FF0016FEFF901AF4E02FF0901AF3E03400F017
:108A0F00901AEAE0F8A3E0F9A3E0FAA3E0FB901ACA
:108A1F00F3E0FEA3E0FFE4FCFDEB2FFFEA3EFEEDEB
:108A2F0039FDEC38FC901AEA121BBC808A901AF5BB
:108A3F00E0604B901AEEE0FBA3E0FAA3E0F9121608
:108A4F00FE7F00FE901AF3F0A3EFF0901AF3EEF012
:108A5F00A3EFF0901AEAE0F8A3E0F9A3E0FAA3E09D
:108A6F00FB901AF3E0FEA3E0FFE4FCFDEB2FFFEA1F
:108A7F003EFEED39FDEC38FC901AEA121BBC901A41
:0C8A8F00EAE0FCA3E0FDA3E0FEA3E0FF92
:018A9B0022B8
:10B58D008052901B48E0FCA3E0FDA3E0FEA3E0FF8A
:10B59D007810121AE0EC4D4E4F6041901B48A3A35A
:10B5AD00E0FEA3E0FFE4FDFCC004C005C006C0073B
:10B5BD00901B48E0FCA3E0FDA3A3E07810121AE075
:10B5CD00D003D002D001D000EF2BFFEE3AFEED39C3
:10B5DD00FDEC38FC901B48121BBC80A6901B48E06C
:10B5ED00FCA3E0FDA3E0FEA3E0FF121A9EE4FDFC28
:01B5FD00222B
:10AD9E00901B50EBF0A3EAF0A3E9F0A3ECF0A3EDC7
:10ADAE00F012C8DC901B50E0FBA3E0FAA3E0F9EE32
:10ADBE008FF012195C901B50E0FBA3E0FAA3E0F9B0
:10ADCE00121874FF901B54E02FFF901B53E035F0C8
:10ADDE009000028FF012197B90000212189FFFAEA6
:10ADEE00F0121874FDACF0D39FEC9E901B50E0FB5C
:10ADFE00A3E0FAA3E0F95006900004E48020C3E437
:10AE0E009DFFE49CFEC3901B54E09FFF901B53E0FC
:10AE1E009E9000028FF012197B900004740112179D
:02AE2E00892277
:0BB9AA00901B50EBF0A3EAF0A3E9F0C3
:10B9B50012C8DC901B50E0FBA3E0FAA3E0F990006D
:10B9C50004121717601E121874FDC3EF9DEE95F053
:10B9D500503090000212189FFDD3EF9DEE95F04078
:10B9E500217F012290000212189FFDD3EF9DEE9555
:10B9F500F0500C121874FDC3EF9DEE95F050037FC7
:04BA050001227F009B
:01BA0900221A
:0CC8DC00C2AF900A76E0FEA3E0FFD2AFEE
:01C8E800222D
:10C73F007B017A1A79A2AD07AC0612AD9E7B017A06
:09C74F001A79A212B9AAEF60F4F4
:01C7580022BE
:10C78B00900A6AE0FBA3E0FAA3E0F9EF12177790A7
:09C79B000A6BE475F00102184874
:10BC6900900A73E0FBA3E0FAA3E0F91216FEFFC203
:10BC7900AF901279E024FFF0901278E034FFF0D20F
:10BC8900AF900A74E475F001121848900A73A3E0A2
:10BC9900FAA3E0D39012779582EA9583400E900A31
:0EBCA900737401F0A3740EF0A37478F07E00A3
:01BCB700226A
:10947400901B48EBF0A3EAF0A3E9F0901B48A3E0AB
:10948400FAA3E04A700302955E901B48E0FBA3A395
:10949400E0F9900020743C1217899000267402753C
:1094A400F00012197B12C8DCE4FCFDC004C005C046
:1094B40006C007901B48E0FBA3E0FAA3E0F9900084
:1094C4001C121717FFE4FE7810121AF3D003D0020F
:1094D400D001D000EF2BFFEE3AFEED39FDEC38FC65
:1094E400EF2401FFE43EFEE43DFDE43CFC901B4818
:1094F400E0FBA3E0FAA3E0F9900034121B509000C3
:109504001FE4121789900022E4121789900021E4C5
:10951400121789900024E4F5F012197B900023E4DB
:10952400121789900028121BF90000000090002CEB
:10953400121BF900000000900030121BF90000001B
:1095440000900038E4F5F012197B90003AE4F5F04D
:0B95540012197B90003CE412178922E2
:0E8DBE00901A71EFF0A3EBF0A3EAF0A3E9F036
:108DCC004A6023901A72E0FBA3E0FAA3E0F990004A
:108DDC001C12171775F03DA42499F582E5F0341296
:108DEC00F583E020E0037F8622901A71E014600E78
:108DFC001460432402705590001F7401803390005E
:108E0C001F74021217897D0212A2B4D3EF648094EE
:108E1C0080400F7B017A1A79757DA07C8C12AD9EF7
:108E2C00802D901A72E0FBA3E0FAA3E0F990001FEA
:108E3C00E41217898019901A72E0FBA3E0FAA3E000
:108E4C00F990001F74011217897F01227F00229074
:108E5C001A72E0FBA3E0FAA3E0F990001F121717B7
:108E6C00FF64046036EF6033901A71E0B4011C7B30
:108E7C00017A1A797512B9AAEF6010901A72E0FB98
:108E8C00A3E0FAA3E0F912B8E98010901A72E0FBA3
:108E9C00A3E0FAA3E0F912BA0A80B4901A72E0FBCC
:0D8EAC00A3E0FAA3E0F990001F121717FFD2
:018EB9002296
:0B22C700901AB8EBF0A3EAF0A3E9F0D6
:1022D200901AD27401F0A3741AF0A374BFF0901A8A
:1022E200B8E0F9A3E0FAA3E0901AD5C9F0A3EAF0A6
:1022F200A3E9F07B017A1A79C112366AEF700812EB
:1023020096477EFF7FFD22901AB8E0FBA3E0FAA376
:10231200E0F9121C52901AC5EBF0A3EAF0A3E9F01F
:1023220090001F121717B40A00400302260C9023D4
:1023320037F82828730223550223AA0224AC022468
:102342001B0226280225410225B202260C02260C77
:102352000225F2129647901AC5E0FBA3E0FAA3E029
:10236200F990002112171720E23B12C231901AC5D0
:10237200E0FBA3E0FAA3E0F990001D121717B440A6
:102382002490001C121717FF12A6257B007A0079F1
:1023920000C003C002C001901AB8E0FBA3E0FAA398
:1023A200E0F9121C72022607129647901AC5E0FB4A
:1023B200A3E0FAA3E0F9900021121717FF30E2031D
:1023C20002268530E41212C231901ACEEFF0D364A5
:1023D2008094804041022967901AC5E0FBA3E0FA8D
:1023E200A3E0F990002C121B06900028121B507DCE
:1023F2001212A2B4901ACEEFF0D3648094804016E9
:10240200901AC5E0FBA3E0FAA3E0F990001F740361
:10241200121789022685022AA6901AC5E0FBA3E0BC
:10242200FAA3E0F9900021121717FF30E4075406CF
:102432007003022628129647901AC5E0FBA3E0FA21
:10244200A3E0F990002112171730E2181294749049
:102452001AC5E0FBA3E0FAA3E0F990001F74011291
:1024620017898043901AC5E0FBA3E0FAA3E0F99034
:10247200002112171730E12C900028121B06EF24BE
:10248200FFFFEE34FFFEED34FFFDEC34FFFC900065
:102492002C121B8CC3121ACF700A901AC57D12120D
:1024A200A2AC800312C226022685129647901AC554
:1024B200E0FBA3E0FAA3E0F990002112171730E243
:1024C200030226AA901AC5E0FBA3E0FAA3E0F99062
:1024D2000021121717FF30E40320E12512C23190C8
:1024E2001ACEEFF0D3648094804013901AC5E0FBBB
:1024F200A3E0FAA3E0F9900020743C0225AC022A82
:10250200A6901AC5E0FBA3E0FAA3E0F990001F74BD
:102512000412178912BB6E129B81901ACEEFF0D370
:10252200648094804016901AC5E0FBA3E0FAA3E011
:10253200F9900020743C121789022986022AA612F9
:102542009647901AC5E0FBA3E0FAA3E0F9900022B7
:1025520012171730E0447D1112C382D3EF648094C6
:10256200804037901AC5E0FBA3E0FAA3E02438F9D3
:10257200E43AFA7D327C0012AD9E901AC5E0FBA3CC
:10258200E0FAA3E0F912BB6E129B81901ACEEFF033
:10259200D3648094805003022AA9901AC5E0FBA359
:1025A200E0FAA3E0F990001F740612178902275C73
:1025B200901AC5E0FBA3E0FAA3E0F99000221217FB
:1025C2001730E00312BB6E129647129B81901ACE0F
:1025D200EFF0D3648094804014901AC5E0FBA3E02E
:1025E200FAA3E0F990001FE41217898018022AA6C4
:1025F200901AC5E0FBA3E0FAA3E0F990001FE412F1
:1026020017891296477EFF7FFA22901AC5E0FBA334
:10261200E0FAA3E0F990001F121717D3940A4006BC
:1026220012B8E9022AA1901AC5E0FBA3E0FAA3E0DE
:10263200F9900028121B06901ACA121BBC90002C9B
:10264200121B06901ACAE0F8A3E0F9A3E0FAA3E08D
:10265200FBC3121ACF602F12A06C129647901AC5B4
:10266200E0FBA3E0FAA3E0F990002112171720E2A1
:1026720012129B8C901ACEEFF0D364809480500398
:10268200022AA902275C901AC5E0FBA3E0FAA3E0A4
:10269200F990002112171730E235129647901AC5A9
:1026A200E0FBA3E0FAA3E0F990001C121717FF1257
:1026B200A6257B007A007900C003C002C001901AEF
:1026C200B8E0FBA3E0FAA3E0F9121C72022AA1907F
:1026D2001AC5E0FBA3E0FAA3E0F990002112171754
:1026E20030E11712964712C226901ACEEFF0D36449
:1026F20080948040028063022AA6901AC5E0FBA360
:10270200E0FAA3E0F990002112171720E4061296CE
:1027120047022A6D901AC5E0FBA3E0FAA3E0F99004
:10272200001F12171764046008900020743C1217EF
:102732008990001F7404121789D3901BC6E094007D
:10274200901BC5E094024018129647129B81901A82
:10275200CEEFF0D3648094804003022A6D022AA651
:10276200E4901AC8F0A3F0901AC1E0F8A3E0F9A32C
:10277200E0FAA3E0FBC000C001C002C003A3E0FB7B
:10278200A3E0FAA3E0F9900023121717FF901BC6EB
:10279200E02FFD901BC5E03400FC121874FBAAF078
:1027A200C002C003901AC5E0FBA3E0FA9000021237
:1027B200189FFF901AEFE5F0F0A3EFF0A37401F079
:1027C200A3741CF0A37447F0901AC5A3A3E02404D9
:1027D200F9E43AFA901AF4EBF0A3EAF0A3E9F0D0A4
:1027E20003D0027F06126C4DD003D002D001D0007C
:1027F200EB2FFFEA3EFEE93DFDE83CFC901AC112D8
:102802001BBC901BC5E0FEA3E0FF901ABDEEF0A337
:10281200EFF04E70030228E4E4901ABCF0A3E0FE4D
:10282200A3E0FF901AC5E0FBA3E0FAA3E0F912C807
:10283200FF12BC69901ABBEFF0A3E0901ABB700FB5
:10284200E0901AC8F0A3E4F0901ABC04F0803FE0D4
:10285200FF901AC9E02FF0901AC8E03400F0901AE5
:10286200C1E0F8A3E0F9A3E0FAA3E0FB901AC8E004
:10287200FEA3E0FFE4FCFDEB2FFFEA3EFEED39FD97
:10288200EC38FC901AC1121BBCE4901ABCF0901AEE
:10289200BBE0FF901AC5E0FBA3E0FAA3E0F912A7A0
:1028A20073901BC574FFF5F012184845F0708290C2
:1028B2001ABCE06041901AC1E0F8A3E0F9A3E0FA83
:1028C200A3E0FB901AC8E0FEA3E0FFE4FCFDEB2FBF
:1028D200FFEA3EFEED39FDEC38FC901AC1121BBC3A
:1028E2008014901AC5E0FBA3E0FAA3E0F990001966
:1028F200E4F5F012197B901AC1E0FCA3E0FDA3E01D
:10290200FEA3E0FF12B58D901AC1121BBC901ABF34
:10291200E0FEA3E0FFE4FCFDA3E0F8A3E0F9A3E0FE
:10292200FAA3E0FBC3121ACF60081296477EFF7F1C
:10293200FC2212A06C901ABDE07002A3E070281273
:102942009647901AC5E0FBA3E0FAA3E0F990002CA9
:10295200121B06900028121B5090002212171730EB
:10296200E003022A07801D901AC5E0FBA3E0FAA348
:10297200E0F912C912901ACEEFF0129647901ACED1
:10298200E0B4A204E4FEFF22901AC5E0FBA3E0FA41
:10299200A3E0F990002C121B8C901ABDE0FEA3E07C
:1029A200FFEF2BFFEE3AFEE439FDE438FC901AC546
:1029B200E0FBA3E0FAA3E0F9900028121B5090007C
:1029C2002212171720E03E901AC5E0FBA3E0FAA3FB
:1029D200E0F990001D121717FF30E00A9000111263
:1029E200189F45F06004EF20E012129B8C901ACEE3
:1029F200EFF0D3648094805003022AA9901ABDE0BC
:102A0200FEA3E0FF22901AC5E0FBA3E0FAA3E0F9DF
:102A1200900028121B06EF2401FFE43EFEE43DFD78
:102A2200E43CFC900028121B50129B8C901ACEEFB3
:102A3200F0D364809480406C901AC5E0FBA3E0FA66
:102A4200A3E0F990001F7409121789E92438F9E408
:102A52003AFA7D327C0012AD9E901AC512C378906C
:102A62001ACEEFF0D36480948040057EFF7F8922E6
:102A7200901AC5E0FBA3E0FAA3E0F990001C12173C
:102A820017FF12A6257B007A007900C003C002C09E
:102A920001901AB8E0FBA3E0FAA3E0F9121C727EDF
:0D2AA200FF7FFF22901ACEE0FF3395E0FE8B
:012AAF002204
:0BA06C00901AC5E0FBA3E0FAA3E0F9A6
:0BA07700901ACFEBF0A3EAF0A3E9F091
:10A0820090002412189FFF901AD2E5F0F0A3EFF08F
:10A09200900034121B06901AD4121BBC901AD2E004
:10A0A2007002A3E0700302A12D901ACFE0FBA3E09F
:10A0B200FAA3E0F9900030121B8CC000C001C0026C
:10A0C200901AD2E0FEA3E0FFE4FCFDA3E0F8A3E0D7
:10A0D200F9A3E0FAA3E02FFFEA3EFEED39FDEC38EA
:10A0E200FCD002D001D000C3121ACF703E901AD217
:10A0F200E0FEA3E0FF901ACFE0FBA3E0FAA3E0F9B1
:10A1020012AAA0901ACFE0FBA3E0FAA3E0F9900014
:10A1120024E4F5F012197B900020743C1217899008
:0BA122000030121B06900034121B508E
:01A12D00220F
:0B704200901A80EBF0A3EAF0A3E9F045
:10704D004A70057EFF7F8522901A80E0FBA3E0FA4F
:10705D00A3E0F990001F121717FDC3940250057E8F
:10706D00FF7FFA229000201217176006EDD3940AC5
:10707D00400812B8E97EFF7FFF22901A80E0FBA343
:10708D00E0FAA3E0F990001F12171764027027E9C8
:10709D002438F9E43AFA12B9AAEF6017901A807DF4
:1070AD000212A2AC901A85EFF0D364809480500345
:1070BD000271F5027141901A80E0FBA3E0FAA3E0A2
:1070CD00F990002412189F45F06029E92438F9E45D
:1070DD003AFA12B9AAEF7003FEFF22901A80E0FB74
:1070ED00A3E0FAA3E02438F9E43AFA7D327C0012E9
:1070FD00AD9E8044901A80E0FBA3E0FAA3E0F990E6
:10710D00001F121717C39405402EE92438F9E43AED
:10711D00FA12B9AAEF6021901A80E0FBA3E0FAA35E
:10712D00E02438F9E43AFA7D327C0012AD9E901AD3
:10713D008012C378E4FEFF22901A80E0FBA3E0FAF0
:10714D00A3E0F912C34A901A83EEF0A3EFF0901A60
:10715D0080E0FBA3E0FAA3E0F9900024EE8FF0129B
:10716D00197BEF4E7003FEFF2290002612189FFF31
:10717D00AEF0D3901A84E09F901A83E09E4005EE06
:10718D00F0A3EFF0D3901A84E09400901A83E0946A
:10719D000240067402F0A3E4F090002412189FFF41
:1071AD00901A83E065F07003A3E06F60057EFF7FAA
:1071BD00FE229000217418121789123B84901A85B3
:1071CD00EFF0640160028020901A80E0FBA3E0FAEA
:1071DD00A3E0F9A3E0FCA3E0FD12C09B901A85EF9C
:1071ED00F0D3648094805007E0FF3395E0FE229049
:1071FD001A80E0FBA3E0FAA3E02438F9E43AFA7D23
:10720D00327C0012AD9E901A80E0FBA3E0FAA3E061
:0A721D00F990002412189FFFAEF054
:017227002244
:10B8E900901B3AEBF0A3EAF0A3E9F0901B3AA3E02E
:10B8F900FAA3E04A604A901B3AE0FBA3A3E0F9905F
:10B90900001FE41217897B007A007900C003C00286
:10B91900C001901B3AE0FBA3E0FAA3E0F990000E06
:10B92900121CF1901B3AE0FBA3E0FAA3E0F99000A6
:10B9390011E4F5F012197B900024E4F5F012197B5B
:01B9490022DB
:10AA0000901CB5EBF0A3EAF0A3E9F0901CB5A3E02D
:10AA1000FAA3E04A700302AA9F901CB5E0FBA3A32F
:10AA2000E0F9900024E4F5F012197B7B007A0079BC
:10AA300000C003C002C001901CB5E0FBA3E0FAA374
:10AA4000E0F990000E121CF1901CB5E0FBA3E0FAB7
:10AA5000A3E0F9900011E4F5F012197B90001F12A9
:10AA60001717FF64036009EF64046004EFB4072F55
:10AA7000901CB5E0FBA3E0FAA3E02438F9E43AFA2D
:10AA80007D327C0012AD9E901CB5E0FBA3E0FAA3E2
:10AA9000E0F990001F74051217897D1112C38222FC
:10C01F00901CB8EBF0A3EAF0A3E9F0901CB8E0FB9A
:10C02F00A3E0FAA3E0F94A602512AA00901CB8E039
:10C03F00FBA3E0FAA3E0F990001F121717FFD394A8
:0FC04F0000400BEFD3940A500512BA0A80DE228C
:0BBA0A00901A7AEBF0A3EAF0A3E9F039
:10BA1500E4901A7EF0A3F012C31C901A7DEFF0306B
:10BA2500E0137B017A1A797A1222C7901A7EEEF01A
:10BA3500A3EFF08010901A7DE030E1097B017A1ABE
:10BA4500797A024B6C901A7EE0F47004A3E0648965
:10BA55006011901A7AE0FBA3E0FAA3E0F94A6003CB
:03BA65001270421A
:01BA680022BB
:0B366A00901ACFEBF0A3EAF0A3E9F008
:10367500E4901AEDF012BC69EF901ADAF0A3E4F0C9
:1036850012BC69901ADBE02FF0901ADAE03EF012D6
:10369500BC69EF901AD8F0A3E4F012BC69901AD96E
:1036A500E02FF0901AD8E03EF012BC69901AE1EFD5
:1036B500F012BC69901AE2EFF012BC69901AE3EFC0
:1036C500F012BC69901AE4EFF012BC69901AE5EFAC
:1036D500F012BC69901AE6EFF012BC69901AE7EF98
:1036E500F012BC69901AE8EFF0901AE1E0FEA3E051
:1036F500FFE4FCFD901AEE121BBC901AEEE0F8A355
:10370500E0F9A3E0FAA3E0FB901AE3E0FEA3E0FFF3
:10371500E4FCFDEB2FFFEA3EFEED39FDEC38FC90B5
:103725001AEE121BBC901AEEE0F8A3E0F9A3E0FA3A
:10373500A3E0FB901AE5E0FEA3E0FFE4FCFDEB2F20
:10374500FFEA3EFEED39FDEC38FC901AEE121BBC8B
:10375500901AEEE0F8A3E0F9A3E0FAA3E0FB901AD3
:10376500E7E0FEA3E0FFE4FCFDEB2FFFEA3EFEED04
:1037750039FDEC38FC901AEE121BBC12BC69901A8C
:10378500E0EFF012BC69901ADFEFF0901AEEE0F866
:10379500A3E0F9A3E0FAA3E0FB901AE0E0FE901A9B
:1037A500DFE0FDEDFFE4FCFDEB2FFFEA3EFEED392A
:1037B500FDEC38FC901AEE121BBC901AE0E054F0B8
:1037C500F0E01313543FFFF0C3901BC6E09F901B1E
:1037D500C5E094004008901AE0E094125003023AC4
:1037E50005901AE0E0FFC3901BC6E09FF0901BC553
:1037F500E09400F012BC69EF901ADCF0A3E4F0123B
:10380500BC69901ADDE02FF0901ADCE03EF0901ACA
:10381500EEE0F8A3E0F9A3E0FAA3E0FB901ADCE000
:10382500FEA3E0FFE4FCFDEB2FFFEA3EFEED39FDD4
:10383500EC38FC901AEE121BBC12BC69EFF9901A19
:10384500D2E0FBA3E0FAA3E0C975F00012195C12FF
:10385500BC69901AD2E0FBA3E0FAA3E0F9EE8FF081
:103865001218D7901AE0E0C39412901ADEF0901A5D
:10387500EEE0F8A3E0F9A3E0FAA3E0FBC000C00185
:10388500C002C00312BC69EFFEE4FCFDD003D00208
:10389500D001D0002BFFEA3EFEED39FDEC38FC905F
:1038A5001AEE121BBC901AEEE0F8A3E0F9A3E0FAB9
:1038B500A3E0FBC000C001C002C00312BC69E4FC68
:1038C500FDD003D002D001D000EB2FFFEA3EFEED84
:1038D50039FDEC38FC901AEE121BBC901ADEE02480
:1038E500FEF0E07089901AEEE0FCA3E0FDA3E0FE97
:1038F500A3E0FF901ACFE0FBA3E0FAA3E0F9121BC7
:1039050036901AD8E0FEA3E0FFA3E0FCA3E0FD7B20
:10391500017A1C7923901B4F7406F01282AB901A22
:10392500E9EBF0A3EAF0A3E9F04A6003023AAD90AF
:103935001AD8E0FEA3E0FF7B017A1C7923901B4F88
:103945007406F0E4FDFC1282AB901AE9EBF0A3EAF1
:10395500F0A3E9F04A7025901AD8E0FEA3E0FF7BBA
:10396500017A1B79CE901B4F7406F0E4FDFC1282A0
:10397500AB901AE9EBF0A3EAF0A3E9F0901AE9E0BD
:10398500FBA3E0FAA3E0F94A6020901ADFE030E1FA
:1039950019901ADAE0FFA3E0900002CF8FF0121918
:1039A5007B901AED7401F0023AAD901ADFE030E237
:1039B50002804D901AD8E0FEA3E0FF12C3D3901AFF
:1039C500ECEFF0901AD8E0FCA3E0FDA3E0FFA3E044
:1039D500901B3BCFF0A3EFF0A37406F0901AECE038
:1039E500901B3EF0A3E4F0A3F0A3F0A3F0A3F07BBB
:1039F500017A1C7923125292C3EF64809480501D82
:103A05007B007A007900C003C002C001901AD5E09E
:103A1500FBA3E0FAA3E0F9121C727F0022EF3395B5
:103A2500E0FE7C007D3D1217AB747B2FF974123ECE
:103A3500FA7B01901AE9EBF0A3EAF0A3E9F0900014
:103A45001FE4121789901BC5E0FEA3E0FF4E601B23
:103A5500E4FD901AE1E0F8A3E0F9A3E0FAA3E02F72
:103A6500FFEA3EFEED39FDEC388018901AE1E0FCE6
:103A7500A3E0FDA3E0FEA3E02401FFE43EFEE43D58
:103A8500FDE43CFC901AE9E0FBA3E0FAA3E0F99021
:103A95000028121B50901AE9E0FBA3E0FAA3E0F915
:103AA50090001D7440121789901AE9E0FBA3E0FA13
:103AB500A3E0F9C003C002C001901AD5E0FBA3E062
:103AC500FAA3E0F9121C72901ADFE0FF901AE9E000
:103AD500FBA3E0FAA3E0F9900022EF12178990000A
:103AE50021EF121789901ADCE0FFA3E0900026CFA2
:103AF5008FF012197B901AE0E0900023121789903D
:103B05001AE1E0FCA3E0FDA3E0FEA3E0FF90002C9A
:103B1500121B50901AE5E0FCA3E0FDA3E0FEA3E034
:103B2500FF900030121B50901AEDE0B40113901A6B
:103B3500E9E0FBA3E0FAA3E0F990001F7401121776
:103B450089901AE9E0FBA3E0FAA3E0F990000412DA
:103B550017177028901C23E0900004121789901CF9
:103B650024E0900005121789901C25E090000612AC
:0E3B75001789901C26E09000071217897F0127
:013B8300221F
:0B3B8400901ADCEBF0A3EAF0A3E9F0DC
:103B8F00900021121717FF901AE9F09000241218D5
:103B9F009FFD901AE7E5F0F0A3EDF0EF30E13DE087
:103BAF002418F0901AE7E03400F0901AE67460F0F1
:103BBF00901AE0121BC800000204901AE0E0FCA368
:103BCF00E0FDA3E0FEA3E02400FFEE3402FEE43D9F
:103BDF00FDE43CFC901AE0121BBC801E901AE8E03A
:103BEF002414F0901AE7E03400F0901AE67450F0C5
:103BFF00901AE0121BC800000000901AE0E0F8A332
:103C0F00E0F9A3E0FAA3E0FBC000C001C002C003CB
:103C1F00901AE7E0FCA3E0FD901ADCE0FBA3E0FACA
:103C2F00A3E0F9121874FBAAF0C002C003901ADCCB
:103C3F00E0FBA3E0FA90000212189FFF901AEFE545
:103C4F00F0F0A3EFF0A37401F0A3741CF0A374477A
:103C5F00F0901ADCA3A3E02404F9E43AFA901AF4E2
:103C6F00EBF0A3EAF0A3E9F0D003D0027F06126CC9
:103C7F004DD003D002D001D000EB2FFFEA3EFEE97A
:103C8F003DFDE83CFC901AE0121BBC901AE0E0F8F6
:103C9F00A3E0F9A3E0FAA3E0FBC000C001C002C09B
:103CAF0003901ADCE0FBA3E0FAA3E0F990003412D2
:103CBF00189FFFE4FCFDD003D002D001D000EB2F02
:103CCF00FFEA35F0FEED39FDEC38FC901AE0121BDF
:103CDF00BC901AE0E0F8A3E0F9A3E0FAA3E0FBC080
:103CEF0000C001C002C003901ADCE0FBA3E0FAA3FE
:103CFF00E0F990003612189FFFE4FCFDD003D002CC
:103D0F00D001D000EB2FFFEA35F0FEED39FDEC3896
:103D1F00FC901AE0121BBC901AE0E0F8A3E0F9A3A4
:103D2F00E0FAA3E0FBC000C001C002C003901ADCA0
:103D3F00E0FBA3E0FAA3E0F990002812189FFFE43C
:103D4F00FCFDD003D002D001D000EB2FFFEA35F0FD
:103D5F00FEED39FDEC38FC901AE0121BBC901AE016
:103D6F00E0F8A3E0F9A3E0FAA3E0FBC000C001C0B4
:103D7F0002C003901ADCE0FBA3E0FAA3E0F9900085
:103D8F002A12189FFFE4FCFDD003D002D001D0000F
:103D9F00EB2FFFEA35F0FEED39FDEC38FC901AE021
:103DAF00121BBC901AE0E0F8A3E0F9A3E0FAA3E03D
:103DBF00FB901AE6E0FE901AE9E0FDEDFFE4FCFD52
:103DCF00EB2FFFEA3EFEED39FDEC38FC901AE012C6
:103DDF001BBC901AE0E0FCA3E0FDA3E0FEA3E024EF
:103DEF0000FFEE3402FEE43DFDE43CFC901AE012CD
:103DFF001BBC901AE0E0FCA3E0FDA3E0FEA3E0FFF4
:103E0F00901ADCE0FBA3E0FAA3E0F990000E121C7D
:103E1F00C1C003C002C001901ADCE0FBA3E0FAA30B
:103E2F00E0F990002412189FFB901AF1E5F0F0A32F
:103E3F00EBF0D001D002D00312898E901AE0121B42
:103E4F00BC901AE0E0FCA3E0FDA3E0FEA3E0FF12AC
:103E5F00B58D901AE0121BBC901AE0A3A3E0FFA34C
:103E6F00E0A3CFF0A3EFF0901ADCE0FBA3E0FAA3FE
:103E7F00E0F990001B121717FD901AE7E0FFA3E07F
:103E8F00901AEECFF0A3EFF0901ADCA3A3E0126923
:103E9F00FFEF6401600122901ADCE0FBA3E0FAA3BC
:103EAF00E0F9121874E5F0FF12C78B901ADCE0FBF3
:103EBF00A3E0FAA3E0F9121874FF12C78B901ADC73
:103ECF00E0FBA3E0FAA3E0F990000212189FE5F0DF
:103EDF00FF12C78B901ADCE0FBA3E0FAA3E0F99086
:103EEF00000212189FFF12C78BE4901ADFF0901A8E
:103EFF00DFE0FFC364809484502A901ADCE0FBA3B8
:103F0F00E0FAA3E02434F9E43AFAEF3395E0FEE95E
:103F1F002FF9EA3EFA1216FEFF12C78B901ADFE056
:103F2F0004F080CAE4901ADFF0901ADFE0FFC36458
:103F3F00809484502A901ADCE0FBA3E0FAA3E024DB
:103F4F0028F9E43AFAEF3395E0FEE92FF9EA3EFA61
:103F5F001216FEFF12C78B901ADFE004F080CA9092
:103F6F001AE6E0FF12C78B901AE9E0FF12C78B7FAA
:103F7F000212C78BE4FF12C78B901AE4E0FF12C73F
:103F8F008B901AE4A3E0FF12C78BE4FF12C78BE4F8
:103F9F00FF12C78B901AE9E030E1147F0212C78B32
:103FAF007F0412C78B7F0212C78BE4FF12C78B7F70
:013FBF000100
:013FC00022DE
:04BB6E007F017E00D5
:10BB7200901ACFEEF0A3EFF0A3EBF0A3EAF0A3E963
:10BB8200F0901AD1E0FBA3E0FAA3E0F990003012A2
:10BB92001B06900034121B5090002C121B8C901A22
:10BBA200CFE0FEA3E0FFEF2BFFEE3AFEE439FDE427
:10BBB20038FCA3E0FBA3E0FAA3E0F9900028021B03
:01BBC2005032
:10BA6900901AD9EBF0A3EAF0A3E9F0901AD9E0FB18
:10BA7900A3E0FAA3E0F9900021ED1217897B007A7F
:10BA8900007900C003C002C001901AD9E0FBA3E00D
:10BA9900FAA3E0F990000E121CF1901AD9E0FBA369
:10BAA900E0FAA3E0F9900011E4F5F012197B900097
:0BBAB90024E4F5F012197B123B8422FC
:0AC37800E0FBA3E0FAA3E0F97D1159
:0BC38200901AD0EBF0A3EAF0A3E9F062
:10C38D0012BA69EFB40111901AD0E0FBA3E0FAA341
:08C39D00E0F9E4FDFC12C09B75
:01C3A5002275
:08A2AC00E0FBA3E0FAA3E0F9D6
:10A2B400901AD2EDF0901ACFEBF0A3EAF0A3E9F0F4
:10A2C400900020121717B43C24901ACFE0FBA3E0AF
:10A2D400FAA3E0F9900028121B06EF2401FFE43EE4
:10A2E400FEE43DFDE43CFC900028121B50901ACF84
:10A2F400E0FBA3E0FAA3E0F9A3E0FD12BA69901A27
:10A30400D3EFF064017058901ACFE0FBA3E0FAA3F6
:10A31400E0F9E4FDFC12C09B901AD3EFF0D3648003
:10A324009480403B901ACFE0FBA3E0FAA3E02438EA
:10A33400F9E43AFA7D327C0012AD9E901ACFE0FB2C
:10A34400A3E0FAA3E0F9900034121B06EF2401FF06
:10A35400E43EFEE43DFDE43CFC900034121B5090CE
:04A364001AD3E0FF29
:01A3680022D2
:0B9B8100901AC5E0FBA3E0FAA3E0F996
:0B9B8C00901ACFEBF0A3EAF0A3E9F081
:109B9700901ACFE0FBA3E0FAA3E0F990000E121CA5
:109BA700C1901AD2EBF0A3EAF0A3E9F0901ACFE044
:109BB700FBA3E0FAA3E0F990001112189FFF901A97
:109BC700D5E5F0F0A3EFF090002412189FFF901A4C
:109BD700D7E5F0F0A3EFF07D1012BA69EFB40111E9
:109BE700901ACFE0FBA3E0FAA3E0F9E4FDFC12C072
:109BF7009B901ACFE0FBA3E0FAA3E0F99000207452
:109C07003C121789901AD2E0FBA3E0FAA3E0F9C04F
:109C170003C002C001901ACFE0FBA3E0FAA3E0F96A
:109C270090000E121CF1901AD5E0FCA3E0FD901AEB
:109C3700CFE0FBA3E0FAA3E0F9900011EC8DF0125E
:109C4700197B901AD7E0FDA3E0900024CD8DF01288
:029C5700197B77
:019C590022E8
:0BC22600901AC5E0FBA3E0FAA3E0F9CA
:10C23100900030121B06900034121B509000221205
:10C241001717901ACFB402057414F080037404F028
:08C25100901ACFE0FD12C38238
:01C2590022C2
:0FC8B1007E007F207D007B017A1C79270221CF3A
:0B851700901C96EBF0A3EAF0A3E9F043
:10852200901C9C74A5F01216FEFFC394E050030247
:10853200863FEFD394EF400302863F901C96E0FB08
:10854200A3E0FAA3E0F8AC02AD037B017A1C791F29
:108552007E007F041221ABEF700302863F901C96CF
:1085620012AE30901C99EBF0A3EAF0A3E9F04A6056
:108572001B901C99E0FBA3E0FAA3E0F990000674BB
:1085820001121744901C9C7402F0806912C18490FD
:108592001C99EBF0A3EAF0A3E9F04A6058E4FF90DB
:1085A2001C96E0FBA3E0FAA3E0F98F827583001228
:1085B2001717FE901C99E0FBA3E0FAA3E0F98F8263
:1085C200758300EE1217890FEFB404D3901C99E063
:1085D200FBA3E0FAA3E0F9900007E41217899000E8
:1085E20004E4F5F012197B900006740112178990C9
:1085F2001C9C7401F0901C9CE064017040901C99DA
:10860200E0FBA3E0FAA3E0F9128BA9901C9CEFF027
:10861200D364809480901C99E0FBA3E0FAA3E0F974
:10862200400512BDEC8016E4121777901C99E0FB0E
:10863200A3E0FAA3E0F9900006E4121789901C9CCB
:02864200E0FF57
:018644002213
:0BB6DB00901CABEBF0A3EAF0A3E9F039
:10B6E600A374A5F0901CABE0FBA3E0FAA3E0F8ACD2
:10B6F60002AD037B017A1C791F7E007F041221AB09
:10B70600EF603A901CAB12AE30E94A60309000060A
:10B716001217176028900007121717FF64016004BC
:10B72600EFB4021990000674FF1217449000061237
:10B7360017177003121777901CAE7401F0901CAEA9
:02B74600E0FF22
:01B7480022DE
:10777E00E4901AC3F012BC69901AB9EFF06411606C
:10778E0004E0B4120FC3901BC6E09408901BC5E032
:10779E0094005006901AC37401F0901AC3E060036F
:1077AE0002786912BC69901ABAEFF012BC69901A8D
:1077BE00BBEFF012BC69901ABCEFF0E4901AC1F066
:1077CE00A3F012BC69901AC1E0FCA3E024BDF582BF
:1077DE00741A3CF583EFF0901AC2E004F070069034
:1077EE001AC1E004F0C3901AC2E09404901AC1E0EA
:1077FE00940040CE901AB9E0FFA3E0FD7B017A1A07
:10780E0079BD129E06AD07AC06ECFF901ABBE0B533
:10781E000705A3E06D6002803C901AB9E0B4111820
:10782E0078D27C1B7D017B017A1C791F7E007F0440
:10783E001221ABEF6002801D901AB9E0B4121C78D1
:10784E00BD7C1A7D017B017A1B79D27E007F0412EA
:10785E0021ABEF6006901AC37401F0901AC3E0607A
:10786E000302791C901AB9E06411705E901AC1F08F
:10787E00A3F0901AC1E0FEA3E0FFC39404EE9400BF
:10788E00400302791CEF7803C333CE33CED8F924EC
:10789E0027F9741C3EFA7B01901AC4EBF0A3EAF0B0
:1078AE00A3E9F0900007121717B4020E901AC4E065
:1078BE00FBA3E0FAA3E0F912BDEC901AC2E004F0CB
:1078CE0070B0901AC1E004F080A8901AB9E064126A
:1078DE00703C7B017A1A79BD12AE38901AC4EBF067
:1078EE00A3EAF0A3E9F04A6025901AC4E0FBA3E0F6
:1078FE00FAA3E0F9900007121717B40111900007D0
:0E790E007402121789900004E4F5F012197B40
:01791C002248
:08AE3000E0FBA3E0FAA3E0F946
:0BAE3800901B31EBF0A3EAF0A3E9F05F
:10AE4300E4A3F0A3F0901B34E0FEA3E0FFC394045B
:10AE5300EE9400505EEF7803C333CE33CED8F9249B
:10AE630027F9741C3EFA7B01C003C002901B31E03A
:10AE7300FBA3E0FAA3E0F8AC02AD03D002D0037E5B
:10AE8300007F041221ABEF701A901B34E0FEA3E0A5
:10AE93007803C333CE33CED8F92427F9741C3EFA92
:10AEA3007B0122901B35E004F0709A901B34E00480
:09AEB300F080927B007A00790026
:01AEBC002273
:10BFDD00E4FDFCEDCEECCE7803C333CE33CED8F9F1
:10BFED002427F9741C3EFA7B01900007121717B431
:10BFFD00011490000412189F45F0600A900004741B
:10C00D00FFF5F012190F0DBD00010CED64044C701D
:01C01D00C260
:01C01E0022FF
:10B25B00E4901ABBF0A3F0901ABBE0FEA3E0FFC38F
:10B26B009404EE94005065EF7803C333CE33CED8FD
:10B27B00F92427F9741C3EFA7B01901AB8EBF0A362
:10B28B00EAF0A3E9F0900007121717B4012E901AF9
:10B29B00B8E0FBA3E0FAA3E0F990000412189F4575
:10B2AB00F07019128BA9EF6013901AB8E0FBA3E0B2
:10B2BB00FAA3E0F99000077402121789901ABCE008
:0CB2CB0004F07093901ABBE004F0808B3C
:01B2D7002254
:108BA900901AC174A5F0E94A7003028CB0C001E4BF
:108BB900901B3BF0A3F0A37402F0E4A3F0F9A3C95E
:108BC900F0A3F0A3E9F0E4A3F0A3F0D001FDFC12B7
:108BD9005292901ABDEFF0C3648094805003028CC6
:108BE900B0E0FF3395E0FE7C007D3D1217AB747B4E
:108BF9002FF974123EFA7B01A3EBF0A3EAF0A3E983
:108C0900F02404F9E43AFAE4FD7F12129E06901A60
:108C1900C3EEF0A3EFF0901ABEE0FBA3E0FAA3E0E5
:108C2900F9901AEEE4F0A37408F07D021269FFEFDF
:108C3900606D7F1212C78BE4FF12C78B901AC3E0D5
:108C4900FF12C78B901AC3A3E0FF12C78BE4901AD7
:108C5900C2F0901AC2E0FFC364809484502A901A2B
:108C6900BEE0FBA3E0FAA3E02404F9E43AFAEF3307
:108C790095E0FEE92FF9EA3EFA1216FEFF12C78BBC
:108C8900901AC2E004F080CA901ABEE0FBA3E0FA91
:108C9900A3E0F9E4FDFC12C09B901AC17401F090A5
:0C8CA9001ABDE0FF12A625901AC1E0FFE2
:018CB500229C
:10C18400E4FDFCEDAE047803C333CE33CED8F9FF1F
:10C194002427F582741C3EF583E0700B74272FF975
:10C1A400741C3EFA7B01220DBD00010CED64044CAD
:08C1B40070D17B007A007900D4
:01C1BC002260
:0B9E0600901AC7EBF0A3EAF0A3E9F00C
:109E1100EFFEEDFFE4FCFDA3121BBC901ACAE0F8B3
:109E2100A3E0F9A3E0FAA3E0FBC000C001C002C0B7
:109E310003901AC7E0FBA3E0FAA3E0F99000011236
:109E41001717FD1216FEFEEDFFE4FCFDD003D00254
:109E5100D001D000EB2FFFEA3EFEED39FDEC38FCDE
:109E6100901ACA121BBC901ACAE0F8A3E0F9A3E049
:109E7100FAA3E0FBC000C001C002C003901AC7E012
:109E8100FBA3E0FAA3E0F9900002121717FE90007D
:109E910003121717FDEDFFE4FCFDD003D002D00142
:109EA100D000EB2FFFEA3EFEED39FDEC38FC901AB5
:109EB100CA121BBC901ACAE0FCA3E0FDA3E0FEA3FA
:109EC100E0FF12B58D901ACA121BBC901ACAE0FCB1
:099ED100A3E0FDA3E0FEA3E0FF05
:019EDA002265
:0BBDEC00901AC7EBF0A3EAF0A3E9F007
:10BDF70012C8DCEE540FFE901C4AE07C002FFFECCB
:10BE07003ECF2401CF3400FED3EF94E8EE940340F5
:10BE1700047E037FE8901AC7E0FBA3E0FAA3E0F9EA
:10BE27009000077401121789900004EE8FF0021931
:01BE37007B8F
:10123200021543E86480F8E933E83360110460F092
:10124200ED33EC337009E8FCE9FDEAFEEBFF220422
:1012520060DED3EB9FEA9EE99DE8C2E78CF0C2F71D
:1012620095F0400CE8CCF8E9CDF9EACEFAEBCFFBE9
:1012720012150E85D0F05804700320D5B3E804701F
:10128200075002B2D502154D92D5EC0460F7E4CCBA
:10129200C0E0C398F8603B94186008400DD0E0FBB2
:1012A200021525E4FBFAC9FC8028E830E406E4C90B
:1012B200FBE4CAFCE830E305E4C9CACBFCE8540706
:1012C2006010F8C3E913F9EA13FAEB13FBEC13FC11
:1012D200D8F130F52FC3E49CFCEF9BFFEE9AFEEDB4
:1012E20099FDD0E0FBEF4E4D4C701222DB0302154C
:1012F2004AEC2CFCEF33FFEE33FEED33FDED30E72D
:10130200EB021525EF2BFFEE3AFEED39FDD0E0FBA7
:1013120050130BBB000302154DED13FDEE13FEEF50
:0813220013FFEC13FC0215257A
:10132A00EC4D6011E8497017ED33EC3304600DE4BD
:10133A00FCFFFEFD22E933E8330470F8021543127C
:10134A00150E58046009E4CC24815006285009027D
:10135A00154D28400302154AC0E0EB4A7044B98093
:10136A0006D0E0FB021539EF4E701CBD8008EBFF7A
:10137A00EAFEE9FD80EBE98DF0A4FEE5F002141324
:10138A00E9CDF9EAFEEBFFEF89F0A4FCE5F0CE899E
:10139A00F0A42EFFE435F0CD89F0A42DFEE435F05B
:1013AA008067EF4E7005BD80D780C3EF8BF0A4AC89
:1013BA00F0EE8BF0A42CFCE435F0F8EF8AF0A42CC4
:1013CA00E5F038FCE433CB8DF0A42CFCE5F03BF8D7
:1013DA00EE8AF0A42CFCE5F038F8E433CF89F0A4C7
:1013EA002CFCE5F038CF3400CE89F0A42FFFE5F0CD
:1013FA003EFEE433C98DF0A42EFEE5F039CD8AF025
:10140A00A42FFFE5F03EFEE43DFD33D0E0FB50079C
:10141A000BBB000F02154DEC2CFCEF33FFEE33FE35
:06142A00ED33FD02152563
:1014300002154DEC5D046005E85904700302154384
:1014400012150E580460F6EC4860F2EC7004FDFED4
:10145000FF22C860DB2481C85009C398600250068F
:1014600002154A9850CAF582E9294B4A7005AB82A9
:1014700002153975F0007C1A7880C3EF9BEE9AED67
:1014800099400DC3EF9BFFEE9AFEED99FDE842F007
:10149000DC23ACF0D0E0FFD0E0FED0E0FDAB82205A
:1014A000E7101BEB60BAEC2CFCEF33FFEE33FEEDE4
:1014B00033FD021525E803F830E705C0F075F000AC
:1014C000EF2FFFEE33FEED33FD40B830E7C280AAC8
:1014D00075F020800E75F010800575F0087D007E97
:1014E000007F003392D530D503121AABEC33401095
:1014F000EF33FFEE33FEED33FDEC33FCD5F0ED22A0
:0E150000E5F0247EA2D513CC92E7CDCEFF22DB
:10929700901A6A121BBC74FFFFFEFDFC901A6AE06D
:1092A700F8A3E0F9A3E0FAA3E0FBC3121ACF6038F2
:1092B7007F807E967D187C4B901A6AE0F8A3E0F9D0
:1092C700A3E0FAA3E0FB1215586002501B7F807ED3
:1092D700967D187CCB901A6AE0F8A3E0F9A3E0FA30
:1092E700A3E0FB121558500F901A6AE0FCA3E0FDAB
:1092F700A3E0FEA3E0FF22901A6AE0FCA3E0FDA32F
:10930700E0FEA3E0FF1215D1901A6E121BBC901A53
:109317006EE0FCA3E0FDA3E0FEA3E0FFEC1214D097
:10932700C8ECC8C9EDC9CAEECACBEFCB901A6AE040
:10933700FCA3E0FDA3E0FEA3E0FF121235E4FBFA75
:10934700F9F812155860264024901A6EE0FCA3E045
:10935700FDA3E0FEA3E0FFEF24FFFFEE34FFFEEDE9
:1093670034FFFDEC34FFFC901A6E121BBC901A6E92
:10937700E0FCA3E0FDA3E0FEA3E0FFEC1214D02283
:10150E00E9D2E7C933E833F892D5EDD2E7CD33EC23
:07151E0033FC5002B2D5229C
:10152500EC30E7100FBF000C0EBE00080DBD000427
:101535000BEB6014A2D5EB13FCED92E7FD2274FFD3
:10154500FCFDFEFF22E480F8A2D574FF13FC7D802C
:03155500E480EF40
:1015580074F8CC6480CCC86480C8F58204604FC33A
:10156800EB9FF5F0EA9E42F0E99D42F0E89C45F0D9
:10157800603C501DE5825FFFE582D313CB5BCBF463
:101588002B5582FB50280ABA002409B9002008808C
:101598001DE5825BFBE582D313CF5FCFF4C3132F26
:1015A8005582FF50090EBE00050DBD00010CC3EBAE
:1015B8009FF5F0EA9E42F0E99D42F0E89C45F06014
:0915C80007CC4820E701B3EC2236
:1015D100EDD2E7CD33EC3392D524814006E4FFFE12
:1015E100FDFC22FCE4CFCECDCC24E0501174FF8071
:1015F100EDC3CC13CCCD13CDCE13CECF13CF04700E
:07160100F030D5DE021AAB48
:10AD1E000291A4E493A3F8E493A34003F68001F216
:10AD2E0008DFF48029E493A3F85407240CC8C33336
:10AD3E00C4540F4420C8834004F456800146F6DF05
:10AD4E00E4800B010204081020408090BD54E47E84
:10AD5E00019360BCA3FF543F30E509541FFEE493FA
:10AD6E00A360010ECF54C025E060A840B8E493A3C1
:10AD7E00FAE493A3F8E493A3C8C582C8CAC583CAEC
:10AD8E00F0A3C8C582C8CAC583CADFE9DEE780BEA4
:01BD9F0000A3
:10160800E709F608DFFA8046E709F208DFFA803EC4
:1016180088828C83E709F0A3DFFA8032E309F608B1
:10162800DFFA8078E309F208DFFA807088828C8319
:10163800E309F0A3DFFA806489828A83E0A3F608CD
:10164800DFFA805889828A83E0A3F208DFFA804CA7
:1016580080D280FA80C680D4806980F2803380107E
:1016680080A680EA809A80A880DA80E280CA8033E7
:1016780089828A83ECFAE493A3C8C582C8CCC5835F
:10168800CCF0A3C8C582C8CCC583CCDFE9DEE7802F
:101698000D89828A83E493A3F608DFF9ECFAA9F0AE
:1016A800EDFB2289828A83ECFAE0A3C8C582C8CC04
:1016B800C583CCF0A3C8C582C8CCC583CCDFEADE1D
:1016C800E880DB89828A83E493A3F208DFF980CC7F
:1016D80088F0EF60010E4E60C388F0ED2402B40478
:1016E8000050B9F582EB2402B4040050AF2323451F
:0616F800822390165873D6
:1016FE00BB010689828A83E0225002E722BBFE02EA
:09170E00E32289828A83E493221C
:10171700BB010CE58229F582E5833AF583E0225087
:1017270006E92582F8E622BBFE06E92582F8E222D1
:0D173700E58229F582E5833AF583E49322EB
:10174400BB010FF8E58229F582E5833AF583E028A9
:10175400F0225009C58229F8E58226F622BBFE094B
:10176400C58229F8E22582F222F8EA2583F583E985
:0317740093282295
:10177700BB010689828A83F0225002F722BBFE0151
:02178700F3224B
:10178900F8BB010DE58229F582E5833AF583E8F096
:10179900225006E92582C8F622BBFE05E92582C842
:0217A900F2222A
:1017AB00EF8DF0A4A8F0CF8CF0A428CE8DF0A42E52
:0217BB00FE220C
:1017BD00BC000BBE0029EF8DF084FFADF022E4CC10
:1017CD00F875F008EF2FFFEE33FEEC33FCEE9DECD9
:1017DD00984005FCEE9DFE0FD5F0E9E4CEFD22ED1F
:1017ED00F8F5F0EE8420D21CFEADF075F008EF2F69
:1017FD00FFED33FD4007985006D5F0F222C398FD5A
:05180D000FD5F0EA22F6
:10181200C2D5EC30E709B2D5E4C39DFDE49CFCEEF1
:1018220030E715B2D5E4C39FFFE49EFE1217BDC395
:10183200E49DFDE49CFC80031217BD30D507C3E490
:061842009FFFE49EFE2260
:10184800C5F0F8A3E028F0C5F0F8E582158270022B
:061858001583E038F022C8
:10185E00A3F8E0C5F025F0F0E5821582700215833D
:06186E00E0C838F0E8229A
:10187400BB010A89828A83E0F5F0A3E0225006873F
:10188400F009E71922BBFE07E3F5F009E319228901
:0B189400828A83E493F5F07401932234
:10189F00BB0110E58229F582E5833AF583E0F5F087
:1018AF00A3E0225009E92582F886F008E622BBFE64
:1018BF000AE92582F8E2F5F008E222E5832AF583AA
:0818CF00E993F5F0A3E993226F
:1018D700BB010789828A83021848500B09C5F02784
:1018E700F7C5F01937F722BBFE0D09F8E325F0F32A
:1018F700C5F019E338F322F889828A8374019325A6
:08190700F0C5F0F8E49338226A
:10190F00BB010DC58229C582C5833AC5830218481C
:10191F005011C58229F808E5F026F618F5F0E58292
:10192F0036F622BBFE11C58229F808E225F0F5F044
:10193F00F218E23582F222F8E58229F582E5832A50
:0D194F00F58374019325F0F5F0E493382240
:10195C00BB010A89828A83F0E5F0A3F0225006F7D6
:0F196C0009A7F01922BBFE06F3E5F009F31922D3
:10197B00F8BB0111E58229F582E5833AF583E8F09E
:10198B00E5F0A3F0225009E92582C8F608A6F0225B
:0D199B00BBFE09E92582C8F2E5F008F22242
:0D19A800EF2BFFEE3AFEED39FDEC38FC228E
:0E19B500C3EF9BFFEE9AFEED99FDEC98FC222D
:1019C30075F008758200EF2FFFEE33FECD33CDCCDB
:1019D30033CCC58233C5829BED9AEC99E58298405E
:1019E3000CF582EE9BFEED9AFDEC99FC0FD5F0D63B
:1019F300E4CEFBE4CDFAE4CCF9A88222B800C1B965
:101A03000059BA002DEC8BF084CFCECDFCE5F0CBA2
:101A1300F97818EF2FFFEE33FEED33FDEC33FCEBDB
:101A230033FB10D703994004EB99FB0FD8E5E4F996
:101A3300FA227818EF2FFFEE33FEED33FDEC33FC83
:101A4300C933C910D7059BE99A4007EC9BFCE99A77
:101A5300F90FD8E0E4C9FAE4CCFB2275F010EF2FBC
:101A6300FFEE33FEED33FDCC33CCC833C810D707BC
:101A73009BEC9AE899400AED9BFDEC9AFCE899F8F7
:0E1A83000FD5F0DAE4CDFBE4CCFAE4C8F9228A
:0D1A9100EF4BFFEE4AFEED49FDEC48FC2254
:0D1A9E00CFF4CFCEF4CECDF4CDCCF4CC22DD
:0E1AAB00C3E49FFFE49EFEE49DFDE49CFC224C
:101AB900EB9FF5F0EA9E42F0E99D42F0EC6480C8A4
:061AC90064809845F02244
:101ACF00EB9FF5F0EA9E42F0E99D42F0E89C45F06D
:011ADF0022E4
:101AE000E8600FECC313FCED13FDEE13FEEF13FFE4
:031AF000D8F12208
:101AF300E8600FEFC333FFEE33FEED33FDEC33FC51
:031B0300D8F122F4
:101B0600BB010DE58229F582E5833AF583021B7454
:101B16005007E92582F80221FBBBFE07E92582F87A
:101B2600022207E58229F582E5833AF5830222132C
:101B3600BB010789828A83021BBC5005E9F8022291
:0A1B46004DBBFE05E9F8022259220A
:101B5000BB010DE58229F582E5833AF583021BBCC2
:101B60005007E92582F802224DBBFE07E92582F8DD
:041B700002225922D2
:0C1B7400E0FCA3E0FDA3E0FEA3E0FF22E4
:0C1B8000E0F8A3E0F9A3E0FAA3E0FB22E8
:101B8C00BB010DE58229F582E5833AF583021B80C2
:101B9C005007E92582F8022223BBFE07E92582F8CB
:101BAC00022230E58229F582E5833AF58302223D53
:0C1BBC00ECF0A3EDF0A3EEF0A3EFF0229C
:101BC800A8828583F0D083D082121BDF121BDF121C
:101BD8001BDF121BDFE473E493A3C583C5F0C58341
:101BE800C8C582C8F0A3C583C5F0C583C8C582C867
:011BF80022CA
:101BF900BB010DE58229F582E5833AF583021BC80D
:101C09005007E92582F8022265BBFE07E92582F81B
:041C190002227E2203
:0C1C1D00A42582F582E5F03583F58322D2
:091C2900E0FBA3E0FAA3E0F922BC
:101C3200F8E0FBA3A3E0F925F0F0E582158270023B
:071C42001583E0FA38F022DF
:091C4900EBF0A3EAF0A3E9F0229C
:101C5200BB010789828A83021C295005E9F8022206
:101C620097BBFE05E9F80222A989828A830222BB78
:101C7200BB011A89828A83D0F0D0E0F8D0E0F9D093
:101C8200E0FAD0E0FBE8C0E0C0F0021C495016E9DF
:101C9200F8D083D082D0E0F9D0E0FAD0E0FBC08265
:101CA200C0830222A0BBFE16E9F8D083D082D0E026
:0F1CB200F9D0E0FAD0E0FBC082C0830222B22258
:101CC100BB010DE58229F582E5833AF583021C29E2
:101CD1005007E92582F8022297BBFE07E92582F821
:101CE1000222A9E58229F582E5833AF5830222BB26
:101CF100BB0120E58229F582E5833AF583D0F0D056
:101D0100E0F8D0E0F9D0E0FAD0E0FBE8C0E0C0F0C4
:101D1100021C495018E92582F8D083D082D0E0F91D
:101D2100D0E0FAD0E0FBC082C0830222A0BBFE1843
:101D3100E92582F8D083D082D0E0F9D0E0FAD0E072
:091D4100FBC082C0830222B22221
:101D4A00D083D082F8E4937012740193700DA3A328
:101D5A0093F8740193F5828883E47374029368603C
:061D6A00EFA3A3A380DF3C
:101D7000E5112582F582E5103583F583B5100485DC
:101D800082112210AF06858211F51022858211F58D
:041D900010D2AF229C
:0D1D9400E5112582F582E5103583F58322E7
:101DA100E3F5F009E208B5F06D606B80F3E3F5F05F
:101DB10009E608B5F060605E80F387F009E608B5D2
:101DC100F054605280F487F009E208B5F0486046AB
:101DD10080F488828C8387F009E0A3B5F0386036FF
:101DE10080F488828C8387F009E493A3B5F027609F
:101DF1002580F388828C83E3F5F009E0A3B5F01622
:101E0100601480F388828C83E3F5F009E493A3B531
:101E1100F004600280F2021ECC808580E7808E8013
:101E2100D2803C8015806C807E809B80B5808B80C9
:101E3100A1804F8070803A021ED889828A83ECFA91
:101E4100E493F5F0A3C8C582C8CCC583CCE493A3C1
:101E5100C8C582C8CCC583CCB5F070606E80E189FD
:101E6100828A83E493F5F0A3E208B5F05E605C80BA
:101E7100F289828A83E0F5F0A3E608B5F04D604B64
:101E810080F389828A83E0F5F0A3E208B5F03C6033
:101E91003A80F389828A83E493F5F0A3E608B5F0EA
:101EA1002A602880F2805389828A83ECFAE493F5D0
:101EB100F0A3C8C582C8CCC583CCE0A3C8C582C87D
:101EC100CCC583CCB5F004600280E27FFFB5F0029F
:101ED1000F2240027F012289828A83ECFAE0F5F029
:101EE100A3C8C582C8CCC583CCE0A3C8C582C8CC71
:101EF100C583CCB5F0D560D380E389828A83ECFABF
:101F0100E0F5F0A3C8C582C8CCC583CCE493A3C8CF
:101F1100C582C8CCC583CCB5F0B160AF80E288F092
:101F2100ED2402B4040050A3F582EB2402B40400B2
:0B1F310050992323458223901E1A7351
:101F3C00E709F60870FA8046E709F20870FA803E65
:101F4C0088828C83E709F0A370FA807EE309F60897
:101F5C0070FA8076E309F20870FA806E88828C83BE
:101F6C00E309F0A370FA806289828A83E0A3F60801
:101F7C0070FA805689828A83E0A3F20870FA804A4C
:101F8C0080D280FA80C680D4806580F28031801047
:101F9C0080A680EA809A80A880DA80E280CA8031AC
:101FAC0089828A83ECFAE493A3C8C582C8CCC58322
:101FBC00CCF0A3C8C582C8CCC583CC70E9800D8990
:101FCC00828A83E493A3F60870F9ECFAA9F0EDFB8E
:101FDC002289828A83ECFAE0A3C8C582C8CCC58367
:101FEC00CCF0A3C8C582C8CCC583CC70EA80DD898F
:101FFC00828A83E493A3F20870F980CE88F0ED24F2
:10200C0002B4040050C4F582EB2402B4040050BAAC
:09201C002323458223901F8C73DD
:10C7E700E4FFFE1216FE600C0FEF70010E09E970F0
:05C7F700F20A80EF22B0
:10202500E3F5F009E208B5F06BDFF58067E3F5F05D
:1020350009E608B5F05EDFF5805A87F009E608B5D0
:10204500F052DFF6804E87F009E208B5F046DFF67C
:10205500804288828C8387F009E0A3B5F036DFF6ED
:10206500803288828C8387F009E493A3B5F025DF5D
:10207500F5802188828C83E3F5F009E0A3B5F0149F
:10208500DFF5801088828C83E3F5F009E493A3B52E
:10209500F002DFF4022154808780E9809080D480AB
:1020A5003E8015806E807E809D80B7808D80A38068
:1020B500518074803C02216089828A83ECFAE49322
:1020C500F5F0A3C8C582C8CCC583CCE493A3C8C525
:1020D50082C8CCC583CCB5F076DFE3DEE1807089BC
:1020E500828A83E493F5F0A3E208B5F062DFF48019
:1020F5005E89828A83E0F5F0A3E608B5F051DFF545
:10210500804D89828A83E0F5F0A3E208B5F040DFCF
:10211500F5803C89828A83E493F5F0A3E608B5F05F
:102125002EDFF4802A8002805789828A83ECFAE4C4
:1021350093F5F0A3C8C582C8CCC583CCE0A3C8C5B8
:1021450082C8CCC583CCB5F006DFE4DEE280007F33
:10215500FFB5F0020F2240027F012289828A83ECBB
:10216500FAE0F5F0A3C8C582C8CCC583CCE0A3C806
:10217500C582C8CCC583CCB5F0D5DFE5DEE380CF1D
:1021850089828A83ECFAE0F5F0A3C8C582C8CCC57C
:1021950083CCE493A3C8C582C8CCC583CCB5F0AFC6
:1021A500DFE4DEE280A988F0EF60010E4E60ABED62
:1021B5002402B404005098F582EB2402B4040050C4
:0A21C5008E232345822390209C7393
:1021CF00EF4E6012EF60010EEDBB010B89828A8327
:1021DF00F0A3DFFCDEFA2289F05007F709DFFCA934
:0C21EF00F022BBFEFCF309DFFCA9F0228B
:0C21FB00E6FC08E6FD08E6FE08E6FF2210
:0C220700E2FC08E2FD08E2FE08E2FF2213
:10221300E493FC740193FD740293FE740393FF2211
:0D222300E6FB08E6F908E6FA08E6CBF8222B
:0D223000E2FB08E2F908E2FA08E2CBF8222E
:10223D00E493F8740193F9740293FA740393FB22F7
:0C224D00ECF608EDF608EEF608EFF622BD
:0C225900ECF208EDF208EEF208EFF222C1
:10226500D083D082E493F608740193F60874029340
:09227500F608740393F674047377
:10227E00D083D082E493F208740193F2087402932F
:09228E00F208740393F274047366
:09229700E6FB08E6FA08E6F9226C
:0922A000EBF608EAF608E9F62263
:0922A900E2FB08E2FA08E2F92266
:0922B200EBF208EAF208E9F2225D
:0C22BB00E493FB740193FA740293F9227F
:00000001FF
